:020000040000FA
:100000000204040000000000F03800003238000054
:10001000583800007E380000A4380000CA380000BC
:10002000F0380000F0380000F0380000F038000030
:10003000F0380000F6320000F0380000F038000020
:10004000F0380000F0380000F0380000F038000010
:10005000F0380000F0380000F0380000F038000000
:10006000F0380000F0380000F0380000F0380000F0
:10007000F0380000F0380000082A0000F0380000D6
:10008000F0380000F0380000F0380000F0380000D0
:10009000F038000018350000F0380000F03800009B
:1000A000F0380000F0380000F0380000F0380000B0
:1000B000F0380000F0380000F0380000F0380000A0
:1000C000F0380000F0380000F0380000F038000090
:1000D000F0380000F0380000F0380000F038000080
:1000E000F0380000F03800007C370000F0380000E5
:1000F000F0380000F0380000F0380000F038000060
:10010000F0380000F0380000F0380000F03800004F
:10011000F0380000F0380000F0380000F03800003F
:10012000F0380000F0380000F0380000F03800002F
:10013000F0380000F0380000F0380000F03800001F
:10014000F0380000F0380000F0380000F03800000F
:10015000F0380000F0380000F0380000F0380000FF
:10016000F0380000F0380000F0380000F0380000EF
:10017000F0380000F0380000F0380000F0380000DF
:10018000F0380000F0380000F0380000F0380000CF
:10019000F0380000F0380000F0380000F0380000BF
:1001A000F0380000F0380000F0380000F0380000AF
:1001B000F0380000F0380000F0380000F03800009F
:1001C000F0380000F0380000F0380000F03800008F
:1001D000F0380000F0380000F0380000F03800007F
:1001E000F0380000F0380000F0380000F03800006F
:1001F000F0380000F0380000F0380000F03800005F
:10020000FFFFFF00FFFFFF00F03800003238000062
:10021000583800007E380000A4380000CA380000BA
:10022000F0380000F0380000F0380000F03800002E
:10023000F0380000F6320000F0380000F03800001E
:10024000F0380000F0380000F0380000F03800000E
:10025000F0380000F0380000F0380000F0380000FE
:10026000F0380000F0380000F0380000F0380000EE
:10027000F0380000F0380000082A0000F0380000D4
:10028000F0380000F0380000F0380000F0380000CE
:10029000F038000018350000F0380000F038000099
:1002A000F0380000F0380000F0380000F0380000AE
:1002B000F0380000F0380000F0380000F03800009E
:1002C000F0380000F0380000F0380000F03800008E
:1002D000F0380000F0380000F0380000F03800007E
:1002E000F0380000F03800007C370000F0380000E3
:1002F000F0380000F0380000F0380000F03800005E
:10030000F0380000F0380000F0380000F03800004D
:10031000F0380000F0380000F0380000F03800003D
:10032000F0380000F0380000F0380000F03800002D
:100800000A0000006F4323000E7F23000E018800C2
:10081000000000000C000700A0AA2E00010020002C
:1008200011000700000020000000E000020032007C
:1008300000000200000000008269020000000000C9
:100840000040DA000000FE004440A900C01E240061
:100850000000E0000300320020002000A00188001A
:100860004440A80000000600910188008000780044
:100870000000EB0015003700E280400032A0B40019
:100880009101BA00E280400032A0B4009102BA00A7
:10089000E280400032A0B4000002EB00472BDE00F3
:1008A000F507B200602CE10004003A000059EB00AB
:1008B0008301E900FDFF3E00040037006128E100EC
:1008C000010032000082EB00040007001101BA00B1
:1008D0000200E000E8FF3A00000006003159BA00CB
:1008E0008301E9000C0032002159BA008301E900BC
:1008F000080032000400E00003003A00E2804000FB
:1009000032A0B400F5FF370011D9BA008301E90025
:10091000FAFF3A008100E800E180400032A0B40014
:10092000000006007C69040000000000AA300400FA
:10093000000000003C30040000000000C42F040050
:10094000000000006E3004000000000014300400BD
:1009500000000000B02F0400000000005A30040026
:100960000000000000300400000000009C2F040084
:10097000000000004630040000000000EC2F0400DE
:1009800000000000A62F040000000000503004000A
:1009900000000000F62F040000000000BE3004003C
:1009A00000000000A030040000000000E22F04005E
:1009B000000000008C300400000000003230040011
:1009C00000000000CE2F040000000000783004007A
:1009D000000000001E30040000000000BA2F0400D8
:1009E0000000000064300400000000000A30040031
:1009F0000000000040310400000000004A31040003
:100A000000000000742F040000000000D42E040039
:100A100000000000DE2E040000000000FC2E040098
:100A200000000000F431040000000000FE3104006A
:100A300000000000062F0400000000007E2F0400CC
:100A400000000000602F040000000000562F04008A
:100A5000000000002E2F040000000000F22E040011
:100A600000000000242F0400000000006A2F040092
:100A7000000000001A2F040000000000102F0400E6
:100A800000000000422F040000000000B831040004
:100A900000000000382F0400000000004C2F04006C
:100AA00000000000E0310400000000005E3104009E
:100AB0000000000036310400000000007C3104001A
:100AC000000000000E31040000000000E6300400C9
:100AD000000000009A3104000000000054310400BE
:100AE00000000000EA31040000000000683104004A
:100AF00000000000FA30040000000000D2300400C2
:100B00000000000086310400000000009031040065
:100B1000000000000431040000000000DC3004008C
:100B200000000000A431040000000000F0300400C8
:100B300000000000C830040000000000B4300400D1
:100B400000000000D63104000000000072310400F3
:100B5000000000002231040000000000CC3104003D
:100B600000000000C231040000000000AE310400AB
:100B7000000000001831040000000000D82F04001D
:100B80000000000082300400000000002830040053
:100B9000000000007C8C0400000000008A85040036
:100BA00000000000D2950400000000002697040019
:100BB000000000009696040000000000F696040075
:100BC000000000006C8C040000000000DE930400B4
:100BD000000000009AB304000000000056850400E5
:100BE000000000009C950400000000009C8F0400A1
:100BF00000000000B08B0400000000002A71040017
:100C0000000000002495040000000000E4940400AB
:100C10000000000086980400000000001096040008
:100C200000000000BAB3040000000000D6940400E5
:100C3000000000001EAC040000000000188C04003E
:100C400000000000FE8F0400000000006297040016
:100C5000000000005692040000000000E08F040035
:100C600000000000DA8F04000000000070B30400F0
:100C70000000000086B30400000000005697040046
:100C800000000000E893040000000000E2AA040055
:100C900000000000A08C040000000000C88C0400CC
:100CA000000000008C8C040000000000B48C0400E4
:100CB00000000000AA8C040000000000D28C040098
:100CC00000000000968C040000000000BE8C0400B0
:100CD0000000000004930400000000002A930400B8
:100CE000000000004C8D0400000000001004B10062
:100CF000070035009001B100040034007000B1001D
:100D0000030035009001B10001003C001000050017
:100D100000000500800078001106B10003003500D6
:100D20009101B10001003C000050A100000006004C
:100D30000A00FA0080017800E20F500028003E000F
:100D4000A0A18100E10F50000800320080232000A4
:100D50000000E000050032000423200025232000CD
:100D60004623200080017800040037000422200080
:100D700025222000462220008322200014409000DB
:100D80000004E000040035008009EB0014409000EE
:100D90000074A00010429800154090000028A300A5
:100DA00003003A00154090000024A00090429800F3
:100DB0008001EB0007003700154090000008A300F9
:100DC000FDFF320063C078000000FB00000B7800DC
:100DD0008301E800828F5100F7FF3A0008003700D6
:100DE00030002000B0BF9F00C3BF9F00D1BF9F0055
:100DF000E2BF9F006A80570000C0DA006FB9970019
:100E0000020078000080FA0000000600020AB90023
:100E1000001BB9000200B8008100420081004300BD
:100E200000000600889FBE008A9FBE008C1F7800CD
:100E3000B5010700BC01330003866C006450E1007B
:100E40002E0032006420E100330032006150E100E6
:100E50002F0032006120E10031003200858555000D
:100E6000EB07B0000900200008042000050037004F
:100E70000804440089844C000A0031000603430042
:100E800087834B000001530081815B00F8FF330032
:100E90000203BE000800A0000804440089844C003E
:100EA000F6FF3900C639DD0083017300010032000E
:100EB000130020008904D1000884D3000998A300FE
:100EC000050032000800A7000300A0008904D1003B
:100ED0000884D3008B05E8008904D1000884D3007E
:100EE0000001EB000281D2009F01070001F0A10088
:100EF0000CF0A70001F0A000940137006420E1008D
:100F0000960132000801BE000200BE00F7FF370064
:100F10006120E100910132006000B800F3FF37006A
:100F20000000200001F82700F0FF3700889FBE0076
:100F30008A9FBE008C1F7800730107007A0133007E
:100F400003866C006450E100240032006420E1005C
:100F5000270032006150E100220032006120E100F0
:100F6000210032008B854200EB07B1000134B8004C
:100F7000003AB8000804420089844A00013AB800E7
:100F80000030B8008880400009014A0004003300A6
:100F90000000400081804800020149008B05E90003
:100FA000C909DD0083017000010032001300200038
:100FB000C814DE004814DD004709DE001200B2004C
:100FC000C808DE00088470006701070001F0A10076
:100FD0000CF0A70001F0A0005C0137006120E100E7
:100FE0005E0132000801BE000200BE00F7FF3700BC
:100FF0006150E100FCFF3A005801370003F0A20005
:10100000889FBE008A9FBE008C1F78003E010700AB
:10101000450133006450E1004F0032006420E100DC
:101020005200320003826C0007003B000905D0002B
:101030000306D000820F54000C065D000200390048
:10104000020032008901780003067800858255008D
:1010500004003D000003FD008103FD008502EA005D
:101060008B854200840F720002003B00600010007C
:10107000E08018006011B8000005EB007A28E1005C
:101080000A00390006007800C75DDD00F707B200EE
:10109000878075002D003700828171000A01780079
:1010A000610560008180D1000080D3008502E900E5
:1010B000F9FF3B00060440008784480002003B0023
:1010C00060041400E0841C000988A30007003200BB
:1010D0008A81710082817100610164008904D100FC
:1010E0000884D3008B05E800170037000978A300B7
:1010F00013003A000B00E000130034008B05E900F8
:101100000804440089844C000A4474000978A30050
:101110000D003A000B00E000070034008B05E900E9
:101120000804440089844C0001003A000B002000B0
:101130000978A300F7FF32000001EB00020037003E
:10114000828171000A017800070107000CF0A700F6
:1011500001F0A000FD0037006420E10002003A0029
:10116000838F6C00FD0033000801BE000200BE004A
:10117000F6003700889FBE008A9FBE0001057800F8
:101180000100E0000400350008003C000000E00021
:10119000200032000500370060001000E0801800D9
:1011A00002003B0001F02C001A0037000004BE00D2
:1011B0006011B8006B0920000982CF0002003900DD
:1011C0000882CF000441B000694252000E00320094
:1011D00008003B0082817100610164008904D10034
:1011E0000884D3008B05E8000442E800F9FF3A00C8
:1011F000050037000804440089844C008B05E90091
:101200000442E900FBFF3A00D70007000AF0A700FC
:1012100001F0A0004F05BE004F04BE000000060014
:101220000001BE00F60007000470A70003F0A10053
:101230006509B100160032000D0035006828E10094
:1012400006003500F0FF2F00F1FF27000300E0004B
:1012500013003B00010028000000050000004000D2
:10126000818048008502E900FCFF3A000800370051
:10127000F88F420002003C008000EB0000000500F7
:101280008100D1000080D3008502E800FCFF3A0015
:101290000300E00002003B0060001000E080180046
:1012A0000000060014002000EA003700889FBE00FE
:1012B0008A9FBE008C1F78000004BE00D00007008B
:1012C0000478A30026003A006120E10025003200E6
:1012D00009F8A30025003A006420E1002100320053
:1012E000F507B1000508A30002003200000040002D
:1012F000818048006044B8000310200002002000F4
:1013000000004000818048000805440089854C00A9
:101310000A0541008B8549000A0550008B8558005D
:10132000030033000A00BE000204740083847400CA
:101330008301D1000281D300830F7100F0FF3A00D6
:101340008904D1000884D30060014900820178003B
:10135000C1ADDE00FB07B000830007007B00370053
:101360000960A0000800BE007800370012022000CB
:1013700002408800F0FF2F00F1FF270073003700C4
:1013800004002000B3003700F4FF2F00B100370045
:1013900004002000CA003700889FBE008A9FBE005C
:1013A0008C1F7800580007001002200002003B004C
:1013B000004088005C0037008A0062006408E10099
:1013C00002003A0000408800640037006108E10034
:1013D000FCFF32000800BE000304780091FE070005
:1013E00001F0A1000501070008F0A6000400370085
:1013F0000001BE0091042400B0FD2000FFFE0700A4
:1014000009F0A70001F0A2005000370060010700BA
:1014100092BD2500E3ED2300C4FE37000001BE00AD
:10142000770007000470A70003F0A10003F8A300F1
:1014300013003A006509B1001000320009003500C0
:101440006928E100020035000100280000000500C5
:1014500000004000818048008502E900FCFF3A005E
:1014600000000600F88F4200050035008100D10021
:101470000080D3008502E800FCFF3A00000006006F
:101480008000EB0000000500839F68000100E00081
:1014900002003D0060001000E08018000300E00042
:1014A00002003D0060011100E08119008F0107007A
:1014B0004F00E00002003B0060001000E0801800D8
:1014C000000006000081EB0098013700811F7800C2
:1014D0000100E00002003D0060001000E080180004
:1014E0000300E00002003D0060011100E0811900EE
:1014F000F70107004F00E00002003B006000100011
:10150000E0801800000006000004BE003C00070058
:101510000003BE000405BE000200BE003800070044
:10152000844F7500000006000200BE006450E10018
:10153000050036006420E100020036000968A300BF
:1015400001003A000800BE000160A0004F067800CC
:101550004F05BE004F04BE0000000600F0FF2F0044
:10156000F1FF2700F9FF370081002000618055005E
:101570000B003D000B00200061FE2F000100E10088
:101580001D00340082817100610164008904D10072
:101590000884D3000000E800FAFF3A007100200040
:1015A0006100640003007000020060000900320066
:1015B00061044400E0844C000988A5000500320065
:1015C0008B05E8006808E10002003A008904D100B8
:1015D0000884D300F20F20000258E10005003D000E
:1015E000C75DDD00F907B20089807500080078004A
:1015F000000006000BF827008B00780000000500B3
:10160000C70ADE00F107B200F50FB2000800320091
:10161000E1CF4200020032000170A000240005006A
:10162000810F70000100320004080500440005002D
:10163000810F700002003A00140005008502E900E5
:101640000000400081C04800FCFF3B000170A0008A
:1016500024000500889FBE008A9FBE00841F78007A
:10166000A9FF07004F00780011003300F0FF2F00A2
:10167000838F6C0006003B00040565000A00A7008C
:101680000800370009F0A60010002000080037000D
:10169000820F5400838F5C0003003900100020008B
:1016A00001003E000000200009F0A7000000EA0051
:1016B0004F05BE004F04BE000000E0000000060021
:1016C000889FBE008A9FBE008C1F78004F26DD00D9
:1016D0008DFF070094FF33006120E10043003200DA
:1016E0006250E10041003E003E0039006420E1000C
:1016F0003C003200058255000F003B000402E80068
:1017000038003A00800F5300818F5B0035003400B1
:101710000800BE0003F0A10001F0A60003F0A00045
:101720000CF0A70036FE070088FF370006034300D1
:1017300087834B000C4646000005530081855B0003
:10174000020033000A03BE000C00A0000402E900FE
:10175000F6FF3B00850578000602430087824B00B8
:1017600004003A006000B80009F0A70001F0A000F2
:1017700076FF37000002520081825A000704E00021
:10178000040033000603430087834B008B05E90008
:10179000FAFF3700090578000604BE000203BE0008
:1017A0006011B80070FF0700E00F5200E08F5A0090
:1017B0000700350002003C000C08A30004003200C2
:1017C0000601BE0003F0A0000CF0A7000CFE07000D
:1017D0000A85680001F0A1000AF0A70001F0A0004E
:1017E0005AFF37000800BE0058FF370010022000E3
:1017F0000CF0A6000040880058FF3700889FBE000C
:101800008A9FBE008C9FBE000004BE007CFF0700C4
:101810000800BE00890678006420E1000800390055
:10182000040032000160A000120220000240880083
:101830005300370091FC2300B0FD20004E0037001C
:101840000006EB0009F0A10003F8230002002000CD
:101850000800BE0093FE07000600340001F82300D4
:10186000000020000801BE006EFD07000004BE005D
:101870002C0020000800BE0093E82300320A230059
:1018800088FE0700120034000801BE00D1FD2300CD
:10189000703D2B00DAFD07000005BE00B3F3230006
:1018A000F27A26000800BE00A0FD070003F823001E
:1018B00002002000D1FD07000801BE00D0FD070096
:1018C0000A01BE0057FD07000004BE000C06E80038
:1018D0000800BE0001F0A1000200200003982300D0
:1018E00070FE07000800BE00160035000801BE00AB
:1018F0008EFD07000005BE0032CD2C0043FB230007
:10190000BFFD0700809FBE001269280003D52B0091
:101910000A00BE0085FD0700620F210013EF2B00B7
:10192000B7FD07000A01BE0080FD07004F01BE00A1
:101930003CFD07000801BE007CFD07000801BE0059
:10194000AFFD07000C00E0000B0032000C10A700F8
:1019500001F0A200B2FD200093FC23006260E100D0
:101960000400320022A9200063F023000C10A7001D
:1019700063F82300A2FD07000DF0A70001F0A2000C
:101980004F06BE004F05BE004F04BE00000006001B
:10199000889FBE008A9FBE008C9FBE00CF000700BC
:1019A000850478000005BE006420E10049003E0087
:1019B0006220E10003003200090035000BF8A300AB
:1019C000440032000BF8A30008003200100220008F
:1019D00000408800F0FF2F00F1FF27003D00370096
:1019E00001F82F00000020003A0037003D000700FA
:1019F00082FD07000006BE000A00BE00324F200034
:101A000053F3230060FE0700060034000C00BE0004
:101A10003400070079FD07000006BE000A00BE0082
:101A2000020037008904E9000C00BE002D00070009
:101A30003EFD07002B00070071FD07000001BE00FE
:101A40000C00BE00F7FC07000005BE000001BE0050
:101A500036FD07000006BE00A2F32300430D2C0054
:101A600067FD0700809FBE000C00BE00D2E3270088
:101A7000D3F02B002DFD07004F01BE00E9FC07004D
:101A80000006BE000A01BE0028FD07000A01BE00D4
:101A90005BFD07000006BE006148B900B5FD070008
:101AA0000005BE0032082800E3952B001FFD07004B
:101AB0000C01BE0052FD07000006BE000A00BE0079
:101AC0000200280013F3230018FD07000C01BE00DC
:101AD0004BFD07004F06BE004F05BE004F04BE0081
:101AE0000000060003F02300020005006022B80099
:101AF000060220000000D0008180D2000482D200C3
:101B00008582D2000000A0000202520083825A00A7
:101B1000030031000202420083824A000000A1005B
:101B20000603E900F3FF3A0000000600889FBE00AC
:101B30008A9FBE008C9FBE00820578000004BE0014
:101B4000AFFE07000800BE006420E1000700390076
:101B500002003A00F1FF2700F0FF2F000160A00013
:101B60001202200002408800550037006120E10089
:101B700003003A000B00A70001F8230050003700D3
:101B800001F0A1000200210093642400C5FD0700BC
:101B90000800BE0004003500B2FD2000930C2400B4
:101BA000FBFD07000004BE000005EB000B00A600D3
:101BB0004F0DDE0001F0A1000004BE0032982F009E
:101BC00023EA2300D9FC07000001EB0003F0230007
:101BD0000B00A70003F8230009FD070090FD070094
:101BE0000000A7000A00A20062FD07000B00E00051
:101BF000030032000200200003F02300FFFC070076
:101C000001F0A2000006BE000200200093042400A0
:101C1000C6FC07000801BE00F9FC0700809FBE005B
:101C20000C00BE0022A22A00D3A72300BFFC07009D
:101C30004F01BE00F2FC07000004BE0001F0A1004D
:101C4000020020000398230096FD07000800BE0054
:101C5000190035000001BE00B4FC07000006BE00FC
:101C6000B2C52900E3622300B0FC070022222B004A
:101C7000F3942B00E2FC07000C01BE00ABFC070054
:101C8000E273280083C02300DDFC07000C01BE00C6
:101C9000A6FC070042AA2A00A3E22B00D8FC0700FA
:101CA0000C01BE00A1FC07000801BE009FFC07005C
:101CB0000801BE00D2FC07000A00A70001F0A20044
:101CC0004F06BE004F05BE004F04BE0000000600D8
:101CD00086FF07000400BE00000006000003BE00EF
:101CE00047FE07006220E100020032000600BE004D
:101CF00005000500E507B100F107B20004F023007C
:101D00008480700007F0A70001F0A0002400050007
:101D1000881F7800000478005001BE004000BE001B
:101D20000400400085804800060149008781490081
:101D3000009CBE000294BE000400E1000588E100A2
:101D40000690E1000798E1000200310068004400BD
:101D50001008E8004F04780000000600F4874700F0
:101D6000889FBE008A9FBE008C9FBE008E1F780099
:101D70000205BE000004BE00D4B79F00E5B79F0077
:101D8000F6B79F0087BF9F000000EB00C0B79F0021
:101D9000B0B79F00A0B79F0090B79F0080B79F008B
:101DA0000D042000BFB097004FB097000001400025
:101DB0000000E0000F003D004F08DE000000710051
:101DC000C0B79F009E00070001003D0012002000E8
:101DD000A100070001003D0012002000A60007003E
:101DE000B1000700B60007000F004000C8FF070061
:101DF000220037004F08DE0000067100CCB79F00BC
:101E00008F00070001003D00120020009200070033
:101E100001003D001200200097000700A20007000B
:101E20000FB297009FB297002FB39700BFB39700F0
:101E3000A90007000000520081805A0002015B00E7
:101E400083815B0080B79F0091B79F00A2B79F007E
:101E5000B3B79F000007EB009F0007000020E100E0
:101E600001A8E10002B0E10003B8E1000100310087
:101E70001E0020000E005600C0B79F004FB2970012
:101E80000400E000070035001000200001002000E1
:101E90006011B80008047000898470000A057100A0
:101EA0008B8571008D06E900BEFF3A000400E0005A
:101EB00003003D00820007000F00400094FF070070
:101EC0004FA897000000E00004003A000FB497000C
:101ED0009FB497002FB59700BFB5970094000700F7
:101EE0004F0778004F06BE004F05BE004F04BE00EE
:101EF0004F01B10000000600881F78001800200084
:101F0000881F780095FF07008F87E9004F0478004D
:101F100000000600801FEB0090FF07008F87E9009C
:101F200000000600889FBE008A9FBE008C1F7800BC
:101F30006E00070007003D0073000700E00F5B0024
:101F4000E08F5B0007003D00320007000006EB0059
:101F5000040037003400070002003D002A0007009B
:101F60001C00200072000700E3FF07000203BE0010
:101F70000002BE000C00E000010032002200070059
:101F80000400BE000601BE004F0678004F05BE00EB
:101F90004F04BE0000000600889FBE008A9FBE005E
:101FA0008C1F78005100070005003D005600070017
:101FB000E00F5B00E08F5B0006003D00040037008F
:101FC0001900070003003D006000B8006011B80070
:101FD0001000070056000700CEFF07000203BE00F6
:101FE0000002BE000C00E000010032000600070005
:101FF0000400BE000601BE004F0678004F05BE007B
:102000004F04BE00000006006000B8006011B80078
:102010000000370004025000858258000603590072
:1020200087835900000006000006EB00E00F520015
:10203000E08F5A00E00F5B00E08F5B0000000600BD
:102040000180400090B79F000001EB008FB0970027
:102050000100E000000006000200700090B79F0041
:102060000180400080B79F000001EB00FFA89700AF
:102070000100E000000006000200700080B79F0031
:10208000018040006FAA9700CF20DE0001007000A1
:10209000F0AF9F0004024200250007004F18DE0049
:1020A0000002720000000600E4AF9F000804440034
:1020B00089844C000A054D008B854D000000060008
:1020C0003FB29700CFB297005FB39700EFB397008E
:1020D00000FE2F00000006003FB09700CFB0970031
:1020E0005FB19700EFB19700000006000205BE0047
:1020F0000004BE00E00F5000E08F5800E00F5900D0
:10210000E08F5900000006006000B8006011B800C0
:1021100008045000898458000A0559008B8559002D
:102120001C002000E00F5200E08F5A000000060063
:102130000800BE000A01BE00000006002800FA00E8
:10214000889FBE008A9FBE008C9FBE0003866B00E6
:102150000C0207000028A30064003A000128A30035
:1021600067003A000008A30062003A000108A300DB
:1021700065003A001E009000BE08900081064000F5
:10218000ED3FB100F4805700EE019000111AB80045
:102190008E099000311BB8009E099000311CB800D8
:1021A000511DB800F485570046000700FE0190005D
:1021B0003A0007008B85E8003E0007008E0990007A
:1021C00040000700EE019000340007008B85E80016
:1021D000380007008E099000400007009E0990001B
:1021E0001B18B800890440000A854800FE019000D1
:1021F000340007008B85E80038000700EE019000EE
:10220000300007008E0990001B18B80089044000B8
:102210000A8548000A98A30008003A000402420018
:1022200085824A0006034B0087834B0008044C005C
:1022300089844C000A054D008D06E90084827200F5
:10224000850273004C3ADD00850272000100320005
:1022500015002000443ADE001400B2004538DE00CC
:10226000CB45DD000B007000C540DE00CB4DDD002E
:102270008B8070004549DE00CB55DD000B017100FD
:10228000C551DE000D037800D701070003F0A1005F
:102290000CF0A70003F0A000CE0137001B18B80017
:1022A0008502400006834800E0834B0060044C0038
:1022B000070037001B18B80006034000878348005A
:1022C000FAFF37001B18B800870340000884480055
:1022D000E0844C0060054D00000006001B18B800AB
:1022E0000804400089844800FAFF37000108A30071
:1022F000B5013A005800BE005801BE00E3FF3700A8
:102300000008A300B0013A0009047800F9FF370083
:1023100081037800BAFC07000001BE006000B8002D
:102320000478A30013003A006220E10015003E008B
:102330000D0039008301D1000281D3008180D300D8
:102340008301D1000281D3008180D3008301D100B9
:102350000281D3008180D3000538B000C42ADD009B
:10236000F300B2008381720007F0A70003F0A00021
:1023700000000600F3FF2700F2FF2F006110B900F4
:10238000FBFF370003FF2700F7FF37008F1FD10047
:10239000C10107008F87E9000000E000000006008F
:1023A000801FEB00BC0107008F87E9000000E00000
:1023B000000006001400FA00889FBE008A9FBE003D
:1023C0008C9FBE000005BE000206BE0068004700EC
:1023D0000C90BE000A90BE00D80107006400E10026
:1023E0001A00320016003E006100E1001A003200BF
:1023F0006E049000FE0490000E0B90009E0B900067
:102400006011B8009E0590000B38B100D501200086
:1024100082817100610164008703D1000683D300CB
:102420008984D3000884D3008502E900F8FF3A00CC
:102430004DFC07000DF0A70001F0A000650137007A
:10244000F1FF2700F0FF2F006201370001F827009D
:1024500000002000F7FF37006000B800F5FF3700EC
:102460001EFE07000509780000000600809FEB00B3
:10247000890107008F87E9000000E00000000600E6
:102480002800FA00889FBE008A9FBE008C9FBE0075
:1024900007067800878669000C003B00030478007B
:1024A0008704780008F0A10009F0A100840F500013
:1024B000858F5800860F5900890F5C000300330098
:1024C0000CF0A20001003A000CF0A1002D01070061
:1024D0006400E1005F003200780147006408E10019
:1024E000610032006C014700748557003200BE0065
:1024F0001201BE003A04BE001A05BE001E03900081
:10250000BE0A90008503530006003D000004FD0054
:102510008104FD000205FD008305FD008703EA003C
:10252000050378000DF8A3000400320060041400D5
:10253000E0841C0060051D00E0851D006022B800DD
:102540007D0320000D38E1008006EB000B00390010
:102550004433DD00F300B20083017300390037001B
:10256000848272000D027800E10664008B85D10040
:102570000A85D3008984D3000884D3008703E90047
:10258000F7FF3B0008004000898048000A0149002D
:102590008B81490004003B0060001000E0801800BF
:1025A00060011900E08119000358A30009003200FE
:1025B0008D82720084827200610260008301D1000A
:1025C0000281D3008180D3000080D3000603E8009D
:1025D0001B0037000348A30017003A000600E00084
:1025E000170034000603E9000D00A30000004800B6
:1025F0008180480002014900838149000348A3000B
:102600000F003A000600E000090034000603E9006C
:102610000000400081804800020149008381490098
:1026200001003A000003EB000348A300F5FF32006D
:102630006022B80002003700848272006182660066
:10264000E900070003F0A1000CF0A70003F0A000D0
:10265000E0003700640147006408E10002003A002E
:102660000DF8A300D8003A003200BE001201BE00EF
:10267000D80037001400FA00889FBE008A9FBE0071
:102680008C9FBE000004BE000205BE00680047002B
:102690000A90BE000890BE00280107000070A70045
:1026A0000BF0A1000BF8A30020003A009E09900057
:1026B0000E099000FE0090006E0090009E029000B7
:1026C0003443200084825200C20032000A003C00E1
:1026D000B4FC2F000428E100140034008301D10071
:1026E0000281D3008180D3000080D3008502E800FE
:1026F000FAFF3A00B7003700B40020000428E100D8
:1027000007003C00000040008180480002014900B1
:10271000838149008502E900FAFF3A00AD003700E5
:102720000300280002002000010037006011B800FB
:102730006000B800A70037002800FA00889FBE009C
:102740008A9FBE008C9FBE0003866B008D00070031
:102750006400E100440032006408E1004A003200F5
:102760006100E100460032006108E10049003200EA
:10277000EC0647006000B8003D02BE003D03BE000D
:10278000F48657006011B8003D04BE003D05BE0050
:102790007D0320000B0037000000A0008D06E9003B
:1027A000130032000402420085824A0006034B00F7
:1027B00087834B00000040008180480002014900EF
:1027C000838149000802520089825A000A035B0093
:1027D0008B835B00F0FF3B000802420089824A00C5
:1027E0000A034B008B834B008D06E900EDFF3A0096
:1027F0008482720086827200F707B20087827200BC
:1028000001003200150020001E0490003E0B9000D5
:1028100006035400E63FB0000368A300070032003F
:102820000000A7000500A0008301D1000281D300B1
:102830008180D3000080D3000603E8008301D1002B
:102840000281D3008180D3000080D3000002EB001E
:102850000482D2006400070003F0A1000CF0A7007E
:1028600003F0A0005B003700640247006408E10049
:10287000550032003400BE003401BE00F6FF3700C0
:102880006108E100500032006011B8006000B8003B
:10289000F1FF370003FF270002002000FBFF370095
:1028A000889FBE00830478000300E0002C00350000
:1028B00003003C0000827000040271002600320018
:1028C00036432000C50020008383CF000A00390072
:1028D0000541B1008283CF00070039000541B100F6
:1028E0008183CF00040039000541B1008083CF000F
:1028F000010039000541B10085C353006022B800D2
:10290000120032000A003B00848272006102600003
:102910008301D1000281D3008180D3000080D300E5
:102920000603E8008743E800F7FF3A000700370096
:102930000000400081804800020149008381490075
:102940000603E9008743E900F9FF3A002600070083
:1029500009F0A70003F0A0004F04BE00000006002D
:1029600060001000E080180060011900E08119008B
:10297000D3FF3B00033E2C00F7FF370007F0A20017
:10298000BFFE3700680447000294BE000094BE00FA
:10299000FC0447008694BE008494BE0009007800C1
:1029A00066000700080078006400070099007800BE
:1029B000814F70000B003B000800BE00860007003E
:1029C0004F00B10003003700F3FF2700F2FF2F0094
:1029D0006110B9004F06BE004F05BE004F04BE0097
:1029E0000080FA00000006001800200057002000B8
:1029F000080453000D003D000600200097FC2F0046
:102A00000740E1001E003400848272006102600011
:102A10008301D1000281D3008180D3000080D300E4
:102A20000804E800F8FF3A00470020006104600055
:102A300005047400040464000D00320061004000CD
:102A4000E080480060014900E081490003B8A5002A
:102A5000070032000603E8006538E10004003A0090
:102A60008301D1000281D3008180D3000080D30094
:102A7000F87F20000830E1000300350008037800EB
:102A80006000B8006011B8004433DD00F300B2000C
:102A90008301730000000600889FBE008A9FBE006D
:102AA0008C9FBE000404BE000605BE00809FBE00D1
:102AB000829FBE0056000700040678000800BE0092
:102AC0000A01BE0052000700840678004F03BE00D2
:102AD0004F02BE008D4F76007FB097001300330089
:102AE000F0FF2F008B8F6B0006003B000D06660089
:102AF0000C00A7000A00370007F0A6001000200015
:102B00000A003700880F5200898F5A008A0F5B0035
:102B10008B8F5B00030039001000200001003E0095
:102B20000000200007F0A7000000EA004F06BE00EA
:102B30004F05BE004F04BE00000006008000780074
:102B40005002BE005003BE004439DE00F700B20060
:102B5000F37F200003016100090032000218E10048
:102B600016003A00850172008301730083817300AF
:102B70000008200015003A00400020001300370034
:102B800085017200830173008381730005003A00A0
:102B900004A8BE0006A8BE00100020000B003700ED
:102BA0000201E9000402420085824A0006034B004C
:102BB00087834B000748A300F9FF32000740A000BD
:102BC00004A8BE0006A8BE002000200080009800D7
:102BD0009200980000000600E48240001078A300F4
:102BE00007003200640240001178A3003400BE00E8
:102BF0001401BE00040032000330A70000000600EC
:102C00003500BE001501BE000330A0000000060024
:102C100005FF270005826100070032000428E1005B
:102C200001003200240005000600070001003A0000
:102C3000440005000408050002000700F9FF3A00FF
:102C4000140005006F82610081027000850271002E
:102C500085027200000006008102D0008502E900B2
:102C60000118780002187800051841000318780050
:102C700004187800051842000408780000000600D7
:102C8000889FBE008A9FBE008C1F78004400F80019
:102C9000070F2000270288003400F8003305900059
:102CA00008F02F000A40E1000400320028028000F2
:102CB0004800B30028028800AA018800811F78001C
:102CC0000403780013029000C30290008301900077
:102CD0008605D000068651000000E9008381E900E6
:102CE0008604E9000C06E900008008000C000000E2
:102CF000050478000B8542000C8009003A1C78001E
:102D000009800900321C7800040478000A85E90073
:102D10005E2CC300038009005E2CC6001201C600B1
:102D20003100CD004F0078003400F9004400F90074
:102D30004F0678004F05BE004F04BE00000006009D
:102D4000881F78008A1F78004400F800080F2000D0
:102D5000280288003400F8003305900008F02F00A6
:102D60000A40E10004003200280280004800B3005D
:102D700028028800AA0188004600F8004800F800F0
:102D80004A00F8004C00F8004E00F8008A0A2C00B7
:102D90003A0288002304900058028800130490002F
:102DA00048028800530590007A028800430590008D
:102DB0006A028800811F780063059000030290007A
:102DC000630252000000E9000080080007000000D4
:102DD000320D7800000000004618C300048009008E
:102DE0004618C4004218C4001201C4003100CD00CE
:102DF000EA0198004F0078004E00F9004C00F900FD
:102E00004A00F9004800F9004600F9003400F900D2
:102E10004400F9004F0578004F04780000000600D8
:102E2000889FBE008A9FBE008C9FBE004400F800B1
:102E3000070F2000270288003400F80007F02F0059
:102E40000338E10004003200270280004700B3008D
:102E500027028800A3018800811F78001900200044
:102E6000804CDD001300200002047800800678000A
:102E70008904D100424EDD00010578000302E9001B
:102E800004800800170000008A0546004218DD0093
:102E90000902E900048008001000000000000000A2
:102EA0004620C3003B025200DF35C1000804400049
:102EB0001381C200AB825200264DC5003E85C4007E
:102EC000BB00CD00BB80CD003A00CA002A80CA00FA
:102ED0000700C9000580C900BA00CD00BA80CD0046
:102EE0000A054600020478008301D0008D06E9003F
:102EF000DFFF3C004F0078003400F9004400F90087
:102F00004F06BE004F05BE004F04BE000000060085
:102F10004600F8005000F80002202000320288002D
:102F200002002800130020008019DD0002817100DA
:102F3000820288000100780001017800260020004C
:102F4000470020008301E90003800800070000001B
:102F50000110E100040034001102BE009208780064
:102F6000E2307B000489BE0087804000121978009F
:102F70005000F9004600F90000000600821F7800AA
:102F8000849FBE008A1F78004400F800040F2000D0
:102F900024028800010578000601C3000080E900D2
:102FA0000080080003000000000000000505F0009C
:102FB0000401F1003200CD000505F0001001F10020
:102FC0003200CD004400F9004F0578004F02BE00EA
:102FD0004F0078000000060001002000F0A08900EA
:102FE00001A1890011C0B300C0412300014878004D
:102FF00000000600C24123001204E00006003A006F
:103000001000200001002000F0A0890001A189002B
:1030100010C0B30000497800D2E62400631C2400ED
:10302000F0A0810001A1810078F707000001BE0037
:10303000900323000100200002004000838048002C
:10304000F0A0890001A189004088DE00CF80DE0069
:1030500000F0A10000000600800078003004E000CD
:10306000FEFF3A00010050000000E90000000600E9
:103070000C00FA00889FBE0000047800CFB09700D3
:10308000F0FF2700D0BF9F008004EB0099BF9F0096
:1030900088BF9F00A8BF9F00200C2000B0BF9F00EA
:1030A00078815700708057005F0007000FB89700C5
:1030B000094878000FB8970008045000080078000D
:1030C0004F04BE000080FA0000000600889FBE008A
:1030D0008A1F7800804078000004E00021003D0055
:1030E0008040EA00D0C6B30080CF50000900340011
:1030F0008104FB0042062000110009008204D80070
:1031000000017800010078004311DD004A502400DE
:103110001F0037000100FB00435024003900370036
:10312000A2002000110009000200D8000001780070
:10313000010078004311DD00030141004300DD0080
:10314000030040003002BE002003BE004220900079
:10315000D2209000F221900062219000F7FB07003E
:103160002E003700D0C6B30080CF500023003400BB
:103170008104FB0042062000110009008204D800EF
:1031800000017800010078004311DD004A5B240053
:103190000A014100A8002000110009000800D80021
:1031A0004300DD000A00400040229000D022900041
:1031B00060239000F0239000028890009288900095
:1031C000B289900022899000DCFB0700801F780004
:1031D00001027800110009008804D8000102FD00F6
:1031E0004F0078000402FB004322DD000A02420087
:1031F0005403BE004402BE00D8FF37000100FB00AC
:10320000435B2400EACF5000C5FF3C004300DD00D3
:10321000030040005001BE004000BE004F05780092
:103220004F04BE00000006008F03B000889FBE0060
:103230008A9FBE008C9FBE008E1F7800E0B79F0063
:10324000F1B79F0082BF9F000000EB00A0B79F0076
:10325000E60437008001EB0050C2B30080CF50007D
:10326000090032000100FB00EFB09700EC040700FA
:10327000E10F4000DD043200AFB097008100E800AC
:10328000A1B79F00D90437007FB197009240780022
:10329000D0C2B30080CF50000C00320007003C00C9
:1032A0006D40500080CF50000D0032006B40400058
:1032B00080CF500019003A000E00370000C3B30061
:1032C00080CF500015003A000F0037000330A000F7
:1032D0007FB297000402E800F4B79F00EAFF3700CE
:1032E0000300A000FFB297008502E800F5B79F0039
:1032F000E5FF37000310A0007FB697000C06E8003A
:10330000FCB79F00E0FF37000320A0007FB09700CC
:103310000000E800F0B79F00DBFF37000318A300B0
:10332000010032000300A1000338A30001003200B5
:103330000320A1000100FB0002FD2F00020040005D
:10334000E90F500010003E008000EB00C1B79F0065
:10335000020278004FB197006A10B900FFB29700DF
:103360001501FB000001410004014100C2B79F00AC
:103370005500FB00F5B79F0004004000E90F500026
:103380000D003E00F3FF37000006EB00CCB79F00B6
:10339000A0C2B30080CF500007003A000FB89700DA
:1033A000C000780080BF9F00C1B79F007FB1970029
:1033B0000201E800F2B79F00E0C2B3007FB29700BD
:1033C000944F100021003A00830678000DE0A00021
:1033D0008400E80064405000914F10000400320067
:1033E000F1B79F008002EB00B5B79F0010003700D7
:1033F0000FBE97004C0078008CBF9F00B0B79F00B5
:10340000FFB097008180E800F1B79F0013003700FC
:103410003FB297006A20B90000004100030040005D
:10342000B0B79F00FFB297008502E800F5B79F0094
:103430007FB697001C01FB0003FD2F000300410035
:10344000E90F5000F2FF36000400370083067800D1
:103450000DC0A0000000EB00B0B79F007FB1970047
:10346000B2407800F2B79F00C17F9F00C0C6B30092
:1034700080CF50002700320014003C00684050000C
:1034800080CF50009D00320009003C006C4050008D
:1034900080CF5000290032006B40400080CF5000A8
:1034A000720032000104E000560432008E00370042
:1034B00060C6B30080CF50001C0032006340400063
:1034C00080CF500088003A008C00370030C7B3002E
:1034D00080CF50001C00320007003C0064405000C8
:1034E00080CF5000130032000040E80080CF500031
:1034F0007D003A001100370050C7B30080CF500064
:103500007D0032006340400080CF500076003A00DA
:103510000B003700000028000D48A30001003A000E
:103520000001200080867600CCFF37000DA0A000AF
:10353000720037000D60A000700037000D50A00031
:103540000D70A0006D0037008FB997004300780020
:1035500083BF9F00000478000000E00001003A00F3
:10356000083223008004EB00010037008104E800EA
:1035700089007800088044001004E000FBFF3A0056
:103580003FB297000400E00003003200890F5200B0
:1035900001003100840478000007EB00CFB29700EF
:1035A000898F520001003600098752004368DE000F
:1035B000E106600019003A000D06780009003700A6
:1035C000EFB097000002200015040700E10F400053
:1035D000030032002FB097000000E800A0B79F0062
:1035E0000C06E8008E0F5600F5FF3A000087EB004E
:1035F0000A003700880078003100FB0001047800E1
:10360000EFB0970006040700E10F4000030032000E
:10361000AFB097008100E800A1B79F000900E90062
:1036200080047800E10F4000F2FF3A000006EB0052
:103630000D00E0000A003A00EC033700EFB09700FD
:1036400000022000F6030700E10F400003003200F3
:103650002FB197000201E800A2B79F000C06E80016
:103660008E0F5600F5FF3A00E00337008FB9970040
:103670004300780083BF9F00CF80DE000101780007
:10368000820178000205BE000004BE000203BE00F5
:103690000002BE004822DE00482EDD000402760053
:1036A000C47F9F000D48A3000A0032000404E0001C
:1036B00008003200E14F420006003200D1FB2F002B
:1036C0000180470004487800184098002900200035
:1036D00002003700D07F9F0019002000D2FB2F008E
:1036E00002844700A6FF3700C3FB2F000384470076
:1036F00019002000A2FF37000D0CB300007020005D
:1037000000826600270232000DC8A30002003200CA
:1037100064002000B4B79F000D48A30005003200EC
:103720000FBA97004401BE004400BE0084BF9F0052
:10373000040037008FBA97004500BE0085BF9F0088
:10374000F3FA0700E0AF9F00F1AF9F0082B79F0040
:1037500093B79F006022B8006033B8006FA897004D
:10376000FFA897000FB197009FB1970007FB0700D4
:103770000000E0000A003D006FA89700FFA8970036
:103780000FB197009FB1970003F0A200E0AF9F0038
:10379000F1AF9F0082B79F0093B79F003D00B30039
:1037A0000000EB0080A79F006022B8006033B800E3
:1037B0006FA89700FFA897000FB197009FB19700DF
:1037C000F7FA07000000E000340032006FA897000D
:1037D000FFA897000FB197009FB19700F5FA070077
:1037E00003FC2F00038147001DFB07000FA097007B
:1037F0000000E9006300B900A200200011000900E8
:103800000200D8008000FD0081A79F000100E000B9
:1038100002003D000100E90080A79F000FA497006F
:103820000840EA0029FE07006FAA9700FFAA970048
:103830000FB397009FB3970040FA0700A0AF9F0017
:10384000B1AF9F00C2AF9F00D3AF9F006022B8000E
:103850000600200007FF2300CCFA07000000E0006C
:1038600002003D000800E9000B0037006022B800AC
:1038700006002000470224002FA89700BFA8970049
:103880004FA99700DFA99700F8FA07000000E000B1
:10389000020035000800E80080A79F003FB29700B3
:1038A000F80F520057003C00D0C6B300804F5200C2
:1038B000290036000485FB004206200011000900A3
:1038C0000285D80000017800010478004311DD0072
:1038D0004B5024000B0141006022B800060020007C
:1038E00007FE23000288900092889000B289900021
:1038F0002289900011FA0700A9002000809FBE00D5
:10390000110009000984D800000478004F00BE00AF
:103910004344DD000B04440048229000D82290006C
:1039200068239000F823900004FA0700801F7800B5
:1039300001027800110009000985D8000102FD008C
:103940004F0078004322DD000B0242005403BE000A
:103950004402BE001F0037000480FB0049502400D1
:10396000EA4F520014003600A200200011000900A6
:103970000280D80000017800010478004311DD00C6
:10398000090141006022B8000600200007FE230064
:1039900042209000D2209000F221900062219000FD
:1039A000E6F907004344DD00090444003802BE0084
:1039B0002803BE00070037004300DD000900400077
:1039C0006022B8000600200007FE23005001BE0060
:1039D0004000BE00D9F907000002BE000203BE008D
:1039E0006FA89700FFA897000FB197009FB19700AD
:1039F000A3FA0700E0AF9F00F1AF9F0082B79F00DE
:103A000093B79F000FA49700E90F540015003C00E6
:103A10006022B8006033B8006FA89700FFA8970035
:103A20000FB197009FB197005DFA07000000E0001A
:103A3000320032006FA89700FFA897000FB19700DF
:103A40009FB197000BFB0700E00F5000E08F58007C
:103A5000E00F5900E08F590028003A00E10F5400B0
:103A6000260034000400200005002E00B6E02200ED
:103A7000170124002FA89700BFA897004FA997000F
:103A8000DFA9970041FA07000000E00002003D00B6
:103A900073005400010037007200540080A79F009B
:103AA0000FC0970089FD0700A0AF9F00B1AF9F0036
:103AB000C2AF9F00D3AF9F000002BE000203BE0052
:103AC0006FA89700FFA897000FB197009FB19700CC
:103AD00019FB0700E7FA07000205BE000004BE005C
:103AE0006000B8006011B800A0A79F00B1A79F00B8
:103AF000C2A79F00D3A79F002E0037006FA8970092
:103B0000FFA897000FB197009FB19700D9FA07005F
:103B10000205BE000004BE00E00F5000E08F580018
:103B2000E00F5900E08F5900020035005CFB0700F0
:103B30001300370010002000010020006011B800C1
:103B400008006000898060000A0161008B816100CB
:103B50008B03D1000A83D3008982D3000882D3006B
:103B60000000720081807200020173008381730083
:103B70004BFB07000002BE000203BE0040FA070034
:103B80000002BE000203BE006FA89700FFA89700C6
:103B90000FB197009FB1970078FB0700A0A79F0087
:103BA000B1A79F00C2A79F00D3A79F000000EB0012
:103BB00080A79F0014C0B300051923000B00370035
:103BC0000400FB004300DD00050040005001BE0082
:103BD0004000BE000040E10001C8E10002D0E10069
:103BE00003D8E100030039000442E800F44F52001A
:103BF000F3FF3A00C47F9F000400FB00BFB09700B2
:103C0000008040008FA09700010040004FB1970056
:103C100000075100BFB197000300E000010032002F
:103C20000E07E90063806600010032000E07E9001C
:103C30000D28A30026003200E18066000D18A300C5
:103C40000C003200D00220000100E00001003A0028
:103C50000080E900EFB0970071020700E10F40001B
:103C6000180032002FB297000402E800A4B79F00AA
:103C7000140037000100E00012003200EFB097009E
:103C80000002200066020700E10F40000D00320034
:103C9000AFB297008502E800A5B79F000900370082
:103CA000EFB09700000320005D020700E10F400025
:103CB000030032002FB697000C06E800ACB79F0057
:103CC0000E07E9000E00E000F5FF3C003D00370064
:103CD0000D38A3000A0032000B003700EFB0970048
:103CE000000220004E020700E10F400003003200F6
:103CF0002FB097000000E800A0B79F000E07E90072
:103D00000E00E000F5FF3C00E18066000D18A30006
:103D10000C003200D00220000100E00001003A0057
:103D20000080E900EFB097003D020700E10F40007E
:103D300024003200AFB097008100E800A1B79F00D7
:103D4000200037000100E0001E003200EFB09700B5
:103D50000002200032020700E10F4000190032008B
:103D60002FB197000201E800A2B79F0015003700AD
:103D70000000FB004300DD000119230001004000AA
:103D80003002BE002003BE000800BE000A01BE00D3
:103D900059F80700A4002000050020006033B80097
:103DA0005CF807000003B000EFB097001C020700AA
:103DB000E10F400003003200AFB197008301E8003B
:103DC000A3B79F004F7A97000440E900C07F9F008F
:103DD000E14F4000E6FF3A000B003700EFB09700DC
:103DE000000320000E020700E10F40000300320034
:103DF000AFB297008502E800A5B79F000FA097001B
:103E00000000E90080A79F000FA097000000E000DD
:103E1000F2FF3C003FB6970020C1B300F20F5600FE
:103E200001003C006FE09700C07F9F00CF789700B3
:103E30000100FB003FB1970000005100E0A79F0088
:103E40000104E00008003200EFB09700E00220001B
:103E5000F3010700E10F400003003200AFB197000B
:103E60008301E800A3B79F004F78970097FC0700F5
:103E70000002BE000203BE002FA09700BFA0970063
:103E80004FA19700DFA19700ACF80700F9F90700F0
:103E90001E0037000000FB004300DD000C1923006A
:103EA0000C0040003002BE002003BE000800BE002F
:103EB0000A01BE0010F80700A40020000500200041
:103EC0006033B80013F807000003B000EFB09700AC
:103ED000D3010700E10F4000030032002FB297002A
:103EE0000402E800A4B79F00CF7A97000500FB000A
:103EF0004300DD000C0040003002BE002003BE0085
:103F00000800BE000A01BE0002F807000205BE005C
:103F10000004BE004F7E97000C40E900C07F9F0068
:103F2000E14F4000DBFF3A000006EB0009003700DC
:103F3000EFB0970000032000B9010700E10F400037
:103F4000030032002FB097000000E800A0B79F00E8
:103F50000C06E800EFA09700810F5600F4FF3A002E
:103F60000D38A300A10132000E00E0009F013400D3
:103F70000006EB00EFB0970000022000A801070048
:103F8000E10F4000030032002FB197000201E8006A
:103F9000A2B79F000C06E8008E0F56009301320076
:103FA000F4FF37000D007800000CB20028003A0042
:103FB0000D00E00005003D008FB997004305BE00ED
:103FC0004304BE0083BF9F00140037000D48A300C8
:103FD0000B0032000FBA97004400BE0084BF9F0060
:103FE0004F89DE00CF91DE000002BE0002037800A0
:103FF000820378000605BE000404BE0007003700F7
:104000008FBA97004500780085BF9F0000047800B4
:10401000CFC4DE00090578008A057800E00F54005F
:10402000E08F5C00E00F5D00E08F5D0020003D0050
:104030003D00B3006000B8006011B80008045000F3
:10404000898458000A0559008B85590018003700EB
:104050000D00E00005003D000FBE97004C05BE00BE
:104060004C04BE008CBF9F00110037000D48A30018
:10407000080032008FBA97004500BE0085BF9F0040
:1040800004017800840178000205BE000004BE002F
:10409000070037000FBE97004C0078008CBF9F00D0
:1040A00000047800090020000A0020000B00200016
:1040B0003FB097000000E00007003A00E00F540016
:1040C000E08F5C00E00F5D00E08F5D0002003A00D1
:1040D00011002000B1B79F000D0778000E0CB20050
:1040E00000042000800F57002F00320003003C0026
:1040F0000E00E000070032003F00370000082000FB
:10410000800F570014003200000C2000800F570071
:1041100039003A0014C0B300051923000B00370022
:104120000400FB004300DD00050040005001BE001C
:104130004000BE000040E10001C8E10002D0E10003
:1041400003D8E1002B0039000442E800F44F52008C
:10415000F3FF3A0027003700000120000100200093
:104160006011B80014C0B3000040E10001C8E100D4
:1041700002D0E10003D8E1001E0039004500200014
:104180000000D0008180D2000281D2008381D20061
:104190008502E900FAFF3A000442E800F04F5200BD
:1041A000F1FF3A00130037008000200001002000DA
:1041B0006011B80014C0B3000040E10001C8E10084
:1041C00002D0E10003D8E1000A0039003C002000E1
:1041D0000000D0008180D2000281D2008381D20011
:1041E0000C06E900FAFF3A000442E800F54F5200DD
:1041F000F1FF3A00C47F9F00CF7897000100FB00D9
:104200003FB19700820F500002003D00C27F9F0027
:1042100004003700BFB19700808F510001003D00BE
:10422000B0B79F004FB297000400E00004003200D6
:1042300063806600020032000402E900C4B79F00F8
:104240000DE8A3000B003200CFB297003FB69700F5
:104250008C8F520003003C000000EB00C0B79F00B1
:1042600004003700CFB097003FB197008280500024
:10427000C1B79F00CF7997000300FB000002EB005D
:1042800094A79F00CFB29700808F520002003400A5
:104290000080520090A79F000D28A3003700320035
:1042A000E18066000D18A3000C003200D00220004F
:1042B0000100E00001003A000080E900EFB0970043
:1042C000D7000700E10F40000E0032002FB6970024
:1042D0000C06E800ACB79F000A0037000100E000C0
:1042E00008003200EFB0970000022000CC00070069
:1042F000E10F4000030032002FB097000000E800FB
:10430000A0B79F009FA097000100E0000F003200BF
:104310000006EB00EFB0970000032000C00007008C
:10432000E10F4000030032002FB197000201E800C6
:10433000A2B79F000C06E8009FA19700830F5600CC
:10434000F4FF3A000002EB0094A79F00BFB2970071
:10435000C328DD00801823008080400091AF9F00BB
:104360004228DD006400500080AF9F006328B90040
:10437000F0A79F0063065000820037001FA6970039
:104380000C00E00011003200688066000F003A0067
:1043900000067800EFB0970000022000A0000700A0
:1043A000E10F4000030032002FB097000000E8004A
:1043B000A0B79F000C06E8009FA09700810F560051
:1043C000F4FF3A000001EB0092A79F00E180660035
:1043D0000D18A3000C003200D00220000100E00004
:1043E00001003A000080E900EFB097008C00070060
:1043F000E10F4000D5FF3200AFB197008301E80024
:10440000A3B79F00D1FF37000100E000CFFF3200CB
:10441000EFB097000002200081000700E10F40008C
:10442000CAFF32002FB297000402E800A4B79F0031
:10443000C6FF370000042000800F57003000320014
:1044400003003C000E00E000070032003D00370092
:1044500000082000800F570011003200000C2000DF
:10446000800F570037003A001FA897003002BE00A7
:104470002003BE000800BE000A01BE009EF6070031
:10448000A4002000050020006033B800A1F607005A
:1044900004C3B30004424000C47F9F0029003700DA
:1044A00075322300D5B79F000D58A30002003A00D3
:1044B00080332300D0B79F001400200005002000A7
:1044C0006033B8008FA897008100E9000500330031
:1044D0000402D0008582D2000683D2008783D200F6
:1044E000F9FF37000800BE000A01BE0082F607008F
:1044F0006F0060005FB197006240780010003700E5
:1045000014002000050020006033B8008C01780002
:104510008301E900050033000402D0008582D20047
:104520000683D2008783D200F9FF37000800BE005F
:104530000A01BE0070F60700674060000043B0004B
:10454000C07F9F004F7A97000400FB00EFB09700F8
:1045500033000700E10F400003003200AFB29700C4
:104560008502E800A5B79F001FA8970068005000CB
:1045700090AF9F008FA89700E480500081AF9F000C
:1045800063065600D0FF2F003FB197000090B9009E
:10459000FFA197000080410063005000800F56008B
:1045A000A4FF3A000D38A300100032001FA29700AC
:1045B0000400E0000D0034000006EB00EFB09700AF
:1045C0000002200016000700E10F40000300320047
:1045D000AFB297008502E800A5B79F000C06E8007F
:1045E0001FA09700800F5600F4FF3A007FB197009C
:1045F000B2407800F2B79F00C17F9F000104E00045
:1046000014FB3A002FB097004F0778004F06BE000A
:104610004F05BE004F04BE008F03B100000006002E
:10462000889FBE000001780001047800B10090006E
:104630000118A3003D0032000198A30003003A00D6
:10464000180090000000E00038003A000190A0003F
:104650003104980082047800F90FB200180090002D
:104660000000E00002003A0028009000000C7800F2
:10467000EA8F540006003A00380090000078A3004A
:1046800003003A0088007800D0002000E4FF070013
:104690009800900058009000808F50000B0032006E
:1046A0000100E8001004980018007800095878000C
:1046B000000C780011C0B30060422300014878006C
:1046C000EA8F540006003200190037008800780095
:1046D00009407800190007008004780014003700B2
:1046E000380090000088A3001100320018019000EB
:1046F000A8009000480090008DF1070098009000FD
:10470000810F500004003200380090000003B30015
:10471000300498008084EB000000EB001004980047
:1047200028009000000C7800010037008084EB0026
:10473000090078004F04BE00000006000200FA00E5
:10474000889FBE00A0FF9F0001047800B100900088
:10475000810478000904B200020032000000FB006E
:10476000360037000118A30005003A000103B3002A
:1047700031049800190498000080EB002F003700E6
:10478000580090000000E00006003A004800900049
:1047900012002000E680570065F107001904980018
:1047A00024003700280090000000E00008003A00D4
:1047B0002042230020049800000C780020002000F4
:1047C00050049800100498000130A00031049800B3
:1047D00018019000A80090004800900054F10700D4
:1047E00028009000000C78000080EB001004980076
:1047F00018007800AFF8970001587800000C780096
:104800002FF89700EA4F50000A003A003800900055
:104810000088A3000700320018019000A800900053
:104820004800900042F1070019049800A800900089
:10483000010C7800AFF897000100FB004F04BE00A8
:104840000080FA00000006000000FA0010002000BE
:10485000842024008001780042A62E00310220002E
:10486000609120002C1602000000000010002000C3
:10487000E42424008001780042A62E0031022000AA
:10488000409220002C1602000000000010002000C2
:10489000442924008001780042A62E003102200025
:1048A000209320002C1602000000000010002000C1
:1048B000A42D24008001780042A62E0031022000A1
:1048C000009420002C1602000000000010002000C0
:1048D0000400240080017800C2852E00110420000D
:1048E000E09420002C1602000000000010002000C0
:1048F0002408240080017800C2852E0011042000C5
:10490000C09520002C1602000000000010002000BE
:104910004410240080017800E28D2E001104200054
:10492000A09620002C1602000000000010002000BD
:104930006418240080017800E28D2E00110420000C
:10494000809720002C160200000000000080FA0072
:10495000000006000000FA001000200004002400FF
:104960008001780002962E0011042000E0942000BF
:104970002C16020000000000100020002408240073
:104980008001780002962E0011042000C0952000BE
:104990002C1602000000000010002000441024002B
:1049A00080017800229E2E0011042000A096200095
:1049B0002C160200000000001000200064182400E3
:1049C00080017800229E2E00110420008097200094
:1049D0002C160200000000000080FA000000060013
:1049E0000000FA000000EB00001088000000EB005F
:1049F000101088000000EB00501088000000EB0051
:104A000060108800B0162000201088000602A9005F
:104A1000000000000622A900000000000642A900D4
:104A2000000000000662A900000000000682A90044
:104A30000000000006A2A9000000000006C2A900B4
:104A40000000000006E2A900000000000702A90023
:104A5000000000000722A900000000000742A90092
:104A6000000000000762A900000000000782A90002
:104A70000000000007A2A9000000000007E2A80053
:104A80000802A900000000000822A90000000000A0
:104A90000842A900000000000862A9000000000010
:104AA0000882A9000000000008A2A9000000000080
:104AB00008C2A9000000000008E2A90000000000F0
:104AC0000902A900000000000922A900000000005E
:104AD0000942A9000000000009C2A900000000006E
:104AE00009E2A9000080FA00000006000600FA00B2
:104AF000000F780021479800220798000602A800BE
:104B0000301080007F0060000000E000FCFF3A00F1
:104B1000000A20001010880009C2BF000044B20043
:104B20000004E000FCFF3A0009C2BF0001C8B30066
:104B3000014060000004E000060032000642A800C8
:104B400006C2BF00644060000004E000FCFF3A00C1
:104B5000EAFF37001E007800C880DE002E009000BB
:104B6000008070001010880009C2BF000044B2002D
:104B70000004E000FCFF3A001E00780010108800DE
:104B800009C2BF000044B2000004E000FCFF3A008C
:104B90002E4090000000FB001010880009C2BF00EA
:104BA0000044B2000004E000FCFF3A000642A80006
:104BB00006C2BF00644060000004E000FCFF3A0051
:104BC0000080FA00000006000600FA0010079800B6
:104BD000210798000602A800301080007F006000C6
:104BE0000000E000FCFF3A00000A200010108800DE
:104BF00009C2BF000044B2000004E000FCFF3A001C
:104C000009C2BF0001C8B300014060000004E00019
:104C1000060032000642A80006C2BF0064406000E1
:104C20000004E000FCFF3A00EAFF37001E0090009D
:104C3000C880DE002E0090000080700010108800F8
:104C400009C2BF000044B2000004E000FCFF3A00CB
:104C50001E0090001010880009C2BF000044B2007E
:104C60000004E000FCFF3A000622A80006C2BF00D4
:104C7000624060000004E000FCFF3A00100A2000DF
:104C80001010880009C2BF000044B2000004E00018
:104C9000FCFF3A0009C2BF0001C8B3000140600038
:104CA0000004E000FBFF3A000662A80006C2BF0055
:104CB000684060000004E000FCFF3A000010800043
:104CC000004F780006A2A8000682A80006C2BF0016
:104CD000704060000004E000FCFF3A000642A800BB
:104CE00006C2BF00644060000004E000FCFF3A0020
:104CF0001E00FB000080FA00000006000000FA0021
:104D00002003A900000000002023A90000000000EB
:104D10002043A800000000002063A900000000005C
:104D2000013220009140780000CEB30000C0700036
:104D300020E3B7000000000021C3BF003040B300F3
:104D400021E3B700000000002143A800000000009C
:104D50002183A8000000000021A3A900000000009A
:104D600021E3A8002203A900000000002223A900DB
:104D700000000000213220009140780030CCB300C8
:104D800000C0600022E3B7000000000022E3A90099
:104D9000000000003132200091407800C0CFB30005
:104DA00000C0600023E3B700000000002343A90017
:104DB0000000000023C3BF007F40600023E3B70072
:104DC00050C0B30024E3B7000000000051322000BF
:104DD0009140780000CEB30000C060000004A00045
:104DE00025E3B7000000000025E3A9002603A90081
:104DF00000000000613220009140780090CFB300A5
:104E000000C0600026E3B700000000002703A900EF
:104E100000000000713220009140780090CFB30074
:104E200000C0600027E3B700813220009140780085
:104E300000CEB30000C0600028E3B700000000000F
:104E400028E3A90000000000913220009140780082
:104E500000CEB30000C0600029E3B70000000000EE
:104E600029E3A9002C03A900000000002C23A800BE
:104E7000000000002C43A800000000002C63A800E4
:104E8000000000002C83A800000000002CA3A80054
:104E9000000000002CC3A800000000002CE3A800C4
:104EA000000000002D03A800000000002D23A80032
:104EB000000000002D43A800000000002D63A800A2
:104EC000000000002D83A800000000002DA3A80012
:104ED000000000002DC3A800000000002DE3A80082
:104EE0003003A800000000003023A90000000000EB
:104EF0003043A900000000003063A900000000005A
:104F00003083A9000000000030A3A90000000000C9
:104F100030C3A9000000000030E3A9000000000039
:104F20003103A900000000003123A90000000000A7
:104F30003143A900000000003163A9000000000017
:104F40003183A9000000000031C3A9000000000067
:104F500031E3A900213320009140780080CFB300D5
:104F600000C0600032E3B7006003A9000000000049
:104F70006023A900000000006043A80000000000BA
:104F80006063A90000000000013620009140780015
:104F900000CEB30000C0700060E3B7000000000066
:104FA0001136200091407800C0CFB30000C06000EF
:104FB00061E3B700000000006143A80000000000AA
:104FC0006183A8000000000061A3A90000000000A8
:104FD00061E3A8006203A900000000006223A900A9
:104FE00000000000213620009140780030CCB30052
:104FF00000C0600062E3B7000000000062E3A900A7
:10500000000000003136200091407800C0CFB3008E
:1050100000C0600063E3B700000000006343A90024
:105020000000000063C3BF007F40600063E3B7007F
:1050300050C0B30064E3B700000000005136200008
:105040009140780000CEB30000C060000004A000D2
:1050500065E3B7000000000065E3A9006603A9004E
:1050600000000000613620009140780090CFB3002E
:1050700000C0600066E3B700000000006703A900FD
:1050800000000000713620009140780090CFB300FE
:1050900000C0600067E3B7008136200091407800CF
:1050A00000CEB30000C060000004A00068E3B700B9
:1050B0000000000068E3A900000000009136200015
:1050C0009140780000CEB30000C0600069E3B700F3
:1050D0000000000069E3A9006C03A80000000000C4
:1050E0006C23A900000000006C43A9000000000030
:1050F0006C63A800000000006C83A80000000000A2
:105100006CA3A800000000006CC3A8000000000011
:105110006CE3A800000000006D03A8000000000080
:105120006D23A800000000006D43A80000000000EF
:105130006D63A800000000006D83A800000000005F
:105140006DA3A800000000006DC3A80000000000CF
:105150006DE3A8007003A900000000007023A900FF
:10516000000000007043A800000000007063A90068
:10517000000000007083A9000000000070A3A900D7
:105180000000000070C3A9000000000070E3A90047
:10519000000000007103A9000000000000000000F2
:1051A0007123A900000000007143A9000000000065
:1051B0007163A900000000007183A90000000000D5
:1051C00071C3A9000000000071E3A900213720008D
:1051D0009140780080CFB30000C0600072E3B70058
:1051E0000080FA00000006000000FA00DE02A900BC
:1051F00000000000D362A90000000000E202A80045
:1052000000000000D762A800000000002124200058
:1052100091407800C0CFB30000C060000014A0002F
:1052200042E2B7000000000042C2BF00C041B3002C
:1052300042E2B7000000000042A2A8000000000007
:1052400042C2A9000000000042E2A90000000000E4
:105250004302A800000000004322A9000000000053
:105260004342A800000000004362A90000000000C3
:105270004382A900000000004422A80000000000B2
:1052800045A2A8000000000045C2A90000000000DF
:1052900045E2A9000000000041A2A90000000000B2
:1052A00041E2A8000000000040C2A9000000000088
:1052B0002126200091407800C0CFB30000C06000DC
:1052C0000014A00062E2B7000000000062C2BF004C
:1052D000C041B30062E2B7000000000062A2A80073
:1052E0000000000062C2A9000000000062E2A90004
:1052F000000000006302A800000000006322A90073
:10530000000000006342A800000000006362A900E2
:10531000000000006382A900000000006422A800D1
:105320000000000065A2A8000000000065C2A900FE
:105330000000000065E2A9000000000061A2A900D1
:105340000000000061E2A8000000000060C2A900A7
:10535000000000000080FA00000006000000FA00D3
:105360000421A900000000000441A9000000000081
:105370004110200091407800F0CCB30000C06000E4
:1053800004E1B7000000000004C1A9000000000013
:1053900005A1A900A580A900A5A0A900A5C0A800F5
:1053A000703821001008880005E1A8008460A90079
:1053B0009460A8000080FA00000006000000FA00D7
:1053C000D302A8008220A900E10A200091407800C1
:1053D00080CFB30000C060000024A000AEE0B700A2
:1053E0008680A9009680A800C702A800C722A8004E
:1053F000C742A800C762A800C782A800C7A2A80029
:10540000C7C2A800C7E2A8000080FA00000006009A
:10541000809FBE00829FBE003400F8002000200064
:10542000A00188000000FA00F2D980004016800038
:105430004800DE0080007800F00F200080816000CE
:1054400082004100802C2300008040000308780087
:105450000200E800F0D98800F0D98000E70F500082
:10546000020034000000EB00F0D988008680A9001B
:105470000080FA003400F9004F01BE004F00BE006A
:10548000004006000600FA0050002000104088008E
:105490003F01370001DA800001814000802C2300A9
:1054A0000000410010017800120798000100E80098
:1054B00000DA880000DA8000E70F500002003400B4
:1054C0000000EB0000DA88001E0090002007980022
:1054D00060072000AE009000808F50008C003200EA
:1054E000600720002E019000800F510012003C0048
:1054F0002E009000F20F50003E003200AE009000EF
:10550000F28F500004003C002E019000F10F51007A
:105510006D003200960037002E009000F40F50000E
:105520005200320090052000AE009000808F5000A5
:105530003F0032008E003700000E20002E01900048
:10554000800F51001B003200000E2000AE009000C2
:10555000808F500005003C00A00A20002E01900022
:10556000800F51000A01320081003700100E200028
:10557000AE009000808F500012003200000F20001B
:105580002E019000800F510001003200780037009A
:10559000C04C800001102000010060000000E0000D
:1055A000FB003A00C04C80000000A000C04C880006
:1055B000F7003700C04C80000010A000C04C8800ED
:1055C000F3003700C04C8000011020000100600093
:1055D0000000E000EE003A00C04C80000080A00017
:1055E000C04C8800C142230020C0B300804878002E
:1055F000E7003700C04C8000610060000000E00060
:1056000004003200C04C80000020A100C04C880083
:1056100003003700C04C80000020A000C04C880070
:10562000C04C80000000A100C04C8800D8003700AA
:10563000C04C8000610060000000E0000400320007
:10564000C04C80000020A100C04C8800030037003F
:10565000C04C80000020A000C04C8800C04C8000DE
:105660000000A100C04C8800C9003700C04C800079
:1056700001102000010060000000E000C4003A00BA
:10568000C04C8000610060000000E00004003200B7
:10569000C04C80000040A100C04C880003003700CF
:1056A000C04C80000040A000C04C8800C04C80006E
:1056B0000000A100C04C8800C04C80000010A10078
:1056C000C04C8800B2003700C04C80006100600010
:1056D0000000E00004003200C04C80000030A10057
:1056E000C04C880003003700C04C80000030A00090
:1056F000C04C8800C04C80000000A100C04C880055
:10570000C04C80000010A100C04C8800A0003700F1
:105710000091200010407800E74F500014003A003C
:10572000C04C8000610060000000E0009800320082
:10573000D0198200E10F500006003A0060CD8000D1
:105740000000A20060CD88001A780200000000006E
:105750000300370070CD80000000A20070CD8800EB
:10576000C04C80000000A100C04C880088003700B9
:10577000C04C8000610060000000E00007003200C3
:10578000C04C80000000A100C04C8800C04C8000CC
:105790000010A100C04C88007D003700C04C800084
:1057A00001102000010060000000E000160032003F
:1057B000C0422300104078008040E900C04223002E
:1057C00001487800C0422300104078000004E00047
:1057D0006F003A00C04C80000080A100C04C8800DF
:1057E000C04C80000030A100C04C8800C04C80003C
:1057F0000020A100C04C8800C04C80000040A100E7
:10580000C04C880062003700C04C8000620060001D
:105810000000E0000C003200C04C80006800600016
:105820000000E00008003A001E0090006A00B90085
:10583000E8004000A08A2B000080400010007800A3
:10584000000F78002B003700C04C8000680060001B
:105850000000E000080032001E0090006A00B9005D
:10586000E6004000A08A2B00008040001000780075
:10587000000F78001F003700C04C800070006000EF
:105880000000E000080032001E0090006A00B9002D
:10589000E4004000A08A2B00008040001000780047
:1058A000000F780013003700C04C800064006000D7
:1058B0000000E000080032001E0090006A00B900FD
:1058C0008080E800A08A2B00008040001000780053
:1058D000000F7800070037001E0090006A00B90032
:1058E00080007800A08A2B00008040001000780023
:1058F000000F78000091200010407800E74F500022
:105900001E003A00F00F20009E0F10001B003C000C
:105910001E00E00019003500000620009E0F100058
:1059200006003400A00720009E0F100003003C007A
:1059300000FE2F001E0F400008003700000420006A
:105940009E0F100005003400A00520009E0F1000DF
:1059500002003C00000220001E0F4000F101200068
:105960009E8F100005003400D0198200E10F500016
:1059700002003A00000820001E0F70001E01900077
:10598000E2CC88001E007800068B020000000000B8
:1059900001DA8000F0D98000808F5000BDFE3A000F
:1059A0000080FA00000006000A00FA00F600370046
:1059B0001E0078008000780000002800808F5000D2
:1059C000070036009E007800F0FF2700008060008E
:1059D000000F78001E00780000000100EA00370088
:1059E000E0198200E60F5000A4003A00D0198200AE
:1059F0000000E000A10032001E0078006101B90043
:105A0000B0FD2F00F1FF2F0002014000838148000C
:105A100032079800430798009005200001002000FD
:105A20003E019000CE019000800F5100818F5900FF
:105A300092003E003E009000CE0090000060010009
:105A4000590037008D0037008C0037008B0037007D
:105A50008A0037005D0037007A0037008700370082
:105A6000810037008500370084003700830037004D
:105A70008200370081003700800037007F00370048
:105A80007E0037007D0037007C0037007B00370048
:105A90007A00370079003700780037005D00370062
:105AA0006B0037005E00370074003700410037009C
:105AB0007200370071003700700037006F00370048
:105AC0006E0037006D0037006C0037006B00370048
:105AD0006A00370069003700680037006700370048
:105AE0006600370065003700640037006300370048
:105AF0006200370061003700600037005F00370048
:105B00005E0037005D0037005C0037005B00370047
:105B10005A0037005900370035003700550037006C
:105B200036003700260037004C00370042003700AF
:105B30005200370051003700500037004F00370047
:105B40004E0037004D0037004C0037004B00370047
:105B50004A00370049003700480037004700370047
:105B60004600370045003700440037004300370047
:105B70004200370041003700400037003F00370047
:105B80003E0037003D0037003C0037003B00370047
:105B90003A003700390037000F0037001A0037008D
:105BA000100037002100370000022000000F7800AD
:105BB0003200370000022000000F78002F0037006D
:105BC00000022000000F78002C00370000022000A7
:105BD000000F78002900370000022000000F780035
:105BE0002600370000022000000F78002300370055
:105BF00000022000000F7800200037000002200083
:105C0000000F78001D00370000022000000F780010
:105C10001A00370000022000000F7800170037003C
:105C200000022000000F780014003700000220005E
:105C3000000F78001100370000022000000F7800EC
:105C40000E00370000022000000F78000B00370024
:105C500000022000000F780008003700000220003A
:105C6000000F78000500370000022000000F7800C8
:105C70000200370000022000000F7800D1198200D6
:105C8000210798002E019000E10F51003A003200E8
:105C9000AE019000E18F510004003C002E00900006
:105CA0000000E0000800320037003700AE0090002E
:105CB000E88F5000090032002E019000E90F5100DA
:105CC00029003200300037001E0078000000FB0081
:105CD000628B0200000000002B003700C04C8000E7
:105CE00001002800010060000000E00026003200F2
:105CF0001E00780076720200000000001E0078008E
:105D0000E80F500004003A00404880000000E9001D
:105D1000404888001C0037000091200010407800A7
:105D2000E74F500003003A000304200013079800D7
:105D3000020037000000EB00100798001E007800FA
:105D40008040780040488000800178000000E80032
:105D5000404888001E01900003007800762502006C
:105D600000000000080037001E0078007672020074
:105D700000000000040037001E0078008000EB00E7
:105D80005C64020000000000248B020000000000A0
:105D9000000F78001E0078000000E00004FF3A00C9
:105DA0000080FA00000006000000FA00103B8200AC
:105DB000000001000080FA00000006000000FA0068
:105DC000B03A8200000001000080FA0000000600E6
:105DD0000000FA00E03A8200000001000080FA00B2
:105DE000000006000000FA00203B820000000100D5
:105DF0000080FA00000006000000FA00303B82003C
:105E0000000001000080FA00000006000000FA0017
:105E1000503B8200000001000080FA0000000600F4
:105E20000000FA00603B8200000001000080FA00E0
:105E3000000006000000FA00703B82000000010034
:105E40000080FA00000006000000FA00903B82008B
:105E5000000001000080FA00000006000000FA00C7
:105E6000A03B8200000001000080FA000000060054
:105E70000000FA00803B8200000001000080FA0070
:105E8000000006000000FA00B03B820000000100A4
:105E90000080FA00000006000000FA00C03B82000B
:105EA000000001000080FA00000006000000FA0077
:105EB000D03B8200000001000080FA0000000600D4
:105EC0000000FA00E03B8200000001000080FA00C0
:105ED000000006000000FA00F03B82000000010014
:105EE0000080FA00000006000000FA00003C82007A
:105EF000000001000080FA00000006000000FA0027
:105F0000D03A8200000001000080FA000000060084
:105F10000000FA00F03A8200000001000080FA0060
:105F2000000006000000FA00003B820000000100B3
:105F30000080FA00000006000000FA00103C820019
:105F4000000001000080FA00000006000000FA00D6
:105F5000203C8200000001000080FA0000000600E2
:105F60000000FA00303C8200000001000080FA00CE
:105F7000000006000000FA00403C82000000010022
:105F80000080FA00000006000000FA00503C820089
:105F9000000001000080FA00000006000000FA0086
:105FA000603C8200000001000080FA000000060052
:105FB0000000FA00703C8200000001000080FA003E
:105FC000000006000000FA00803C82000000010092
:105FD0000080FA00000006000000FA00903C8200F9
:105FE000000001000080FA00000006000000FA0036
:105FF000A03C8200000001000080FA0000000600C2
:106000000000FA00B03C8200000001000080FA00AD
:10601000000006000000FA00C03C82000000010001
:106020000080FA00000006000000FA00D03C820068
:10603000000001000080FA00000006000000FA00E5
:10604000E03C8200000001000080FA000000060031
:106050000000FA00F03C8200000001000080FA001D
:10606000000006000000FA00003D82000000010070
:106070000080FA00000006000000FA00B03D820037
:10608000000001000080FA00000006000000FA0095
:10609000103D8200000001000080FA0000000600B0
:1060A0000000FA00203D8200000001000080FA009C
:1060B000000006000000FA00303D820000000100F0
:1060C0000080FA00000006000000FA00403D820057
:1060D000000001000080FA00000006000000FA0045
:1060E000503D8200000001000080FA000000060020
:1060F0000000FA00603D8200000001000080FA000C
:10610000000006000000FA00703D8200000001005F
:106110000080FA00000006000000FA00803D8200C6
:10612000000001000080FA00000006000000FA00F4
:10613000903D8200000001000080FA00000006008F
:106140000000FA00C03D8200000001000080FA005B
:10615000000006000000FA00A03D820000000100DF
:106160000080FA00000006000000FA00D03D820026
:10617000000001000080FA00000006000000FA00A4
:10618000E03D8200000001000080FA0000000600EF
:106190000000FA00F03D8200000001000080FA00DB
:1061A000000006000000FA00003E8200000001002E
:1061B0000080FA00000006000000FA00103E820095
:1061C000000001000080FA00000006000000FA0054
:1061D000203E8200000001000080FA00000006005E
:1061E0000000FA00303E8200000001000080FA004A
:1061F000000006000000FA00403E8200000001009E
:106200000080FA00000006000000FA00503E820004
:10621000000001000080FA00000006000000FA0003
:10622000603E8200000001000080FA0000000600CD
:106230000000FA00703E8200000001000080FA00B9
:10624000000006000000FA00803E8200000001000D
:106250000080FA00000006000000FA00903E820074
:10626000000001000080FA00000006000000FA00B3
:10627000A03E8200000001000080FA00000006003D
:106280000000FA00B03E8200000001000080FA0029
:10629000000006000000FA00C03E8200000001007D
:1062A0000080FA00000006000000FA00D03E8200E4
:1062B000000001000080FA00000006000000FA0063
:1062C000E03E8200000001000080FA0000000600AD
:1062D0000000FA00F03E8200000001000080FA0099
:1062E000000006000000FA00003F820000000100EC
:1062F0000080FA00000006000000FA00103F820053
:10630000000001000080FA00000006000000FA0012
:10631000203F8200000001000080FA00000006001B
:106320000000FA00303F8200000001000080FA0007
:10633000000006000000FA00403F8200000001005B
:106340000080FA00000006000000FA00503F8200C2
:10635000000001000080FA00000006000000FA00C2
:10636000603F8200000001000080FA00000006008B
:106370000000FA00703F8200000001000080FA0077
:10638000000006000000FA00803F820000000100CB
:106390000080FA00000006000000FA00903F820032
:1063A000000001000080FA00000006000000FA0072
:1063B000A03F8200000001000080FA0000000600FB
:1063C0000000FA00B03F8200000001000080FA00E7
:1063D000000006000000FA00C03F8200000001003B
:1063E0000080FA00000006000000FA00403B820036
:1063F000000001000080FA00000006000000FA0022
:10640000C03A8200000001000080FA00000006008F
:106410000000FA00E001A90000000000E021A9004E
:1064200000000000E041A90000000000011E200063
:106430009140780070CEB30000C06000E0E1B7008A
:1064400000000000E0A1A90000000000E0C1A900D8
:1064500000000000E0E1A90000000000E1C1BF0071
:106460007040B300E1E1B70000000000E1A1A90025
:1064700000000000E1E1A900211E20009140780009
:1064800000C7B30000C07000E2E1B70000000000E8
:10649000E2E1A80000000000E301A8000000000005
:1064A000311E20009140780090CFB30000C0600002
:1064B000E3E1B70040062000200F88000080EB00D9
:1064C000300F8800E522A8006960A80000000000E5
:1064D00068C0A8000000000068E0A8008B40A90088
:1064E0009B40A9000080FA00000006000A00FA00A4
:1064F000300798003E009000024020001100090083
:106500000200D800200798003E00900002402000C2
:10651000110009000200D8008000FD00100798005B
:106520002E009000400798004E009000E10F5000B0
:10653000140032004E009000E10F500004003C00B7
:106540004E0090000000E0000800320024003700F8
:106550004E009000E20F5000120032004E009000FA
:10656000E30F5000160032001D0037001E0090009F
:1065700080004000808A2A0000804000100F7800D0
:1065800017003700014020001E00900000805000DE
:1065900080004000808A2A0000804000100F7800B0
:1065A0000F0037001E00900080004000808A2A0003
:1065B0000080400010007800000FEA00080037005B
:1065C000014020001E00900000805000800040002C
:1065D000808A2A000080400010007800000FEA0046
:1065E0001E0078000080FA00000006003600F80067
:1065F000809FBE00829FBE00849FBE00869FBE001B
:10660000881F78003400F80020002000A0018800D6
:106610000200FA00E01281000000E800E0128900A8
:10662000E112810000F42100808F500005003A0043
:106630002040800000D0A000204088000000EB0037
:10664000E012890090CD80000000E80090CD880025
:1066500091CD800080CD8000808F500005003900F2
:106660000000EB0090CD880030CD80000000E800F5
:1066700030CD880050A081000000E80050A08900C3
:1066800051A08100E03F8200808F5000050035005E
:106690000000EB0050A0890040CD80000000E80021
:1066A00040CD8800F09F8100FC0F500010003400A6
:1066B00050A081000000E0001F003A0040CD8000A3
:1066C00061406000614060006140600061406000C6
:1066D00000414000612D200091407800D0CFB300F0
:1066E00000C0600002407000D6E2B7001200370020
:1066F00060A081000000E0000F00320090CD80001B
:106700000000E0000C003A0030CD800061406000E5
:1067100061406000614060006140600000414000F5
:10672000612D200091407800D0CFB30000C0600000
:1067300002407000D6E2B700C04C80000104200087
:10674000010060000000E00003003200304C8000D7
:106750000000E800304C8800D01281000000E80002
:10676000D0128900D0198200000F78009E007800B6
:10677000E18F5000640032001E007800E10F5000ED
:1067800004003C009E0078000100E000060032009A
:10679000940037009E00780063805000E30F5000A3
:1067A00090003E0058003700C1CD8000D0CD800061
:1067B00000807000A0CD8800E0198200E70F500033
:1067C00020003A00A0CD80000000E000110032005F
:1067D00070CD80000000E0000E00320030CD80005F
:1067E00022002000110009000200D8008000FD00F6
:1067F000614060006140600000414000612D200068
:1068000091407800D0CFB30000C06000024070001B
:10681000D6E2B700D03F82000000E00009003A0055
:1068200000D2020000000000C01281008000400081
:10683000C09920000080400010007800F0C00200E5
:1068400000000000C04C8000010420000100600036
:106850000000E00063003A00C8128100068C0200CC
:10686000000000000001780088004400C09920006A
:106870000080400002087800C01281000000E8009B
:10688000C0128900C112810000402000808F50009A
:106890000B003A00E0198200E60F500003003A00B6
:1068A0001000200020DA880003003700C04C800070
:1068B00000B0A000C04C88000000EB00B0128900BE
:1068C000C112810000802000808F500045003A00F6
:1068D0000000EB00C0128900E0198200E60F5000B2
:1068E00003003A001000200020DA8800030037007F
:1068F000C04C800000B0A000C04C880000402000C8
:10690000B0128900370037000000EB00A0CD8800EE
:10691000B0CD80000000E0001100320060CD8000AA
:106920000000E0000E00320030CD80002200200088
:10693000110009000200D8008000FD0061406000E5
:106940006140600000414000612D200091407800CE
:10695000D0CFB30000C0600002407000D6E2B700A4
:10696000902D2300104078000004E0000A0032005F
:10697000B0CD800061406000614060000041400097
:10698000212E200091407800D0CFB30000C06000DD
:1069900002407000E2E2B7000000EB0030338A00F2
:1069A000D03F82000000E00002003A00A85A020036
:1069B00000000000D1128100F0182000808F5000EC
:1069C000080034000000EB00D01289002040800055
:1069D0000070A000204088002040800000E0A0005F
:1069E00020408800D1128100F0182000808F5000D4
:1069F000050034000000EB00D01289002040800028
:106A00000070A000204088008460A9000080FA0087
:106A10003400F9004F0478004F03BE004F02BE005F
:106A20004F01BE004F00BE003600F90000400600D6
:106A30003600F800809FBE00829FBE00849FBE008B
:106A4000869FBE003400F80020002000A0018800CE
:106A50001200FA0010CD80000000E80010CD880080
:106A600071A0810061806000004178000100E800B1
:106A700070A089000204E0002E003200B09B81006B
:106A80000000E900B09B8900B09B81000000E0009D
:106A900005003A00809B81000000E800809B89008F
:106AA000803E2000B09B8900513482007038210064
:106AB000808F500006003C00503482000000E0004F
:106AC0000300350010002000600798000200370026
:106AD0008000EB0061079800503482006E01900046
:106AE0000000410050348A002135820070382100B6
:106AF000808F500006003C00203582000000E0003E
:106B000003003500130020005307980002003700EF
:106B10000000EB005007980020358200DE00900056
:106B20000080400020358A00E0CD80000000E800B1
:106B3000E0CD880040A081000000E0000B003A009A
:106B4000CFC2BF000042B2000001EB004207980034
:106B50000004E00002003A00130020004307980000
:106B60004E009000D0CD8800DA003700F03F820060
:106B70000000E00009003200D4C2BF0061406000A4
:106B80008000EB00310798000004E0000B003A00A1
:106B9000120020003207980008003700CFC2BF0063
:106BA0000042B2008001EB00330798000004E000CF
:106BB00002003A001000200030079800BE0090004C
:106BC00011079800F03F82000000E0000900320049
:106BD000CFC2BF000042B2000001EB0022079800C4
:106BE0000004E0000B003A00130020002307980087
:106BF00008003700D4C2BF00614060008000EB0095
:106C0000210798000004E00002003A001200200072
:106C100022079800AE019000030F78000000EB00FF
:106C2000D0CD880000A081000000E90000A089000C
:106C300000A081000000E0000A003C00909D81005F
:106C400000A08900F09F81000000E900F09F89000A
:106C5000F09F81000000E00002003C000000EB001B
:106C6000F09F8900F09F81006101B90072079800D0
:106C7000030F980080022000010020007E01900098
:106C80008E099000800F5100818F590091003E00C5
:106C90007E0090008E089000006001007B003700AD
:106CA0007A00370079003700780037007700370026
:106CB00076003700750037006C0037006B00370036
:106CC000600037004C0037004B0037004A003700A7
:106CD00049003700480037004700370046003700BA
:106CE0003D0037003C0037003B0037003A003700DA
:106CF0002F0037001E0037001D0037001C00370032
:106D00000F0037000E0037000D0037000C00370071
:106D10000B0037000A003700090037000800370071
:106D20000700370006003700050037000400370071
:106D30000300370002003700010037000000370071
:106D400020A081000000E00005003200A09D81002D
:106D50009E00900001007000A09D89005D0037003A
:106D6000B09D81001E007000B09D89005900370061
:106D7000B09D81001E007000B09D8900A19D810022
:106D80001E00900000807000A09D8900A09D8100E1
:106D90000000E00003003A00B09D81000000E00028
:106DA0004C00320038DE02000000000049003700CD
:106DB000D09F81000000E00007003A00813B2300E3
:106DC00010C0B300804878001000200010A0890097
:106DD00010002000D09F8900A19D81001E0090001E
:106DE00000807000A09D8900B09D81001E00700091
:106DF000B09D890037003700A19D81001E009000E2
:106E000000807000A09D8900B09D81001E00700070
:106E1000B09D890010A081000000E0002D003A0024
:106E2000A09D81000000E00003003A00B09D8100B9
:106E30000000E0002700320038DE02000000000001
:106E400024003700E09F81000000E00007003A00C6
:106E5000813B230020C0B300804878001000200050
:106E600010A0890010002000E09F8900A19D8100F2
:106E70001E00900000807000A09D8900B09D8100E0
:106E80001E007000B09D890012003700A19D810096
:106E90001E00900000807000A09D8900B09D8100C0
:106EA0001E007000B09D890010A081000000E0006D
:106EB00008003A00A09D81000000E00003003A00B5
:106EC000B09D81000000E0000200320038DE0200C8
:106ED000000000008760A9000080FA003400F9007B
:106EE0004F03BE004F02BE004F01BE004F00BE0068
:106EF0003600F90000400600801F78003400F800DA
:106F000020002000A00188000000FA0010002000EE
:106F100010DA88008A00A9000080FA003400F90025
:106F20004F007800004006002400FA00700F98001F
:106F3000F1008000E0FB2F0000804000100078008E
:106F40006F00600030079800F1008000C0FB2F0048
:106F50000080400090007800210798000000EB00BE
:106F6000100798000E0037009E0190007E089000E8
:106F70000000E9001E0190007400B900820040008A
:106F800040712C00E140780068004700008041001B
:106F9000014878001E0090000000E80010079800EB
:106FA0001E009000F30F5000EFFF34003E009000F1
:106FB0006F4F6000F0002000100798001B003700A2
:106FC0001E0190001217980090C0B3009E4F100051
:106FD0000300340071C3B30001679800020037005A
:106FE00002C3B300026798000E6090009E4040000C
:106FF000680047001E119000000041000148780021
:10700000AE00900000002F00008060004C00DE0009
:10701000004F78002E0090004400DD00200798000B
:107020001E0090000000E800100798001E0090006D
:10703000F30F5000E2FF3400680047008040EB008F
:1070400041509800680147008040EB0040C0B30009
:107050007A71020000000000000000000000000043
:10706000FFFF37003600F800809FBE00829FBE0001
:10707000849FBE00869FBE003400F80020002000E0
:10708000A00188000000FA0010002000A6FF070001
:107090000080FA003400F9004F03BE004F02BE002A
:1070A0004F01BE004F00BE003600F9000040060050
:1070B0003600F800809FBE00829FBE00849FBE0005
:1070C000869FBE003400F80020002000A001880048
:1070D0000000FA002000200093FF07000080FA0063
:1070E0003400F9004F03BE004F02BE004F01BE0046
:1070F0004F00BE003600F900004006003600F800E0
:10710000809FBE00829FBE00849FBE00869FBE00FF
:107110003400F80020002000A00188000000FA00E0
:107120003000200080FF07000080FA003400F900E2
:107130004F03BE004F02BE004F01BE004F00BE0015
:107140003600F900004006003600F800809FBE00BF
:10715000829FBE00849FBE00869FBE003400F80060
:1071600020002000A00188000000FA00400020005C
:107170006DFF07000080FA003400F9004F03BE00E5
:107180004F02BE004F01BE004F00BE003600F900A6
:10719000004006003600F800809FBE00829FBE00BF
:1071A000849FBE00869FBE003400F80020002000AF
:1071B000A00188000000FA00500020005AFF0700DC
:1071C0000080FA003400F9004F03BE004F02BE00F9
:1071D0004F01BE004F00BE003600F900004006001F
:1071E0003600F800809FBE00829FBE00849FBE00D4
:1071F000869FBE003400F80020002000A001880017
:107200000000FA007000200047FF07000080FA002D
:107210003400F9004F03BE004F02BE004F01BE0014
:107220004F00BE003600F900004006000200FA00E0
:10723000000F78001E0078004300DE00610060004F
:107240000004E0000300320010002000803B8900B1
:10725000020037000000EB00803B890070FF2F0028
:107260001E006000E0198A000080FA00000006009D
:107270000200FA00008181000000E00003003400F9
:1072800000818100000F7800020037000000EB0051
:10729000000F78001E0078000080FA000000060051
:1072A0000400FA00000F7800110798001E00780013
:1072B000108189001E0090000000E00003003A00E9
:1072C00040012000F0808900080037001E00900077
:1072D000E10F500003003A00B0042000F080890064
:1072E000020037001E009000F08089000080FA0044
:1072F000000006000400FA00000F78001E0078006D
:10730000CAFF0700C04C80000090A100C04C88005C
:10731000780007001E007800100798009E0090007B
:10732000E68F5000190032001E009000E60F50005A
:1073300005003C009E00900060804000E20F50007D
:107340001A003E00040037001E009000E70F5000B6
:107350000100320015003700C04C800000B0A100D1
:10736000C04C88002900070074580200000000008B
:1073700000002000A11F2400B0268A00C1268A0038
:10738000A658020000000000080037000000EB00D3
:1073900020DA8800D0CC2C0051232400B0268A00AB
:1073A000C1268A00AA24020000000000B226820042
:1073B000C32682000000200001F82300120702000B
:1073C0000000000050278A0061278A000000EB00BF
:1073D000209689000000EB00309689000000EB0049
:1073E000D0198A004E710200000000008040EB00BE
:1073F00070C0B300B8730200000000000000EB0092
:10740000D03F8A000080FA00000006000000FA0069
:107410000000EB00C08089000000EB00E0808900E4
:107420000000EB00503B89006000B800A08189009B
:10743000B1818900B0042000F08089002003200081
:1074400010818900E0968100F1968100B2FD200054
:10745000930C2400960702000000000002002000A8
:10746000A35F24001207020000000000C08589000D
:10747000D1858900C0972D0001D2230000868900A4
:1074800011868900C0858100D18581000286810036
:107490001386810000080200000000002086890099
:1074A00031868900C0858100D185810002868100F6
:1074B00013868100FE07020000000000408689005C
:1074C000518689000000EB00960007000000EB00E9
:1074D000D0198A00DE22A900E222A900C04C800057
:1074E0000070A100C04C8800000000000080FA007D
:1074F000000006000600FA000000EB00000F780014
:107500002C0037001E017800217722000040EB009C
:1075100000F178000000EB00100798002000370011
:107520001E00900080004000A06C280000804000F9
:1075300090007800210798002E0090004400DE00A3
:1075400020079800030037002E0090000000D100B3
:10755000200798002E009000610060000000E0000D
:10756000F9FF32002E0090000000D10020079800A3
:107570009E0078002E009000808F500005003A0099
:107580001E0178001E0090008040780020772200C5
:10759000017178001E0090000000E80010079800BC
:1075A0009E009000F00F2000808F5000DCFF340020
:1075B0001E0FE800F07F20009E0F1000D1FF340066
:1075C000430107000000EB005600070020032000E5
:1075D000008189006000B800008389001183890060
:1075E0000000EB00907B89000000EB00703B8900FD
:1075F0000000EB00808189000000EB0060818900C1
:107600000000EB00708189006000B800508B890099
:10761000618B89006000B800D08B8900E18B890004
:107620000000EB00008B890050002000108B8900C7
:107630000000EB00208B89006000B8008082890088
:10764000918289006000B80060828900718289009F
:107650006000B800C0828900D18289006000B80053
:10766000A0828900B1828900D0CC2C00C1EC23001B
:107670004082890051828900E21723006000B8002F
:107680000089BE00E21723006000B80020019800C6
:1076900031019800621823006000B8000089BE0024
:1076A000621823006000B8002001980031019800A2
:1076B0006000B800908B8900A18B89006000B80041
:1076C000908B8900A18B89006000B800B08B890085
:1076D000C18B89000000EB00508189000000EB00A5
:1076E000603B89000000EB00A08089000000EB00F7
:1076F000403B89000000EB00303B89000000200087
:10770000812C240060868900718689008040EB000E
:1077100070C0B300B8730200000000000080FA00DF
:10772000000006000200FA00000F78001E0078003A
:10773000CF80DE00BA080200000000000200200036
:10774000A35F240096070200000000000240220010
:1077500043972400120702000000000010090200F5
:1077600000000000C0808900C0808100CF80DE0062
:10777000BA0802000000000002002000A35F2400FD
:107780000008020000000000E0858900F185890002
:10779000E2858100F3858100B0FD2000910C24007A
:1077A0001207020000000000E2968100F3968100BB
:1077B0009607020000000000C0858900D18589007D
:1077C000E2858100F385810000002000011824007B
:1077D0001207020000000000E0828900F1828900A7
:1077E0000080FA00000006000400FA00100798006C
:1077F0000000EB00000F78000C0037001E0078003E
:107800004200DD00800078001E00900000814000F2
:107810001E007800C200DD0040F72200008040001A
:107820001000BE000089BE001E0FE800F00020001E
:107830009E0F1000F1FF34000080FA0000000600E7
:107840000400FA00100798000000EB00000F780019
:107850000C0037001E0078004200DD008000780038
:107860001E009000008140001E007800C200DD0074
:1078700040FC2200008040001000BE000089BE00D5
:107880001E0FE800F00020009E0F1000F1FF3400F2
:107890000080FA00000006000400FA00008FBE001D
:1078A00010002000403B8900B2FD2000930C240012
:1078B0001E00BE009607020000000000E285810065
:1078C000F38581001207020000000000C0858900D6
:1078D000D18589006000B800908B8900A18B890058
:1078E0006000B800708B8900818B8900303B81007B
:1078F0000000E0000300320040002000A08089006A
:107900000200370040012000A0808900C08581006E
:10791000D185810002868100138681000008020063
:10792000000000002086890031868900C085810022
:10793000D18581000286810013868100FE07020046
:107940000000000040868900518689004086810041
:10795000518681006011B800520902000000000049
:107960000000E00001003400030037006000B800B0
:1079700040868900518689000000EB00308B890029
:107980000000EB00408B89000080FA000000060038
:107990000200FA00000F78001E00E00003003A0029
:1079A0000000EB00B08089000200370010002000CA
:1079B000B080890080BB20009E0F100003003A00B9
:1079C00010002000303B8900020037000000EB006F
:1079D000303B89001E007800CF80DE00BA0802002C
:1079E00000000000B2FD2000930C24009607020066
:1079F00000000000E2858100F3858100120702008B
:107A0000000000000086890011868900C085810081
:107A1000D1858100A2818100B3818100000802002C
:107A20000000000002868100138681000008020029
:107A3000000000002086890031868900C085810011
:107A4000D1858100A2818100B381810000080200FC
:107A5000000000000286810013868100FE070200FC
:107A60000000000040868900518689004086810020
:107A7000518681006011B800520902000000000028
:107A80000000E00001003400030037006000B8008F
:107A90004086890051868900303B81000000E0006B
:107AA0000500320000002000011F240060868900CC
:107AB000718689000400370000002000812C24001A
:107AC00060868900718689000080FA000000060047
:107AD0000200FA000000EB00000F780015003700EC
:107AE0001E007800C300DD00000E2300008140006E
:107AF0006000B8000089BE001E0078004300DD0071
:107B0000E4004000000E2300008140006000B80047
:107B10000089BE001E007800C200DD0040F7220090
:107B20000081400010002000010020000089BE00FC
:107B30001E0FE800F00020009E0F1000E8FF340048
:107B40000000EB00000F78000A0037001E007800EC
:107B5000C200DD0040062300008140006000B80044
:107B60000089BE0040BE2C0061092400060B0700FE
:107B70001E0FE800400120009E0F1000F3FF3400AC
:107B8000A0002000008189000000EB003081890006
:107B90000000EB00208189000000EB00408189009B
:107BA00000002000412B240040828900518289007E
:107BB0000080FA00000006000A00FA00889FBE005C
:107BC0000001200030079800008023002007980063
:107BD000208023001007980000E52100000F7800A6
:107BE000803B81000000E0000200320080002000A5
:107BF00030079800A08081000000E00034003200CF
:107C0000A08081000000E900A0808900A0808100A0
:107C10000000E0002C003C000000EB00A080890088
:107C20000000EB00403B8900C0858100D1858100C8
:107C30000286810013868100000802000000000017
:107C40002086890031868900C0858100D185810028
:107C50000286810013868100FE07020000000000FA
:107C60004086890051868900C0858100D1858100C8
:107C700002002000A35F240096070200000000001D
:107C8000B2FD2000930C2400120702000000000047
:107C9000E0968900F1968900408681005186810036
:107CA0006011B80052090200000000000000E0006E
:107CB00001003400060037006000B80040868900EB
:107CC000518689000200370010002000403B8900E7
:107CD0000000EB00708C89009E013700B11281001A
:107CE000708C81000080400080004000C09920001E
:107CF000008040001000780030358900B01281000B
:107D00000000E00042003A00718C8100F01F20006A
:107D1000808F50001E003C00708C810000004000ED
:107D20001E044000303581002200200011000900AF
:107D30000200D800CF80DE00BA0802000000000078
:107D40000002BE00708C8100C200DD00A08E280001
:107D5000008040001001BE000400BE009607020033
:107D6000000000001009020000000000000C780074
:107D7000708C810000004000800078002E00900090
:107D8000808040000000EB00800878007E00370013
:107D9000708C8100000040009E00400000C02F0059
:107DA00000844000708C8100000040009E00400074
:107DB00000C02F0000804000900478003035810022
:107DC00022002000110009000200D800CF80DE0050
:107DD000BA080200000000000002BE00708C8100A2
:107DE000C200DD00A08E2800008040001001BE000F
:107DF0000400BE0096070200000000001009020007
:107E00000000000000804400000C78005E00370095
:107E1000718C8100F01F2000808F50001E003C00FC
:107E2000708C8100000040001E044000708C8100B6
:107E3000000040001E0040009004780030358100B2
:107E400022002000110009000200D800CF80DE00CF
:107E5000BA080200000000000002BE00718C810020
:107E6000F03F200001005000C200DD00A08E28007D
:107E7000008040001001BE000400BE009607020012
:107E80000000000010090200000000000080440013
:107E9000000C780021003700708C81000000400049
:107EA0009E00400000C02F0000844000708C8100C4
:107EB000000040009E00400000C02F0000804000F5
:107EC0009004780030358100220020001100090064
:107ED0000200D800CF80DE00BA08020000000000D7
:107EE0000002BE00718C8100F03F200001005000B4
:107EF000C200DD00A08E2800008040001001BE00FE
:107F00000400BE00960702000000000010090200F5
:107F10000000000000804400000C7800718C81009B
:107F2000F03F2000808F500017003A00C04C8000C6
:107F30000090A000C04C88000000EB0040079800B3
:107F40000D0037004E0090000000400080007800D7
:107F50002E009000808040004E0090000000400005
:107F60001E00400010007800800878004E0090004D
:107F70000000E80040079800CE009000F01F2000AD
:107F8000808F5000EFFF3400C0858100D1858100D3
:107F9000A2818100B381810000080200000000007E
:107FA00032982F0023622400960702000000000090
:107FB00010090200000000000001BE000036810030
:107FC000113681000200400083804800003689009D
:107FD0001136890000368100113681004C09DD0020
:107FE0004400DE0000007100C488DE0080007800DC
:107FF000F0FF2000008060007632020000000000E8
:108000004035890000368100113681004C09DD00C1
:108010004400DE0000007100C488DE0080007800AB
:108020000040200080804000F0FF200000806000C1
:1080300076320200000000005035890030358100A2
:108040006104B900503581006103B90088007800EF
:1080500006007800000AB80007C0B90005017800E2
:108060000001410009B0B90000014100820278001E
:10807000E4358900F5358900303581006104B900A7
:10808000403581006103B90088007800060078005F
:10809000000AB80007C0B9000501780000014100DE
:1080A00009B0B9000001410082027800C43589009E
:1080B000D5358900E0358100F13581004109DD00C9
:1080C0004F00DE0000007100CF88DE00903589008F
:1080D000C0358100D13581004109DD004F00DE004F
:1080E00000007100CF88DE0080358900C033810038
:1080F000923581002169220000004000010040000B
:1081000002087800C0338100823581002168220096
:10811000000040000100400002087800C0338100E8
:108120000000E80042002000110009000200D80011
:108130008000FD00C0338900C03381000000E000F2
:1081400081003A00B03381000000400080007800D8
:10815000A06822008080400044002000639120003D
:1081600022692200100020004016020000000000DA
:10817000B03381000000400080007800A06722003A
:1081800080804000440020002393200022682200C9
:10819000100020004016020000000000E0198200DC
:1081A000E80F500008003A00B03381000000E800FA
:1081B00022002000110009000200D8008000FD000C
:1081C000B033890007003700B03381000000E800B9
:1081D00042002000110009000200D8008000FD00CC
:1081E000B0338900B03381000000E00056003A004F
:1081F0004400200043922000A2682200E16A22008D
:108200001000200040160200000000004400200082
:1082100003942000A2672200C16A220010002000FF
:1082200040160200000000007035810020358900F2
:108230006035810010358900E3942000E26A220055
:10824000016A220010002000A016020000000000B9
:10825000C3952000C26A2200E169220010002000BC
:10826000A016020000000000A3962000426A22002F
:10827000C169220010002000A016020000000000CA
:1082800083972000226A2200A169220010002000AA
:10829000A01602000000000000358100CF80DE0043
:1082A000BA08020000000000020D23000089BE0091
:1082B000F0348100CF80DE00BA0802000000000028
:1082C000020D23002001980031019800E034810064
:1082D000CF80DE00BA08020000000000820D2300FB
:1082E0000089BE00D0348100CF80DE00BA080200D1
:1082F00000000000820D2300200198003101980049
:10830000000D23005001BE004000BE0032040700F3
:10831000000D23005001BE004000BE0037030700DF
:10832000800D23005001BE004000BE00A1040700E4
:108330000000E00004003200800D23005001BE0068
:108340004000BE009B050700708C81000000E80023
:10835000708C8900718C8100F03F2000808F50006C
:108360005EFE34004F04BE000080FA0000000600EC
:108370002400FA00889FBE00008023002007980098
:10838000208023001007980000E52100000F7800EE
:10839000A0702D0031BA23001039890021398900DD
:1083A000C0858100D185810002002000A35F2400E8
:1083B0009607020000000000B2FD2000930C24008C
:1083C0001207020000000000E0968900F196890083
:1083D0000000EB005007980001033700B112810044
:1083E0005E0090000080400080004000C0992000A6
:1083F000008040001000780070388900B0128100C1
:108400000000E00042003A00DE009000F01F200073
:10841000808F50001E003C005E0090000000400075
:108420001E04400070388100220020001100090065
:108430000200D800CF80DE00BA0802000000000071
:108440000002BE005E009000C200DD00A08E280089
:10845000008040001001BE000400BE00960702002C
:10846000000000001009020000000000000C78006D
:108470005E00900000004000800078002E00900018
:10848000808040000000EB00800878007E0037000C
:108490005E009000000040009E00400000C02F00E1
:1084A000008440005E009000000040009E004000FC
:1084B00000C02F00008040009004780070388100D8
:1084C00022002000110009000200D800CF80DE0049
:1084D000BA080200000000000002BE005E0090002A
:1084E000C200DD00A08E2800008040001001BE0008
:1084F0000400BE0096070200000000001009020000
:108500000000000000804400000C78005E0037008E
:10851000DE009000F01F2000808F50001E003C0005
:108520005E009000000040001E0440005E009000CD
:10853000000040001E004000900478007038810068
:1085400022002000110009000200D800CF80DE00C8
:10855000BA080200000000000002BE00F13F200047
:108560005E00900000805000C200DD00A08E280058
:10857000008040001001BE000400BE00960702000B
:10858000000000001009020000000000008044000C
:10859000000C7800210037005E00900000004000D1
:1085A0009E00400000C02F00008440005E0090004C
:1085B000000040009E00400000C02F0000804000EE
:1085C000900478007038810022002000110009001A
:1085D0000200D800CF80DE00BA08020000000000D0
:1085E0000002BE00F13F20005E00900000805000BD
:1085F000C200DD00A08E2800008040001001BE00F7
:108600000400BE00960702000000000010090200EE
:108610000000000000804400000C7800DE009000A4
:10862000F03F2000808F500017003A00C04C8000BF
:108630000090A000C04C88000000EB0040079800AC
:108640000D0037004E0090000000400080007800D0
:108650002E009000808040004E00900000004000FE
:108660001E00400010007800800878004E00900046
:108670000000E80040079800CE009000F01F2000A6
:10868000808F5000EFFF3400C0858100D1858100CC
:10869000A2818100B3818100000802000000000077
:1086A00032982F0023622400960702000000000089
:1086B00010090200000000000001BE00D039810056
:1086C000E13981000200400083804800D0398900F0
:1086D000E1398900D0398100E13981004C09DD00A0
:1086E0004400DE0000007100C488DE0080007800D5
:1086F000F0FF2000008060007632020000000000E1
:1087000080388900D0398100E13981004C09DD00D1
:108710004400DE0000007100C488DE0080007800A4
:108720000040200080804000F0FF200000806000BA
:108730007632020000000000903889007038810015
:108740006104B900903881006103B90088007800A5
:1087500006007800000AB80007C0B90005017800DB
:108760000001410009B0B900000141008202780017
:108770007439890085398900703881006104B90035
:10878000803881006103B900880078000600780015
:10879000000AB80007C0B9000501780000014100D7
:1087A00009B0B90000014100820278005439890003
:1087B0006539890070398100813981004109DD0006
:1087C0004F00DE0000007100CF88DE00D038890045
:1087D00050398100613981004109DD004F00DE0020
:1087E00000007100CF88DE00C0388900803781002A
:1087F000D23881006170220000004000010040007A
:108800000208780080378100C2388100E16F2200C1
:10881000000040000100400002087800803781001D
:108820000000E80042002000110009000200D8000A
:108830008000FD0080378900803781000000E00063
:10884000E4013A00703781000000400080007800A9
:10885000A06F22008080400044002000E3942000AC
:10886000627022001000200040160200000000008C
:10887000703781000000400080007800606F2200A7
:108880008080400044002000C3952000E26F220059
:108890001000200040160200000000007037810028
:1088A0000000E80022002000110009000200D800AA
:1088B0008000FD0070378900703781000000E00003
:1088C000C4013A0024002000A3962000A26F2200D9
:1088D000617122001000200040160200000000001C
:1088E0002400200083972000626F22004171220043
:1088F000100020004016020000000000B038810087
:10890000CF80DE00BA08020000000000D0368900E7
:10891000E1368900A0388100CF80DE00BA0802006D
:1089200000000000B0368900C1368900D0368100D1
:10893000E1368100D2368100E336810096070200DD
:10894000000000000004BE00B0368100C136810086
:10895000B2368100C3368100960702000000000095
:108960000001BE000800BE00000802000000000078
:10897000F036890001378900D0368100E136810068
:1089800072368100833681009607020000000000E5
:108990000004BE0090368100A1368100B23681000D
:1089A000C336810096070200000000000001BE00EF
:1089B0000800BE00FE07020000000000827A2200CC
:1089C000F3312400960702000000000010378900F0
:1089D00021378900123981002339810000002000ED
:1089E00001F82300FE07020000000000923781001A
:1089F000A337810096070200000000000004BE00BB
:108A0000F0368100013781005609020000000000A5
:108A1000123981002339810096070200000000000E
:108A20000001BE000800BE000008020000000000B7
:108A300090378900A1378900F03681000137810025
:108A40006011B800C0090200000000000000E00052
:108A500001003A001700370050368100613681006E
:108A6000A299290093F1230096070200000000005C
:108A70000004BE001037810021378100F2368100EA
:108A8000033781001207020000000000D2CC2C0046
:108A9000C3EC230096070200000000000001BE00A6
:108AA0000800BE00000802000000000050368900E7
:108AB000613689005036810061368100100902005C
:108AC00000000000403689004036810010179800F1
:108AD0001E1090000000E00003003D009E1090007A
:108AE0008100EA0011179800B0FA2F001E119000C3
:108AF000000041000017980040368100700F980078
:108B00007E0890000000E00003003D00FE08900099
:108B10008100EA00710F9800B0FA2F007E099000E2
:108B2000000041000E1190000090B900CF80DE00DF
:108B300020368900313689001239810023398100BD
:108B40000000200001F82300FE07020000000000E2
:108B5000323981004339810096070200000000008D
:108B60000004BE002036810031368100BA080200C0
:108B700000000000123981002339810096070200AD
:108B8000000000000001BE000800BE000008020056
:108B900000000000303989004139890030398100F6
:108BA0004139810002002000A34F24005209020035
:108BB000000000000000E000010035000300370065
:108BC00010002000603B8900020037000000EB002D
:108BD000603B8900D0368100E13681009036890003
:108BE000A1368900B0368100C13681007036890017
:108BF0008136890030408000680060000000E0009D
:108C00000F003A004136810080022000808F500022
:108C100003003400616E220010C0B3008048780069
:108C20004136810080FD2F00808F500012003D00F2
:108C3000616E22000040EB00804878000E00370093
:108C40004136810080022000808F500003003400F4
:108C5000616E22000040EB008048780041368100C0
:108C600080FD2F00808F500003003D00616E2200C8
:108C700010C0B30080487800C06E22001040780019
:108C80000080FB00600F98006E089000E10F50001C
:108C900019003200EE089000E28F500046003200CA
:108CA0006E0990000200E00001003200C9003700A8
:108CB000606E2200104078000004E000C5003A0019
:108CC000706E2200104078008040E800706E220034
:108CD00001487800C16E220010C0B30080487800BF
:108CE000A06E2200104078008040E800A06E2200B4
:108CF00001487800B7003700606E2200104078000D
:108D00000004E00005003A00706E22001040780078
:108D10008040E800706E220001487800A06E2200BA
:108D200010407800F64F50001D003A00706E22008F
:108D300010407800EB4F50000C003600C16E22004E
:108D400020C0B30080487800816E220000C0EB0094
:108D500080487800906E2200104078008040E80043
:108D6000906E22000148780006003700C16E220094
:108D70000040EB0080487800916E22000040EB003C
:108D800080487800A16E22000040EB008048780007
:108D9000716E22000040EB00804878008D003700A3
:108DA000A06E2200104078008040E800A06E2200F3
:108DB0000148780087003700606E2200104078007C
:108DC0000004E00005003A00706E220010407800B8
:108DD0008040E800706E220001487800A06E2200FA
:108DE00010407800F64F500023003A00806E2200B9
:108DF000104078000080FB000000D1008040780027
:108E0000806E220001487800806E220010407800B9
:108E1000804078000174A100806E22000148780033
:108E2000706E220010407800EA4F500006003E00AD
:108E3000806E22009040780000C8B30080C07000AF
:108E4000806E220001487800716E22000040EB0025
:108E500080487800906E2200104078008040E80042
:108E6000906E220001487800A16E22000040EB00C5
:108E70008048780005003700A06E2200104078007E
:108E80008040E800A06E220001487800906E220029
:108E900010407800E74F50004E003A00806E2200EC
:108EA000104078000004E0003B003D00806E22008E
:108EB000104078000080FB004200DE008040780017
:108EC000806E220001487800806E220010407800F9
:108ED000FF406000806E220001487800603B810006
:108EE0000000E0002C003200806E2200104078006C
:108EF000FF4F500003003A00304080000020A100E6
:108F000030408800806E220010407800FB4F5000F7
:108F100003003A00304080000020A000304088006C
:108F20003040800001042000010060000000E000EB
:108F300007003200806E220010407800E44F50009D
:108F400003003A00304080000020A100304088003B
:108F5000806E2200104078000081FB0030408000CD
:108F60004200DE00614060008080FB0002004100A2
:108F70008100400020DD2B006141780062479800AD
:108F80006E4090000004E000030032006E4090004C
:108F90007672020000000000816E22000040EB00AB
:108FA00080487800A16E22000040EB0080487800E5
:108FB000916E22000040EB0080487800716E220024
:108FC0000040EB0080487800C16E22000040EB00BA
:108FD000804878005E0090000000E800500798008C
:108FE000DE009000F03F2000808F5000FBFC34003A
:108FF0004F04BE000080FA00000006000C00FA00DA
:10900000889FBE002007980031079800420798000B
:1090100053079800B08081000000E0000A003A0089
:109020006000B800908B8900A18B89006000B800B7
:10903000708B8900818B89006000B800A081890055
:10904000B1818900E10037002E029000BE0290003D
:10905000601823001001BE000400BE00FE070200DD
:10906000000000000002BE00E01723002001900075
:10907000B00190000400BE0096070200000000004E
:109080000004BE004E029000DE0290006018230033
:1090900020019000B00190000400BE00FE07020015
:1090A000000000000002BE00E01723001001BE0017
:1090B0000400BE0096070200000000000001BE0090
:1090C0000800BE00FE07020000000000008FBE0086
:1090D000E01723001000BE00621823000089BE00C4
:1090E000E0172300B00090002000900062182300D9
:1090F00020019800310198002E009000BE009000E1
:10910000E21723000089BE004E009000DE009000B0
:10911000E21723002001980031019800A29929004C
:1091200093E923001E00BE00C409020000000000F5
:109130000000E00001003C0003003700A099290076
:1091400091E92300008FBE00A299290093E92B002A
:109150001E00BE0052090200000000000000E000F6
:109160000100350003003700A099290091E92B0088
:10917000008FBE00908B8100A18B810022852B0087
:10918000E3F7230096070200000000000004BE0081
:109190000200200003E823001E00BE009607020024
:1091A000000000000001BE000800BE000008020030
:1091B00000000000908B8900A18B8900403B81005A
:1091C0000000E00025003200908B8100A18B81001F
:1091D000008FBE00A299290093E923001E00BE0063
:1091E000C4090200000000000000E00008003C008C
:1091F000A299290093E92B001E00BE00520902002B
:10920000000000000000E000010035000B00370006
:10921000C2392500936423001E00BE009607020099
:1092200000000000C2858100D38581000008020093
:1092300000000000C0858900D185890072712B0073
:10924000139D23001E00BE009607020000000000D0
:10925000A0818900B181890033003700908B8100A3
:10926000A18B8100728B8100838B810096070200A5
:10927000000000006011B800C409020000000000F6
:109280000000E00001003C0004003700708B81000A
:10929000818B8100008FBE00020037006000B800A3
:1092A000008FBE00A299290093E923001E00BE0092
:1092B000C4090200000000000000E00008003C00BB
:1092C000A299290093E92B001E00BE00520902005A
:1092D000000000000000E000010035000B00370036
:1092E000C2392500935C23001E00BE0096070200D1
:1092F00000000000C2858100D385810000080200C3
:1093000000000000C0858900D1858900F226210077
:1093100033A823001E00BE009607020000000000D4
:10932000A0818900B1818900C0858100D18581003B
:10933000A2818100B38181000008020000000000CA
:109340002286810033868100C409020000000000EB
:109350000000E00001003C0008003700208681008A
:1093600031868100C0858900D18589006000B80000
:10937000A0818900B181890014003700C085810077
:10938000D1858100A2818100B381810000080200A3
:1093900000000000428681005386810052090200CD
:1093A000000000000000E000010035000700370069
:1093B0004086810051868100C0858900D185890061
:1093C0006000B800A0818900B18189004F04BE000F
:1093D0000080FA00000006000C00FA00889FBE0022
:1093E000200798003107980042079800530798001B
:1093F0002E009000BE0090002E019000BE01900053
:1094000096070200000000000004BE004E0090001D
:10941000DE0090004E019000DE01900096070200F1
:10942000000000000001BE000800BE0000080200AD
:10943000000000005609020000000000008FBE007E
:10944000528B8100638B81001E00BE00C4090200A4
:10945000000000000000E00001003C0013003700A5
:10946000508B8100618B810022852B00E3F7230064
:1094700096070200000000000004BE00A2702D004C
:1094800033BA23001E00BE00960702000000000051
:109490000001BE000800BE0000080200000000003D
:1094A000508B8900618B890012003700508B81003E
:1094B000618B8100E2CE2700F3F7230096070200BC
:1094C000000000000004BE00F226210033B023009B
:1094D0001E00BE0096070200000000000001BE0052
:1094E0000800BE000008020000000000508B890048
:1094F000618B8900508B8100618B8100020020000C
:1095000003F82300C4090200000000000000E0008E
:1095100001003D0024003700800D23001000BE0034
:10952000528B8100638B8100120702000000000053
:10953000820D23000089BE00800D2300B000900042
:1095400020009000528B8100638B81001207020083
:1095500000000000820D23002001980031019800D6
:10956000000D23001000BE00528B8100638B810030
:109570001207020000000000020D23000089BE0057
:10958000000D2300B000900020009000528B81005D
:10959000638B81001207020000000000020D23000F
:1095A00020019800310198004F04BE000080FA00AD
:1095B000000006001A00FA00889FBE008A1F78008B
:1095C00070079800010F9800120F9800230F980061
:1095D0000000EB0060079800208B810010079800C6
:1095E0001E009000EF0F500072003C007E009000C3
:1095F0008E0890007E0190008E0990009607020070
:10960000000000000004BE001E089000AE0890009C
:109610001E099000AE0990009607020000000000AD
:109620000001BE000800BE000008020000000000AB
:10963000200798003107980002002000030824004A
:109640002E009000BE009000C4090200000000003F
:109650000000E00001003C00040037000000200092
:1096600001F8230020079800310798001E0590009C
:109670001E009000C200DD00400623000080400074
:109680001000BE00820C2E00C3F7230096070200D4
:10969000000000000004BE00C2E02C0073C42300E0
:1096A0002E009000BE00900096070200000000000F
:1096B0000001BE000800BE0000080200000000001B
:1096C0000001BE00C250DD004006230000804000C3
:1096D0000288BE00018B81001E009000810F5000A7
:1096E00014003A001000200060079800088B8100E9
:1096F000008B8100C200DD00400623000080400096
:109700001000BE000200200013462400960702004D
:109710000000000010090200000000006101B90013
:10972000C240DD0040FC2200008040000288BE00F4
:10973000130037000000EB00600798001E04900043
:109740001E009000C200DD004006230000804000A3
:109750001000BE0002002800B34324009607020058
:109760000000000010090200000000006101B900C3
:10977000C240DD0040FC2200008040000288BE00A4
:10978000108B810080004000406328000080400072
:10979000900078001E009000808F500002003A0078
:1097A000108B8100008B89001E0090000000E800F3
:1097B000100798000083810011838100E2828100FC
:1097C000F38281000008020000000000008389008D
:1097D000118389000083810011838100F22621001A
:1097E00033D02300C4090200000000000000E000A4
:1097F00001003D0068003700008381001183810073
:10980000F226210033D02300C80902000000000026
:1098100000838900118389001E009000EF0F500023
:1098200005003A00008B8100EF0F500002003A0063
:1098300010002000600798000000EB00100798005F
:10984000902F200051012D004007980051079800EB
:109850000000EB00000F7800170037001E007800B2
:10986000C200DD0040062300008040001001BE0061
:1098700022079800330798004E019000DE01900007
:109880002E009000BE009000C409020000000000FD
:109890000000E00001003C00060037009E01780057
:1098A000138B89002E009000BE00900040079800A6
:1098B000510798001E0FE800F10020009E8F100055
:1098C000E6FF3400603B81000000E0002A00320027
:1098D000508181008000E800008B8100808F500063
:1098E00004003A00308181000000E80030818900E6
:1098F00008003700508181008000E900008B810062
:10990000808F500003003A00308181000000E900A0
:109910003081890022818100420F98008041EB0054
:109920006357980090132000CE089000808F50005D
:109930000200340012C0B30062579800CE099000B4
:109940000300E800208189006E5090000004E000D0
:109950000F00320031818100800C20000088B900A6
:10996000408189000000EB00308189000000EB009D
:1099700020818900060037000000EB00408189004B
:109980000000EB00308189000000EB00208189009D
:10999000008B8100508189009E009000218B8900FE
:1099A0006E0090004F0578004F04BE000080FA0062
:1099B000000006001E00FA00889FBE00300F9800CD
:1099C000410F9800520F9800630F98000040EB0081
:1099D000404798000000EB00000F78006082810093
:1099E000718281008082890091828900A082810039
:1099F000B1828100C0828900D18289003E08900036
:109A0000CE08900060828900718289005E08900013
:109A1000EE089000A0828900B182890080828100D6
:109A20009182810062828100738281009607020028
:109A3000000000000004BE00C0828100D1828100CD
:109A4000A2828100B382810096070200000000001C
:109A50000001BE000800BE00000802000000000077
:109A6000100F9800210F9800808281009182810060
:109A7000A2828100B38281009607020000000000EC
:109A80000004BE006082810071828100C282810078
:109A9000D382810096070200000000000001BE0092
:109AA0000800BE00FE0702000000000070079800DA
:109AB000010F98007E0090008E0890007E019000BB
:109AC0008E09900096070200000000000004BE000E
:109AD0001E089000AE0890001E099000AE0990008C
:109AE00096070200000000000001BE000800BE0052
:109AF00000080200000000005609020000000000FB
:109B000002002000A347240012070200000000000A
:109B10003007980041079800508B8100618B8100CD
:109B20000200200003122400C4090200000000000B
:109B30000000E00001003C0021003700E8808100C7
:109B40007E0090008E0890003E019000CE019000B3
:109B500012070200000000001009020000000000CF
:109B60000001BE00C240DD0040F72200008040003E
:109B70000288BE000800E800E0808900E8808100DB
:109B80001E089000AE0890003E019000CE019000AB
:109B9000120702000000000010090200000000008F
:109BA0000001BE00C240DD0040F7220000804000FE
:109BB0000288BE000800E800E0808900120037003B
:109BC000E3808100C218DD0040F7220000814000E0
:109BD00020002000010020000089BE000300E800F2
:109BE000E0808900E3808100C218DD0040F7220098
:109BF0000081400020002000010020000089BE00FC
:109C00000300E800E0808900E08081006F006000D0
:109C1000E0808900E0198200E20F50000F003A0056
:109C20007E0090008E08900001F0A2000001BE00AE
:109C30001E089000AE089000CC0902000000000051
:109C4000B2FD200093042400000802000000000080
:109C500050079800610798000D0037007E009000C3
:109C60008E0890000001BE001E089000AE08900013
:109C7000CC09020000000000B2FD20009304240083
:109C800000080200000000005007980061079800DB
:109C90005E009000EE00900068000700E01982006E
:109CA0000000E00021003A00808281009182810062
:109CB000628281007382810096070200000000002A
:109CC0000004BE00C0828100D1828100A282810096
:109CD000B382810096070200000000000001BE0070
:109CE0000800BE000008020000000000100F9800ED
:109CF000210F98001E0A9000AE0A90000000EB00B1
:109D0000100798006011B8000400BE00C4090200EA
:109D1000000000000000E00001003C0007003700E8
:109D20001000200010079800040037005E0090002B
:109D3000EE00900094020700100798001E009000AB
:109D40000000E00016003A00703B81000000E000D7
:109D500013003200907B81000000E0001F00320001
:109D6000907B81004280DE00907B8900917B8100A6
:109D7000F07F200000806000907B8900917B810053
:109D80002077220061417800424798000000EB00F4
:109D9000907B890010002000000F78000F00370032
:109DA000907B810000004000907B8900917B8100C6
:109DB0001E00900000807000907B89001E009000C3
:109DC0000000E00003003A0010002000703B890012
:109DD000020037000000EB00703B89001E00E0002D
:109DE000130032004E4090000004E00010003200EA
:109DF000603B81000000E0000D0032004E4090000A
:109E0000F74F400002003A0000C6B30040479800F8
:109E1000E0198200E70F5000030032004E4090002E
:109E200076720200000000000000EB00000F7800D6
:109E30004F04BE000080FA00000006001000FA0087
:109E4000889FBE004007980051079800F08081006D
:109E5000CF80DE00BA08020000000000008FBE00C4
:109E6000E01982000000E000190032000040EB0021
:109E7000704F9800B2FD200093F423004E00900034
:109E8000DE009000C4090200000000000000E000B5
:109E900001003D000200370011C0B300714F98006F
:109EA0007E4890000004A2000004E00008003A0090
:109EB00042BE2C00630124004E009000DE009000A2
:109EC00052090200000000000000E0001C00340005
:109ED000E01982000000E000BE003A000040EB0004
:109EE000604F98006011B8004E009000DE009000B6
:109EF000C4090200000000000000E00001003D0075
:109F00000200370011C0B300614F98006E48900006
:109F10000004A2000004E000AE003A00B2FD200000
:109F2000930424004E009000DE00900052090200CD
:109F3000000000000000E00001003400A500370030
:109F4000E0198200E20F500009003A004E01900033
:109F5000DE019000B0FD200091FC2300FE0702000E
:109F60000000000020079800310798000800370023
:109F7000B2FD200093FC23004E009000DE00900014
:109F8000FE0702000000000020079800310798003B
:109F90002E009000BE009000B08B8900C18B89001C
:109FA000E01982000000E0000A0032002E0090005C
:109FB000BE00900001F0A10002002000C338240080
:109FC0009607020000000000200798003107980063
:109FD000090037002E009000BE00900001F0A100A3
:109FE00002002000633124009607020000000000F8
:109FF0002007980031079800428281005382810037
:10A000002E009000BE0090005209020000000000E7
:10A010000000E000010035001E0037001E01BE00F8
:10A020000000200001F82B001207020000000000D1
:10A030000200200003F823000008020000000000D6
:10A0400042828100538281009607020000000000D6
:10A050000004BE001E01BE000000200001F8230025
:10A0600012070200000000002E019000BE019000C7
:10A0700096070200000000000001BE000800BE00BC
:10A08000000802000000000040828900518289001F
:10A09000260037000200200003002C001E00BE0036
:10A0A00096070200000000000001BE000000200032
:10A0B00001F8230012070200000000000200200047
:10A0C00003F8230000080200000000004282810023
:10A0D0005382810096070200000000000004BE00C9
:10A0E0001E00BE000001BE000008020000000000CB
:10A0F0000001BE000000200001F82300120702004A
:10A10000000000002E019000BE01900096070200A2
:10A11000000000000001BE000800BE0000080200B0
:10A120000000000040828900518289006081810026
:10A13000F40F50000500340000002000811C2400B2
:10A1400040828900518289000300370060818100CC
:10A150000000E800608189000000EB007081890048
:10A16000B08B8100C18B81006011B800C40902006E
:10A17000000000000000E00001003D000600370084
:10A18000308B81000000E800308B89000000EB007C
:10A19000408B890005003700408B81000000E800FB
:10A1A000408B89000000EB00308B8900308B8100F0
:10A1B000E40F5000E7003C00408B8100E40F5000AA
:10A1C000E4003C006000B800B08B8900C18B8900BE
:10A1D000E0003700E01982000000E00019003200C2
:10A1E0008040EB00514F9800223D2500B30724002A
:10A1F0004E009000DE009000C40902000000000044
:10A200000000E00001003D000200370010C0B30074
:10A21000504F98005E4890000004A2000004E00047
:10A2200008003A0002DE2E00F30A24004E009000DF
:10A23000DE00900052090200000000000000E00073
:10A240001D003400E01982000000E000C1003A0067
:10A250008040EB00414F9800B2FD200093042400A1
:10A260004E009000DE009000C409020000000000D3
:10A270000000E00001003D000200370010C0B30004
:10A28000404F98004E4890000004A2000004E000F7
:10A29000B0003A00B2FD2000930C24004E00900064
:10A2A000DE00900052090200000000000000E00003
:10A2B00001003400A7003700E0198200E20F5000CF
:10A2C00009003A004E019000DE01900040BE2C00D3
:10A2D00061092400FE07020000000000200798002A
:10A2E000310798000800370042BE2C0063092400A3
:10A2F0004E009000DE009000FE070200000000000B
:10A3000020079800310798002E009000BE009000B2
:10A31000B08B8900C18B8900E01982000000E00049
:10A320000A0032002E009000BE00900001F0A10053
:10A3300002002000C338240096070200000000003D
:10A340002007980031079800090037002E00900080
:10A35000BE00900001F0A100020020006331240043
:10A3600096070200000000002007980031079800BF
:10A3700042828100538281002E009000BE00900036
:10A3800052090200000000000000E000010035005A
:10A390001E0037001E01BE000000200001F82B0047
:10A3A00012070200000000000200200003F8230052
:10A3B00000080200000000004282810053828100F8
:10A3C00096070200000000000004BE001E01BE004F
:10A3D0000000200001F82300120702000000000026
:10A3E0002E019000BE0190009607020000000000C0
:10A3F0000001BE000800BE000008020000000000CE
:10A400004082890051828900260037000200200026
:10A4100003002C001E00BE00960702000000000092
:10A420000001BE000000200001F823001207020016
:10A43000000000000200200003F8230000080200D2
:10A4400000000000428281005382810096070200D2
:10A45000000000000004BE001E00BE000001BE009F
:10A4600000080200000000000001BE000000200003
:10A4700001F8230012070200000000002E019000E6
:10A48000BE01900096070200000000000001BE001F
:10A490000800BE00000802000000000040828900A1
:10A4A0005182890070818100F40F5000080034004F
:10A4B000E01982000000E00008003A0000002000DF
:10A4C000812C2400408289005182890003003700DA
:10A4D000708181000000E800708189000000EB00BD
:10A4E00060818900B08B8100C18B81006011B80050
:10A4F000C4090200000000000000E00001003D006F
:10A5000006003700308B81000000E800308B8900A6
:10A510000000EB00408B890005003700408B810074
:10A520000000E800408B89000000EB00308B8900C0
:10A53000308B8100E40F500006003C00408B81000E
:10A54000E40F500003003C006000B800B08B8900AD
:10A55000C18B890060818100E20F5000030034004C
:10A5600010002000503B8900020037000000EB0083
:10A57000503B8900508B8100618B810002002000DC
:10A5800003122400C4090200000000000000E000E3
:10A5900001003C001E003700E01982000000E000CE
:10A5A00009003200408281005182810010090200BE
:10A5B00000000000800078004006200001005000EC
:10A5C00000818900080037004082810051828100AB
:10A5D0001009020000000000800078004006200002
:10A5E00001005000008189000181810010818100FB
:10A5F000808F50000300350010002000603B890070
:10A60000070037000000EB00603B890004003700C2
:10A610000000EB00008189000000EB00603B890036
:10A62000E01982000000E0001B003200B08B8100C6
:10A63000C18B8100A299290093F12300C409020073
:10A64000000000000000E00001003C0004003700B2
:10A65000A099290091F12300B08B8900C18B89005A
:10A66000B08B8100C18B8100A299290093F12B004E
:10A6700052090200000000000000E0000100350067
:10A680001F003700A099290091F12B00B08B8900A1
:10A69000C18B89001A003700B08B8100C18B81000B
:10A6A0000200200003F82300C4090200000000009B
:10A6B0000000E00001003C00040037000000200022
:10A6C00001F82300B08B8900C18B8900B08B810019
:10A6D000C18B81000200200003F82B005209020008
:10A6E000000000000000E000010035000400370019
:10A6F0000000200001F82B00B08B8900C18B89007D
:10A7000062868100738681000000200001F82B0022
:10A7100012070200000000000200200003F82300DE
:10A720000008020000000000728B8100838B810012
:10A7300096070200000000000004BE00628681004F
:10A740007386810000002000010A24001207020025
:10A7500000000000B28B8100C38B810096070200CD
:10A76000000000000001BE000800BE00000802005A
:10A7700000000000708B8900818B89004F04BE00AF
:10A780000080FA0000000600D600FA00889FBE0094
:10A790008A1F780060A7980071A7980020DC2B0022
:10A7A00001CF27004007980051079800B2FD200014
:10A7B000930424006EA09000FEA09000C409020043
:10A7C000000000000000E00001003D000300370031
:10A7D00040622800000F7800020037004061280026
:10A7E000000F78000000EB001007980049003700C8
:10A7F0001E0590001E00900022002000110009009C
:10A800000200D800C300DD00000E230000804000DD
:10A810001000BE000004BE009E009000A08C280026
:10A82000614078000000FB004200DD001E00400097
:10A830001001BE006EA09000FEA09000FE07020076
:10A84000000000000001BE0003F0A1000800BE00EF
:10A8500000080200000000000001BE00EC004700FC
:10A860004250DD00010040000288BE001E00900042
:10A87000EC0047004200DD00010040001000BE0077
:10A880004E019000DE01900052090200000000001D
:10A890000000E00001003500070037001E009000B6
:10A8A000EC0047004200DD00010040001001BE0046
:10A8B00042079800530798009E0190001E009000E8
:10A8C00022002000110009000200D8004300DD0032
:10A8D000E4004000000E2300008040001000BE0095
:10A8E0000000400081804800800078001E00900039
:10A8F0006100600000814000C10820008E8040009F
:10A900000380410002B078001E0090000000E800C3
:10A91000100798001E009000FF0F5000B4FF340095
:10A920000000EB00100798004D0037001E0090005B
:10A93000EC0047004200DD00010040001002BE00B4
:10A940001E00900070004000EC0047004200DD0057
:10A95000010040001001BE000400BE0052090200C8
:10A96000000000000000E000010035001C0037007E
:10A970001E0490001E009000EC0047004200DD0025
:10A98000010040001000BE004E019000DE0190006A
:10A99000FE070200000000000001BE00C340DD0011
:10A9A000000E2300008040000288BE001E029000BE
:10A9B0001E009000C10820008E8040000000400072
:10A9C000608078006101B9004320DD00E4004000B0
:10A9D000000E2300008040000288BE001D003700EA
:10A9E0001E0490001E00900070004000EC00470024
:10A9F0004200DD00010040001000BE004E0190004A
:10AA0000DE019000FE070200000000000001BE0011
:10AA1000C340DD00000E2300008040000288BE001D
:10AA20001E0290001E00900070004000C10820002F
:10AA30008E80400000004000608078006101B90015
:10AA40004320DD00E4004000000E230000804000B1
:10AA50000288BE001E0090000000E8001007980069
:10AA60001E009000EF0F5000B0FF34006000B800EF
:10AA700020079800310798000000EB0010079800AD
:10AA8000290037001E0090004300DD00E400400074
:10AA9000000E2300008040001000BE0002002000D5
:10AAA0000301200000027800810278000200780093
:10AAB0008300780000016200018062006102B8003A
:10AAC00014AF980025AF98001EA89000AEA8900083
:10AAD000C000DD000000200010AF980021AF9800FA
:10AAE0001EA89000AEA890006112B80014AF9800A4
:10AAF00025AF98001EA99000AEA99000020070003A
:10AB0000838070002E019000BE0190000200400082
:10AB10008380480020079800310798001E009000AD
:10AB20000000E800100798001E009000EF0F500092
:10AB3000D4FF34002E019000BE01900000002000E0
:10AB400001082000800F5100818F590007003A0052
:10AB5000FA170200000000008000780000002100C9
:10AB60008080600001AF98000B0037008001EB008F
:10AB700003AF98002E019000BE019000000020005D
:10AB800001082000800F5100818F5900020034001D
:10AB90001400200004AF98000EA890004F05780024
:10ABA0004F04BE000080FA00000006000800FA0012
:10ABB000881F78002000200080007800A04A2B0029
:10ABC00000017800810178000180230090002000BE
:10ABD00010170200000000000180230090002000F8
:10ABE000881702000000000002802300018023007B
:10ABF00000202000BE170200000000000000EB0053
:10AC0000000F7800150037009E0178001E007800C4
:10AC10008000400060262200008040001000780084
:10AC20006300B90000017800001020001E005000F1
:10AC3000C200DD000080230000804000100078008A
:10AC4000000041004201DE008380410060262200B6
:10AC500000804000020878001E0FE800F00F20007E
:10AC60009E0F1000E8FF34000000EB00000F78009A
:10AC70002D0037001E0078003007980001022000E8
:10AC80001E804000800040006026220000804000BE
:10AC9000100478006140B900BA080200000000000A
:10ACA00010079800210798000800E00008003D0008
:10ACB00002002000037824001E009000AE009000E7
:10ACC000000802000000000010079800210798000B
:10ACD0001E009000AE0090000200200003F8230048
:10ACE0000008020000000000060A02000000000048
:10ACF00002002000030C2400960702000000000060
:10AD00000E0A02000000000000017800BE01900061
:10AD1000BE01900083804100604622000080400018
:10AD2000020878001E0FE800F00720009E0F1000B8
:10AD3000D0FF34000000EB0030238900CC76020005
:10AD400000000000E0198200E60F500004003A0005
:10AD50005076020000000000687B02000000000046
:10AD60000000EB00000F78000E0037001E00780096
:10AD7000C200DD0000802300808040000000EB0066
:10AD8000800878001E0078004200DD008080E80026
:10AD900000802300808040000000EB0080087800E5
:10ADA0001E0FE800F01F20009E0F1000EFFF340080
:10ADB0004F0478000080FA00000006000200FA004C
:10ADC000000F78001E007800CF80DE00BA08020075
:10ADD00000000000404C8800514C88000080FA00C0
:10ADE000000006000200FA00000F78001E00780044
:10ADF00070198A000080FA00000006000200FA00C4
:10AE0000000F78001E00780060198A000080FA00A8
:10AE1000000006000000FA00D01982000080FA004D
:10AE2000000006002200FA00000F780011079800C9
:10AE30001E007800001798008E109000E38F5000DD
:10AE4000280032000E119000E30F51000A003C0070
:10AE50008E119000E18F5100180032000E1090000A
:10AE6000E10F50001A003C008E1090000100E0003D
:10AE70000E003200930037000E119000E50F5100D4
:10AE8000420032008E119000E58F51002B003500FA
:10AE90000E109000E60F5000520032008E1090000D
:10AEA000E78F50006B003200860037006011B80059
:10AEB000420F9800530F98008300370000002000D5
:10AEC00001F82300400F9800510F98007E003700D2
:10AED0000200200003F82B00420F9800530F980047
:10AEE000790037009E009000F0072000808F50000E
:10AEF0000A003400011020001E0090000080500065
:10AF0000C200DD00A0172C00008040001001BE0030
:10AF1000220F9800330F9800030037006000B8003C
:10AF2000200F9800310F98002E099000BE09900064
:10AF3000420F9800530F9800630037009E00900066
:10AF4000F0072000808F500008003C001E00900099
:10AF5000C200DD00A0172C00008040001001BE00E0
:10AF6000020F9800130F9800030037006000B8002C
:10AF7000000F9800110F98000E0990009E09900094
:10AF8000420F9800530F98004F0037009E0090002A
:10AF9000F0072000808F50000A003C001E00900047
:10AFA000C200DD00A0172C00008040001000BE0091
:10AFB0000001BE0003F0A20062079800730798002A
:10AFC000030037006000B800600798007107980020
:10AFD0006E019000FE019000420F9800530F980000
:10AFE000390037009E009000F0072000808F50004D
:10AFF00008003C001E009000C200DD00A0172C00DD
:10B00000008040001001BE004207980053079800DE
:10B010000B003700011020001E009000008050003F
:10B02000C200DD00A0172C00008040001000BE0010
:10B030000001BE0003F0A2004207980053079800E9
:10B040004E009000DE009000400F9800510F9800D5
:10B050001D0037009E009000F0072000808F5000F8
:10B060000A003C001E009000C200DD00A0172C006A
:10B07000008040001000BE000001BE0003F0A200EE
:10B0800022079800330798000900370001102000BC
:10B090001E00900000805000C200DD00A0172C00B0
:10B0A000008040001001BE0022079800330798007E
:10B0B0002E009000BE009000400F9800510F9800A5
:10B0C00001003700040037004E099000DE099000AF
:10B0D000620F9800730F98006E089000FE089000B1
:10B0E0000080FA00000006000000FA000000EB00FB
:10B0F00060198A000000EB0070198A000000EB0064
:10B1000050198A000000EB0090198A000000EB0043
:10B11000A0198A000000EB0080198A000000EB00F3
:10B1200030238A0000002800B14B2400404C8800E6
:10B13000514C880040912000104078000000FB0036
:10B1400020268A000080FA00000006000400FA00B1
:10B1500020002000101A8A0000F4210020228A001A
:10B160000000EB0030228A000000EB00B0198A00DA
:10B170000000EB00C0198A000000200001F8230045
:10B18000D0268A00E1268A0020228200CF80DE00BD
:10B19000BA08020000000000D2268200E3268200E6
:10B1A0009607020000000000E0858900F185890013
:10B1B000404C8000514C8000B2FD2000930C2400D4
:10B1C0009607020000000000E2858100F3858100FF
:10B1D000120702000000000070278A0081278A0001
:10B1E000E2858100F38581000000200001F8230042
:10B1F000120702000000000030278A0041278A0061
:10B20000E14C240040C0B3008048780010002000CA
:10B2100050268A000000EB00F0198A000000EB00C5
:10B22000001A8A00E01982005E0007000000EB00AF
:10B23000100798000A0037001E009000C200DD00D1
:10B2400040F7220000814000100020000100200093
:10B250000089BE001E0090000000E8001007980062
:10B260001E009000EF0F5000F3FF34000000EB00D1
:10B2700070228A00803E200080228A00803E2000CA
:10B2800090228A000000EB00A0228A000000EB0060
:10B29000B0228A0080C12F00C0228A0080C12F0006
:10B2A000D0228A000000EB00E0228A000000EB00C0
:10B2B000F0228A000000EB0000238A000000EB006F
:10B2C00010238A00803E200020238A000000EB002B
:10B2D000100798000B0037001E01900081462400E3
:10B2E00010C0B30000F178001E01900091482400C6
:10B2F00030C0B30000F178001E0090000000E800AC
:10B30000100798001E009000FF0F5000F2FF34005D
:10B310001E019000814624000040EB0000F17800FF
:10B320001E019000914824000040EB0000F17800DD
:10B330000000EB0010079800070037001E01900086
:10B34000A14A2400F0C1B30000F178001E00900073
:10B350000000E800100798001E009000E10F500068
:10B36000F6FF34001E019000A14A24000040EB00CB
:10B3700000F178000000EB0030268A000000EB00AE
:10B3800040268A004000200060268A000000EB0072
:10B3900090268A000000EB00A0268A000080FA00B8
:10B3A000000006000400FA00000F78001E0078007C
:10B3B000E0198A00E01982004300DE0061006000AD
:10B3C0000004E0000800320000002000A127240053
:10B3D000B0268A00C1268A00101A820000004000B0
:10B3E00040228A0016003700E0198200E70F500063
:10B3F0000D003A00A09A2100104078000000FB00E8
:10B40000CF80DE00BA08020000000000A2992900E7
:10B4100093F923001207020000000000B0268A0002
:10B42000C1268A000600370000002000A11F24006A
:10B43000B0268A00C1268A00101A820040228A00A3
:10B44000E0198200E60F500004003A00D0CC2C0036
:10B4500051232400B0268A00C1268A00B226820029
:10B46000C32682000000200001F82300120702001A
:10B470000000000050278A0061278A00E01982003E
:10B4800067006000100798001E009000E40F500055
:10B490001E0032001E009000E40F500007003C0028
:10B4A0001E0090000000E000230035001E00900008
:10B4B000E20F50000B003400110037001E00900016
:10B4C000E60F5000070032001E009000E60F50000B
:10B4D000130035001E009000E70F500013003200EB
:10B4E0001500370030002000D0198A00C08D2B00D5
:10B4F00081D8230090338900A133890012003700DE
:10B5000060002000D0198A000F0037006000200082
:10B51000D0198A001000200060198A000A00370044
:10B5200030002000D0198A000700370010002000EA
:10B53000D0198A000400370030002000D0198A009A
:10B540000000EB00E0198A000080FA00000006000D
:10B550002400FA00F0282C0051CF2300F0268A00A6
:10B5600001278A00702782008127820032982F00ED
:10B570002362240096070200000000001009020068
:10B58000000000000001BE000019820011198200B5
:10B59000020040008380480000198A0011198A00C7
:10B5A00000198200111982004C09DD004400DE0000
:10B5B00000007100C488DE0080007800F0FF2000E9
:10B5C000008060007632020000000000CF80DE00C4
:10B5D000BA08020000000000600798007107980098
:10B5E0000019820011198200CC09DD004400DE0040
:10B5F00000807100C488DE008000780000402000D8
:10B6000080804000F0FF2000008060007632020061
:10B6100000000000CF80DE00BA0802000000000039
:10B620004007980051079800E0198200E60F50008B
:10B6300009003A000000200001F82300200F9800C4
:10B64000310F98000000200001F82300000F98003F
:10B65000110F980060003700E0198200E70F5000DA
:10B6600053003A0060322400104078000000FB00D4
:10B67000101798001E109000E40F500010003200C8
:10B680009E109000E58F5000260032001E119000A1
:10B690000200E000010032003C00370090278200E9
:10B6A000A1278200200F9800310F9800B227820056
:10B6B000C3278200020F9800130F98003300370051
:10B6C0003122820000022000808F500008003C00E0
:10B6D00030228200C200DD00A03B2C000080400030
:10B6E0001001BE00720F9800031798000400370085
:10B6F000F021860001228600700F98000117980043
:10B700007E0990008E119000220F9800330F980050
:10B710002E089000BE089000000F9800110F9800AE
:10B720001A0037003122820000022000808F500072
:10B730000A003C003122820010022000010050006B
:10B74000C200DD00A03B2C00008040001001BE00C4
:10B75000520F9800630F980004003700D01D860038
:10B76000E11D8600500F9800610F98005E0990005F
:10B77000EE099000220F9800330F98002E089000D9
:10B78000BE089000000F9800110F98002E0990003D
:10B79000BE09900092278A00A3278A000E08900015
:10B7A0009E089000B0278A00C1278A000A0037004F
:10B7B00031228200302682009AFD0700200F980077
:10B7C000310F9800312282004026820095FD07004B
:10B7D000000F9800110F9800F026820001278200C8
:10B7E0002E099000BE09900096070200000000009C
:10B7F0006E019000FE01900096070200000000001C
:10B80000100902000000000030079800F0268200B6
:10B81000012782000E0990009E0990009607020001
:10B82000000000004E019000DE019000960702002B
:10B83000000000001009020000000000200798002E
:10B84000BE0090002E00900080804000F0FF20009D
:10B850000080600010079800302282000000E8009D
:10B8600030228A00009781001197810032278200E0
:10B8700043278200000802000000000000978900B2
:10B88000119789000097810011978100522782004B
:10B8900063278200C4090200000000000000E000ED
:10B8A00001003D009700370000978100119781004B
:10B8B0005227820063278200FE070200000000007A
:10B8C00000978900119789000000EB0030228A0060
:10B8D000E019820067006000400F9800CE089000D9
:10B8E000E48F50000D003C004E099000E30F510022
:10B8F0004A003D00CE099000E18F5100290032003E
:10B900004E089000E10F50002B003C00CE08900044
:10B910000100E0001E003200440037004E09900094
:10B92000E60F510038003200CE099000E68F51003A
:10B93000040035004E089000E70F5000010032006F
:10B940003A0037006032240090407800A04F240075
:10B9500001487800490107008040780060322400E7
:10B9600001487800A04F240010407800E44F5000B8
:10B970002E003A006032240010407800E54F50005D
:10B980002A0032001002200030228A0027003700EF
:10B9900009020700804078006032240001487800E6
:10B9A000220037004C0207008040780060322400FB
:10B9B000014878001D0037004702070080407800EA
:10B9C0006032240001487800603224001040780082
:10B9D000E14F500004003A006132240030C0B3004F
:10B9E0008048780011003700603224001040780051
:10B9F000E34F50000D003A006132240010C0B30044
:10BA00008048780009003700450007008040780032
:10BA100060322400014878000400370072020700F9
:10BA2000804078006032240001487800E0198200EC
:10BA3000E60F5000330032006032240010407800DE
:10BA40000000FB00622682006500B9000200400091
:10BA500080004000E0372C0000804000100F78008C
:10BA6000007020001E0060004880DE0030268A0042
:10BA7000000720001E0060004480DE0040268A008F
:10BA80009E0078006780600060268A00241982008A
:10BA900060268200C200DD00E044240000804000F7
:10BAA000100078006101B900C220DD0040F72200DB
:10BAB000008040000288BE000400E80020198A00CF
:10BAC00024198200602682004200DD008080E800A8
:10BAD000E044240000804000100078006101B900BB
:10BAE000C220DD0040F72200008040000288BE0036
:10BAF0000400E80020198A00201982006F0060000D
:10BB000020198A001E0090000180200001004000E2
:10BB1000BE8B0200000000000080FA00000006005A
:10BB20000400FA00E04C240090407800314798006F
:10BB300050912000104078000004E00040003200E6
:10BB400030408000680060000000E00018003A000B
:10BB500080322400104078000080FB00610060000B
:10BB60000004E00009003200604C8000714C80004D
:10BB700092338100A333810000080200000000001E
:10BB800070278A0081278A0020003700604C8000DF
:10BB9000714C800092338100A3338100FE070200C4
:10BBA0000000000070278A0081278A0017003700F4
:10BBB00080322400104078000080FB0061006000AB
:10BBC0000004E00009003200604C8000714C8000ED
:10BBD00092338100A3338100FE07020000000000C1
:10BBE00070278A0081278A0008003700604C800097
:10BBF000714C800092338100A33381000008020061
:10BC00000000000070278A0081278A00803224000B
:10BC1000104078000080FB000000D10080407800D8
:10BC200080322400014878005091200010407800B4
:10BC30008040E900509120000148780088003700DA
:10BC40005191200080C0B3008048780031408000CE
:10BC500000082000008060000000E00007003200C3
:10BC60007032240010407800204798003040800057
:10BC70000070A1003040880002003700EA01070090
:10BC8000204798002E4090000000FB00760602003E
:10BC9000000000000000E000050032002E4090008F
:10BCA0000000FB008A060200000000002047980008
:10BCB0002E409000E14F50000E003200AE40900048
:10BCC00000C4B30080CF50000A003C00AE4090009A
:10BCD00000C2B30080CF5000060032002E4090001A
:10BCE000ED4F5000030032002E409000EA4F50000C
:10BCF00004003A00304080000020A100304088005D
:10BD000003003700304080000020A0003040880051
:10BD1000304080004200DE00614060008080FB0017
:10BD2000F0252200104078000080FB00808F50003A
:10BD300010003200AE4090007032240001487800BC
:10BD4000304080000070A00030408800304080000B
:10BD5000640060000000E00003003200B001200039
:10BD6000000F780022003700F0012000000F78005B
:10BD70001F0037000000EB00000F78000F003700B5
:10BD80001E017800304080004200DE00614060000B
:10BD90008080FB00020041008100400020DD2B007C
:10BDA000614078008080FB002E4090000000FB0086
:10BDB000808F5000040032001E0FE800F0012000C8
:10BDC0009E0F1000EEFF34001E00E0000300320062
:10BDD000F10120009E8F100005003400F0012000CA
:10BDE000000F7800F12522000040EB008048780029
:10BDF0001E007800804078008032240001487800DE
:10BE000080322400104078000040400080407800DC
:10BE1000803224000148780080322400904078006D
:10BE2000E0CFB30080C06000803224000148780079
:10BE3000803224009040780000CCB30080C07000B5
:10BE40008032240001487800304080004200DE004B
:10BE50006140600080407800F025220001487800B1
:10BE6000E04C2400BE409000014878003E40900025
:10BE70000000FB000080FA00000006001000FA003D
:10BE8000E0198200E50F500003003A0040228200D2
:10BE90007007980002003700110020007107980019
:10BEA0007E009000000F7800E04C24009040780065
:10BEB00031479800902682000000E00048003A00D8
:10BEC000F01982000000E00045003A00560107002A
:10BED00020479800AE40900000C6B30080CF5000CD
:10BEE00007003400AE409000A0C7B30080CF5000E0
:10BEF00003003C001000200060079800020037009B
:10BF00008000EB00610798006E009000F0278A0027
:10BF10002E4090000000FB0050079800DE009000CB
:10BF2000E28F50000A0032005E009000E30F5000E4
:10BF3000010032000C00370050C0B30030479800B9
:10BF40003E4090000000FB0040079800970037003B
:10BF500040C0B300304798003E4090000000FB0016
:10BF600040079800910037002E4090000000FB0031
:10BF70008A06020000000000204798002E40900032
:10BF8000FF4F50000E003400AE409000A0C5B3003B
:10BF900080CF50000A003C002E4090008000FB0043
:10BFA00000FE2F0000804000800040004065280017
:10BFB000008040001000780090268A0006003700BC
:10BFC000AE40900000C6B30080CF500002003A009F
:10BFD0000097250090268A000000EB00F0198A00E7
:10BFE000F1198200310798003E009000E10F5000E7
:10BFF0003F003200BE009000E28F5000520032003D
:10C000003E0090000000E0000100320056003700C2
:10C010009026820001002C0001006000200798009B
:10C0200000002800AE009000808F50001000320009
:10C0300000002C00AE009000808F500014003200F1
:10C0400000002400AE009000808F500001003200FC
:10C050001800370010002000F0198A001E00780038
:10C06000001A8A0050C0B300304798001300370010
:10C0700010002000F0198A001E0078006300B9004B
:10C08000001A8A0050C0B300304798000B003700F8
:10C0900020002000F0198A001E00780000004000F7
:10C0A0000000E900001A8A0040C0B3003047980041
:10C0B0000200370040C0B30030479800902682004D
:10C0C0004200DD0090268A009126820000002C00AC
:10C0D000808F500024003A00F02782000000E0002A
:10C0E000210032000000EB0090268A001E0037007D
:10C0F000001A82000000E900001A8A00001A82007B
:10C100000000E0000D003C001E00E900001A8A005B
:10C11000001A82000000E00003003400200020002C
:10C12000F0198A00020037000000EB00F0198A00C5
:10C1300040C0B300304798000B0037000040EB00D0
:10C140003047980008003700001A82000000E9001C
:10C15000001A8A00001A82000000E00002003C0081
:10C160000000EB00F0198A003E409000E54F5000BF
:10C1700003003A0010002000B0CD88000500370011
:10C180003E4090000004E000020032000000EB009E
:10C19000B0CD8800E04C2400BE40900001487800FB
:10C1A0003E4090000000FB00400798004E009000C9
:10C1B0000080FA00000006000400FA00E04C2400B1
:10C1C0009040780011479800902682000000E0001F
:10C1D0002A003A00502682000000E00005003200EC
:10C1E00020C0B300104798000000EB0050268A00E2
:10C1F000320037008C000700004F78001E00FB0063
:10C20000100798009E009000E28F50000D00320051
:10C210001E009000E30F5000040032009E009000CA
:10C22000E18F5000040032000900370050C0B30015
:10C23000104798002100370020C0B3001047980035
:10C240001E00370040C0B300104798001B003700A5
:10C250009E00FB00F00F2000008060008000400086
:10C26000A06C2800008040001000780090268A0012
:10C2700020C0B300104798001000370090268200BD
:10C280000000E00003003D000040EB001047980074
:10C290000200370020C0B3001047980090268200AB
:10C2A0000000400090268A00902682000000E000F6
:10C2B00002003A001000200050268A00E04C2400C2
:10C2C0009E409000014878001E4090000000FB0056
:10C2D0000080FA00000006000400FA0090268200A8
:10C2E000FF006000A08C2800614078001047980093
:10C2F000902682000000400090268A00A02682003E
:10C300000000E00026003A00502682000000E00015
:10C31000030032000000EB0050268A002E00370098
:10C3200041000700004F78001E00FB001007980036
:10C330001E009000E20F50000D0032001E00900021
:10C34000E30F5000040032001E009000E10F500087
:10C35000040032000900370050C0B30010479800B5
:10C360001D0037000000EB00A0268A001A003700ED
:10C3700040C0B30010479800170037009E00FB0034
:10C38000F00F20000080600080004000A06C2800BA
:10C390000080400010007800A0268A000E003700C0
:10C3A000A02682000000E00003003D0090268200ED
:10C3B0000000A00090268A00A02682000000400015
:10C3C000A0268A00A02682000000E00002003A00B9
:10C3D0001000200050268A001E4090000000FB0044
:10C3E0000080FA00000006000200FA000E000700BC
:10C3F000004F78001E00FB00E30F500001003200E8
:10C400000300370050C0B300104798000200370007
:10C4100040C0B300104798001E4090000000FB0091
:10C420000080FA00000006000C00FA00881F780067
:10C43000D019820050079800DE009000E38F500072
:10C44000770032005E019000E30F51000A003C00CB
:10C450005E009000E10F5000AB003200DE00900063
:10C46000E18F50000C013C005E0190000200E000F2
:10C470000B0032000A0137005E009000E50F50000B
:10C4800085003200DE009000E58F50002700350067
:10C490005E019000E60F51000600320000013700F7
:10C4A00020C0B300104798000000EB0070198A000C
:10C4B000FB00370030C0B3001047980070198200AD
:10C4C0000000E000F6003200601982000000E00089
:10C4D0000D00320050002000D0198A00E0198200BF
:10C4E00050228A0050002000E0198A000000EB0072
:10C4F00060198A000000EB0030238A0020C0B300DE
:10C5000010479800E60037000000EB00D0198A00C1
:10C510000000EB0030238A0020C0B30010479800D1
:10C520000000EB0070198A00DD003700E01982007E
:10C53000E60F50003200320030238200400798009E
:10C5400090482400CE009000E14078001147980008
:10C550000041EB00624798001E4090000004E0009C
:10C5600002003A0010C0B30060479800CE0090006F
:10C570000100E80030238A006E4190000204E000D0
:10C5800003003A00501982000000E000C4003200AD
:10C590000000EB0050198A00601982000000E000E2
:10C5A0000D00320050002000D0198A00E0198200EE
:10C5B00050228A0050002000E0198A000000EB00A1
:10C5C00060198A000000EB0030238A0020C0B3000D
:10C5D00010479800B20037000000EB00D0198A0025
:10C5E0000000EB0030238A0020C0B3001047980001
:10C5F0000000EB0070198A00E222A900A8003700B1
:10C60000F0C1B300104798000000EB00D0198A0079
:10C610000000EB0030238A00E222A900A0003700CE
:10C62000E0198200E60F500008003A003023820033
:10C63000A14A240060C17800124798000000E80079
:10C6400030238A00000000000600370030238200FB
:10C650008146240060C17800124798000000E8007D
:10C6600030238A001E4090000004E0008C003A0055
:10C6700010002000D0198A000000EB0030238A004F
:10C68000E0198200E60F50008500320010C0B300B0
:10C6900010479800820037003023820000047800A1
:10C6A000F04A24002C18020000000000800F540003
:10C6B0000C00390050228200E0198A000000EB00D3
:10C6C000D0198A000000EB0030238A0020C0B3009C
:10C6D000104798000000EB0070198A00E222A900C0
:10C6E0006F00370050002000E0198A0031238200DB
:10C6F000F04A240061417800124798000100E800E8
:10C7000030238A00660037005E0207001047980059
:10C71000000000001E4090000000FB002007980071
:10C720002E009000EE0F500014003200AE0090007A
:10C73000EE8F500007003C002E019000E10F5100E9
:10C74000310032002E009000E20F50002100320034
:10C7500035003700AE009000F08F50001800320016
:10C760002E019000F00F5100100035002E009000B7
:10C77000F10F5000070032002B003700100020009E
:10C780000A920200000000000040EB0010479800F1
:10C79000430037008000EB001E4090004600070079
:10C7A0000040EB00104798003D003700289602003B
:10C7B000000000000040EB001047980038003700F0
:10C7C0005A960200000000000040EB00104798005D
:10C7D00033003700C1198200B0198200808F5000E9
:10C7E00006003A00C04C800000A0A000C04C8800A9
:10C7F0000040EB00104798002900370000C2B3004A
:10C800001047980026003700701982000000E000F1
:10C810002300320040002000D0198A000000EB0005
:10C8200030238A001E003700009920009E409000AF
:10C83000014878000091200010407800E74F500038
:10C8400005003A00E0CC80007E920200000000006B
:10C850000000E000030032001200200012079800E0
:10C86000020037000000EB00100798002E409000F7
:10C8700061406000C14C80000080FB0061006000EE
:10C880004D01DD00F0FF2D0080806000828070008F
:10C89000C14C88000200370010C0B3001047980058
:10C8A000000000001E4090000000FB004F047800D4
:10C8B0000080FA00000006001800FA00204F9800DF
:10C8C000610798006E0090000000E0001B0032003D
:10C8D0002E4890000000FB00300F98003E089000AA
:10C8E000E50F50000F003200BE089000E68F5000A8
:10C8F0000F0032003E099000E40F510001003200A9
:10C90000DE01370010002000A0198A00D019820033
:10C91000E60F5000D9013A001000200070198A007B
:10C92000D60137001000200090198A00D30137008B
:10C930001000200080198A00D0013700D019820031
:10C94000E10F500024003A002E489000EE4F5000B6
:10C9500021003A0030022000400798000E00370006
:10C96000C1198200403424007E419000827078001A
:10C970000100E800C0198A00E0198200E70F5000AA
:10C9800005003A0001C8B3007E40900000C070006E
:10C9900076720200000000004E0190004E009000F0
:10C9A0000000E800400798008000EB0002007800DB
:10C9B000E425020000000000704798007E409000CF
:10C9C0000004E000E6FF3A00C04C800000D0A10067
:10C9D000C04C8800A9013700D0198200E10F500037
:10C9E00076003A002E489000F14F500073003A0054
:10C9F0008000EB00A0002000E42502000000000001
:10CA00000000FB004800DD00200798008000EB00DC
:10CA1000B0002000E4250200000000008000FB00C0
:10CA2000F00F2000808060002E0090000100400088
:10CA3000200798002E0090003006B000800078009B
:10CA4000600C2000808F500003003E00E01982003F
:10CA5000E70F5000080032002E0090004206200030
:10CA6000110009000200D80001C3B300814040005A
:10CA7000415798000200370042C5B3004257980062
:10CA80004E509000604798002E0090004206200013
:10CA9000110009000200D8008000FD002007980066
:10CAA000C1198200403424006E41900082707800E9
:10CAB0000100E800C0198A00E0198200E70F500069
:10CAC00005003A0001C8B3006E40900000C070003D
:10CAD00076720200000000002E0090006900400005
:10CAE000F20F500008003E00EE40900000C3B3007B
:10CAF00080CF50000A003200EE40900040C5B300E5
:10CB000080CF5000060032002E009000A2002000CE
:10CB1000110009000200D8000043B00060479800EF
:10CB2000C1198200403424006E4190008270780068
:10CB30000100E800C0198A00E0198200E70F5000E8
:10CB400005003A0001C8B3006E40900000C07000BC
:10CB500076720200000000002E009000A20020006B
:10CB6000110009000200D8008000FD000043B00061
:10CB700060479800C1198200403424006E41900043
:10CB8000827078000100E800C0198A00E019820074
:10CB9000E70F500005003A0001C8B3006E40900056
:10CBA00000C070007672020000000000C04C8000DF
:10CBB00000D0A100C04C880030013700D01982009D
:10CBC000E10F500022003A002E489000EF4F500035
:10CBD0001F003A000000EB00100798001500370016
:10CBE0009E00900020392300614F78001E04E00071
:10CBF00013003200C1198200403424001E41780025
:10CC0000827078000100E800C0198A00E0198200F3
:10CC1000E70F500004003A0000C8B3001E40700047
:10CC200076720200000000001E0090000000E80084
:10CC3000100798001E009000EF0F5000E8FF34002E
:10CC4000C04C800000D0A100C04C88000B01370010
:10CC50000091200010407800E74F500009003A0092
:10CC600020CD80000000E00006003A00C04C8000AB
:10CC700000D0A000C04C880000992000AE48900071
:10CC8000014878002E4890008000FB00F00720004B
:10CC900000806000E80F5000C20032002E48900073
:10CCA000804078000174A100005024000148780001
:10CCB000E0422300104078000080FB00100F980035
:10CCC0001E099000E20F5100870032001E089000FC
:10CCD000E20F500007003C009E0890000100E000B9
:10CCE000110032001E099000E10F510017003200C0
:10CCF0008C003700B00420009E089000808F500008
:10CD00005A003200300520001E099000800F5100AB
:10CD100044003200200420009E089000808F5000C4
:10CD2000400032007F00370000502400904078001F
:10CD300000C2B30080CF50007D003A00E1422300E2
:10CD400010C0B300804878007900370000502400FC
:10CD5000104078000000FB00000F98003005200014
:10CD60000E099000800F510026003200300520008F
:10CD70008E089000808F50000D003C0020042000A1
:10CD80000E099000800F510016003200B004200000
:10CD90008E089000808F50001600320000022000A4
:10CDA0000E099000800F5100610032001900370019
:10CDB000B00620008E089000808F50000D003200D9
:10CDC000300720000E099000800F51000D00320046
:10CDD000200620008E089000808F50000100320055
:10CDE0000C003700E142230020C4B30080487800E3
:10CDF0004F003700E1422300B0C4B3008048780000
:10CE00004B003700E142230030C5B3008048780072
:10CE100047003700E14223000040EB0080487800E3
:10CE2000430037000050240090407800B0C4B300A5
:10CE300080CF500005003200005024009040780060
:10CE4000B0C6B30080CF500004003A00E142230096
:10CE500020C0B3008048780035003700E14223004D
:10CE60000040EB008048780031003700005024007B
:10CE7000104078000000FB0070079800E0042000DC
:10CE80007E019000800F51000F003200E00620006C
:10CE9000FE009000808F50000B0032000002200046
:10CEA0007E019000800F5100010032000A0037001F
:10CEB00020C0B300204F9800E142230010C0B3000F
:10CEC000804878001A003700E142230020C0B300F8
:10CED0008048780016003700E14223000040EB0054
:10CEE00080487800120037000050240090407800FD
:10CEF00000C2B30080CF500006003A0020C0B3004B
:10CF0000204F9800E142230010C0B3008048780011
:10CF100007003700E14223000040EB008048780022
:10CF200003003700E14223000040EB008048780016
:10CF3000C1198200403424002E499000827078008C
:10CF40000100E800C0198A00C1198200F00F20001A
:10CF5000808F5000020034000000EB00C0198A00EE
:10CF60002E4890008000FB00F007200080806000C9
:10CF700000022000808F5000060032002E489000F2
:10CF80008000FB00F007200000806000F00F5000E0
:10CF90003A003C00102882000000E80010288A00B7
:10CFA00036003700D0198200E10F500027003A0008
:10CFB0000091200010407800E74F500023003A0015
:10CFC00010288200E10F50001C003200C1198200BD
:10CFD000B0198200808F500018003200C019820002
:10CFE0000000E900C0198A00C01982000000E000BA
:10CFF00002003D00F00F2000C0198A00C119820014
:10D0000040342400614078008000FB00F0072000DD
:10D010008080600000022000808F500017003A00DE
:10D0200010288200E10F5000140034001028820004
:10D030000000E90010288A0010003700C04C800072
:10D0400000D0A100C04C88000C003700C21982003B
:10D050004134240080C0B30000F178000200E800F1
:10D06000C0198A00C1198200F00F2000808F500083
:10D07000020034000000EB00C0198A000080FA00B2
:10D08000000006000200FA00C1198200B0198200F7
:10D09000808F50003800320000912000104078004E
:10D0A000E74F500003003A00102882000000E00023
:10D0B00031003200B1198200403424006140780010
:10D0C000804078000174A100014F78000091200099
:10D0D00010407800E74F500006003A00B019820077
:10D0E000413424001E41780002F07800B01982001B
:10D0F00090A18900B01982000000E800B0198A00F0
:10D10000B1198200F00F2000808F5000020034001F
:10D110000000EB00B0198A0000C2B3009E4F10005F
:10D120000300320000C1B3009E4F100003003C001A
:10D13000102882000000E90010288A0010288200D0
:10D140000000E00002003D000000EB0010288A0013
:10D150005080200010407800704060000004E00023
:10D160000900320011C0B3001E407800567C020056
:10D1700000000000040037000000EB0010288A00C7
:10D1800010C0B300004F7800A01982000000E0003A
:10D19000040032000000EB00A0198A0010002000FB
:10D1A00070198A00901982000000E000040032002B
:10D1B0000000EB0090198A001000200060198A001E
:10D1C000801982000000E000040032000000EB0043
:10D1D00080198A001000200050198A001E00FB00F0
:10D1E0000080FA00000006000000FA000000EB00DA
:10D1F000C0198A00C0198200B0198A000000EB0033
:10D2000050198A000000EB0090198A000000EB0022
:10D21000A0198A000000EB0080198A000080FA0043
:10D22000000006000200FA00C1198200B019820055
:10D23000008F50001E00E00002003D0000102000A2
:10D240001E0F40001E0078000080FA00000006005B
:10D250000400FA00008FBE001E00BE00E00F500068
:10D26000E08F58000800340040002000010020003A
:10D27000BE0F1000AE8F180003003C001E007800A7
:10D28000101A8A000200370020002000101A8A00BD
:10D290000080FA00000006000200FA00C1198200B6
:10D2A000B0198200808F50000E003200B219820047
:10D2B00040342400E240780000C0EB0000CF600062
:10D2C0000200E800B0198A00B1198200F00F2000B6
:10D2D000808F5000050034000000EB00B0198A0078
:10D2E000020037000040EB00004F78001E00FB00FA
:10D2F0000080FA00000006000000FA000080FA003A
:10D30000000006005000FA00881F78006600470001
:10D31000515F2C0015000900315878006001B10000
:10D320007C004700B2602C001500090032587800DC
:10D330006001B100200320000E00400013622C00A9
:10D3400015000900335878006001B100A19A21004E
:10D3500040C1B30080487800019B210050C0B30059
:10D3600080487800900120008091890060042000AE
:10D37000909189002000200040338A000000EB00DB
:10D3800020CD8800313A800000E02F00008060004E
:10D39000E001B300303A88000000000044C7BF003D
:10D3A000F043B20044E7B7000000000041742000E1
:10D3B0009140780000CEB30000C0600044E7B700A1
:10D3C000000000003200200081072000A00920009A
:10D3D00033742000814978008049780082497800C0
:10D3E000120020006104200070052000237420003A
:10D3F00081497800804978008249780043C7BF009E
:10D4000002C7B3008240600000C3B30080CF500069
:10D41000FAFF3A00D202A800CDA2A8006820A80016
:10D42000D2E2A900D4E2A800D342A80081E0A9007A
:10D4300040062000200F8800D222A9001000200002
:10D44000B07B020000000000F42802000000000091
:10D450007E260200000000000832020000000000EA
:10D46000F024020000000000DE7002000000000056
:10D47000213923000040EB0080487800C0032000E1
:10D4800040EA88001E61A900E11120009140780067
:10D49000F0CCB30000C060000044A0001EE1B70063
:10D4A000409C2000D00888000000EB00E0088800C5
:10D4B0008760A9001FE1A8009760A8002103200051
:10D4C0008E8040000040EB00C05098002A7102009E
:10D4D00000000000220320000E0141008040EB000C
:10D4E0000040EB007A710200000000001102800091
:10D4F000F0F12F000080600010028800BE8502005D
:10D5000000000000A0A08900A0A081000000E000B1
:10D5100014003200A0A081004880DE006F4060004F
:10D5200003C3B300834040007C00470031489800AB
:10D53000A0A081004480DE006F40600002C3B30001
:10D54000824040007C00470051489800A0A0810024
:10D550006F40600003C3B300834040007C0047007D
:10D5600061489800E0C2BF00704060000004E00025
:10D570004F003200A20020008000EB00E0532C009E
:10D58000CA88020000000000007D200050700200E8
:10D59000000000008000EB0000542C00267C0200FC
:10D5A000000000008000EB000000EB009A7C02000D
:10D5B00000000000100798001E0090000000E0002E
:10D5C00032003A008000EB00100020009A7C02003C
:10D5D00000000000800078001E0090000100400064
:10D5E000100798001E0090000000E00027003A009D
:10D5F000A0002000200798000B0037002E019000AB
:10D600002E009000E4005000003D2300E14078002F
:10D610006600470000004100014878002E0090009D
:10D620000000E800200798002E009000F20F500044
:10D63000F2FF3400660047008050900030C4B30011
:10D6400080CF50000C003A00660047001050900058
:10D650000000FB006A00B900800078006600470007
:10D66000205090000000FB008080400000DF2F0071
:10D670000080400090A08900660147008040EB00D8
:10D6800010C0B3007A71020000000000A0A0810069
:10D690000000E0000B0035007C0147008040EB00FB
:10D6A00020C0B3007A7102000000000005003700BE
:10D6B00052542C008040EB0010C0B3007A7102007D
:10D6C00000000000B2552C008040EB0040C0B300C9
:10D6D0007A7102000000000012572C008040EB001D
:10D6E00050C0B3007A7102000000000072582C0094
:10D6F0008040EB0060C0B3007A71020000000000BF
:10D70000D2592C008040EB0070C0B3007A71020047
:10D7100000000000803E2000507002000000000069
:10D72000E7C2BF00624060000004E0001D003A0054
:10D730000040EB006C70020000000000325B2C0027
:10D740008040EB0020C0B3007A71020000000000AE
:10D75000925C2C008040EB0030C0B3007A71020074
:10D7600000000000F25D2C008040EB0040C0B300E0
:10D770007A71020000000000325B2C008040EB0058
:10D7800050C0B3007A710200000000001002800057
:10D79000010E200001007000100288000048040003
:10D7A00001000000DE29020000000000200020002F
:10D7B0005093020000000000F190200020C0B30050
:10D7C00080487800088A0200000000001000200055
:10D7D000B0808900B08081008040780030912000C6
:10D7E0000148780024240200000000000000EB0043
:10D7F0007A39020000000000019120000040EB0097
:10D80000804878008000EB000000EB00E425020077
:10D81000000000008040780030C7B30080CF500087
:10D8200002003A00ACA80200000000008000EB00FB
:10D8300000022000E42502000000000010479800CC
:10D840009E40900040C6B30080CF500002003A00D6
:10D850006495020000000000E2B202000000000037
:10D8600000802000BE8B0200000000002C61A80098
:10D87000C11220009140780000C3B30000C07000C6
:10D880002CE1B700C003200040EA8800100020000F
:10D8900050EA880048EA80006140B900BA080200F6
:10D8A0000000000060279800712798000800E00041
:10D8B00008003D0002002000037824006E20900044
:10D8C000FE20900000080200000000006027980081
:10D8D000712798006E209000FE2090002269290098
:10D8E0008301240096070200000000000E0A0200D7
:10D8F000000000005009880040EA8000010020007C
:10D9000080017800A22526000219B8008002D0000C
:10D910000302780005024200A52526000588B9000B
:10D9200000024200840178005009800001002000BC
:10D93000C000DD0000002000000051004009880008
:10D940008A00A9002DE1A9009A00A80030408000BB
:10D950000060A000304088000000EB002007980025
:10D96000140037000000EB00100798000A00370091
:10D970002E0090009E0090004700DD000101400055
:10D98000E19B21000040EB0000F178001E009000B8
:10D990000000E800100798009E009000F0072000AB
:10D9A000808F5000F2FF34002E0090000000E8004D
:10D9B000200798002E009000E20F5000E9FF34008D
:10D9C0000091200010407800E74F50000A003A0014
:10D9D0005092810061928100404C8800514C880037
:10D9E0005092810061928100E0968900F196890051
:10D9F000C2C20200000000000CDE020000000000B5
:10DA0000D4C2BF00614060008000EB005127980045
:10DA10000004E000020032001200200052279800AB
:10DA2000DE21900043A089000040EB006C700200F2
:10DA300000000000AE2902000000000000003700D6
:10DA400040802000104078000044B2000004E00054
:10DA50000F003200408020009040780000C8B300E2
:10DA600000C060000004E000090032002040800097
:10DA70000070A10020408800B6980200000000005D
:10DA8000204080000060A10020408800ECFF3700AB
:10DA9000D01982000000E00047003A00B0A08100E9
:10DAA0000000E00018003200B0A08100ACD60200F7
:10DAB00000000000B0A081002040900076720200BB
:10DAC00000000000B0A08100304090000004E000A1
:10DAD00008003200B1A08100B0A081003040900069
:10DAE000A0409800B1A081000040EB00B040980039
:10DAF00005003700B0A081008040EB0001487800AD
:10DB00000000EB00B0A08900C04C80000180200024
:10DB1000010060000000E00005003200C04C800001
:10DB200000B0A100C04C8800DC3D020000000000F5
:10DB300020DA8000E10F500004003A000000EB0002
:10DB400020DA8800B8410200000000004080200078
:10DB5000104078000042B2000004E00006003200ED
:10DB6000204080000050A10020408800204080001C
:10DB70000060A00020408800408020001040780015
:10DB8000704060000004E000180032004C8D02007C
:10DB90000000000040A081000000E0000200320010
:10DBA00042E8020000000000204080000040A10088
:10DBB000204088000D00370040A081000000E000F8
:10DBC0000A00320040802000104078007040600061
:10DBD0000004E0000500320042E8020000000000FE
:10DBE000204080000040A10020408800C04C800000
:10DBF00001402000010060000000E000050032004C
:10DC0000C04C800000A0A100C04C8800348E0200EF
:10DC100000000000C04C80000100210001006000F5
:10DC20000000E00005003200C04C800000C0A100F0
:10DC3000C04C88009094020000000000C04C80009E
:10DC400001002200010060000000E0000700320037
:10DC5000C04C800000D0A100C04C8800009920007A
:10DC600010407800767202000000000090A1810050
:10DC70000000E00002003500B6DA020000000000FB
:10DC8000C04C800001082000010060000000E0009E
:10DC900005003200C04C80000070A100C04C88001C
:10DCA000188C020000000000C04C8000010420001D
:10DCB000010060000000E0000B003200314C8000E9
:10DCC00000002200808F5000070034000000EB00AD
:10DCD000304C8800C04C80000060A100C04C88001F
:10DCE0004C8D020000000000C04C8000012020008C
:10DCF000010060000000E00005003200C04C800020
:10DD00000090A100C04C8800D65502000000000021
:10DD100010DA8000E10F50000B003A000000EB0029
:10DD200010DA880050EA80000000E80050EA88001D
:10DD3000127B02000000000030082000E0CC8800C8
:10DD4000FE8F020000000000809B81000000E000C8
:10DD5000020032008286020000000000E01982000A
:10DD6000E70F50000300320040A081000000E000F7
:10DD70001C003200D0198200E10F500019003A0057
:10DD8000210F800040062000808F500015003200D7
:10DD900050802000104078000044B2000004E000F1
:10DDA000100032002040800000E0A10020408800E8
:10DDB000C04C8000700060000000E00004003A00E9
:10DDC000E7C2BF00624060000004E00003003A00C8
:10DDD0005CDD02000000000002003700E8DC020009
:10DDE00000000000408020009040780000C8B30090
:10DDF00000C060000004E000070032002040800006
:10DE00000070A10020408800D0A5020000000000A2
:10DE1000F4970200000000002DC1BF0001C8B3004C
:10DE2000014060000004E00002003200BA7A020003
:10DE300000000000508020001080FB004400DE0045
:10DE4000614060008080FB00508020001080FB005B
:10DE50004500DE00614060000080FB000080600043
:10DE60000000E00005003200627A020000000000BD
:10DE70002040800000D0A10020408800E096810072
:10DE8000F19681007233810083338100FE07020026
:10DE90000000000010090200000000004027980068
:10DEA0004E2090000000E00003003D00CE209000D6
:10DEB0008100EA00412798004E2190006110B900CE
:10DEC000BA0802000000000002002000030A24003B
:10DED000C4090200000000000000E00001003C0056
:10DEE0001B003700E0968100F196810002002000BF
:10DEF000A317240012070200000000000200200007
:10DF000003F02300000802000000000010090200D6
:10DF1000000000008000780000FE2F00008040001C
:10DF2000209789009A76020000000000E019820024
:10DF3000E60F500004003200209781000E750200A9
:10DF400000000000020037005076020000000000D0
:10DF5000E0968100F1968100703389008133890059
:10DF6000422A02000000000010A081000000E00032
:10DF70000400320012E60200000000000000EB0086
:10DF800010A08900D42C0200000000004CC4020044
:10DF90000000000080A081000000E000A8FE320028
:10DFA0000000EB0080A0890038CE020000000000D5
:10DFB000A3FE37000000FA00D802A800D822A8006B
:10DFC000D842A800D862A800D882A800D8A2A80089
:10DFD000D8C2A800D8E2A8000080FA00000006001D
:10DFE0000000FA00D802A900D822A900D842A9004E
:10DFF000D862A900D882A900D8A2A900D8C2A900D5
:10E00000D8E2A9000080FA00000006000000FA0033
:10E0100006000900000000000080FA000000060071
:10E020000000FA000C000900000000000080FA0067
:10E03000000006000000FA00A00F09000000000028
:10E040000080FA00000006000200FA000000EB0069
:10E05000000F780002003700F6FF07001E0FE800EF
:10E06000900F20009E0F1000FBFF34000080FA008C
:10E07000000006000200FA000000EB00000F78002C
:10E0800002003700EBFF07001E0FE800100320001E
:10E090009E0F1000FBFF34000080FA000000060015
:10E0A0000400FA00100798000000EB00000F780051
:10E0B00002003700DFFF07001E0FE8001E01780096
:10E0C0001E0090006A00B900800F5100F9FF39006E
:10E0D0000080FA00000006000600FA0040479800A1
:10E0E00001CCB30020C0B300E80107004E4090000F
:10E0F0000080FB00000F7800280037001E00780029
:10E100008040780080CBB30000C070008040780071
:10E1100020C0B300DD01070001C4B30020C0B3007C
:10E12000DA010700012522000040EB00804878005A
:10E130000000EB0010079800060037008040EB005D
:10E140000040EB00930107001E0090000000E80073
:10E15000100798009E009000F0032000808F500070
:10E16000F6FF34000000EB001007980006003700AF
:10E170008040EB000040EB00860107001E0090008D
:10E180000000E800100798009E009000F0032000B7
:10E19000808F5000F6FF34001E0FE8007000200052
:10E1A0009E0F1000D5FF3400012522000040EB0037
:10E1B000804878000080FA00000006000000FA00A5
:10E1C000DC02A900DC22A900DC42A900DC62A90073
:10E1D000DC82A900DCA2A900DCC2A900DCE2A90063
:10E1E000D642A800D662A800D682A800D6A2A8006F
:10E1F000D6C2A900CDC2A900D802A900D822A90080
:10E20000D842A900D862A900D882A900D8A2A90042
:10E21000D8C2A900D8E2A900D202A900D222A9003E
:10E22000D242A900D262A900D282A900D2A2A9003A
:10E23000D2C2A900F1C3B30020C0B300930107000C
:10E240000040EB00A4FF0700D1C2A8000080FA0044
:10E25000000006000000FA001000070040C0B300F4
:10E260009DFF07008040EB0070C0B3004001070035
:10E270000080FA00000006000000FA0001C4B300AC
:10E2800020C0B3008101070081CBB30020C0B300E0
:10E290007E0107000080FA00000006000200FA007C
:10E2A0000000EB00000F7800060037009E007800A9
:10E2B000602823008080400000C2B30080487800BE
:10E2C0001E0FE800B00320009E0F1000F7FF34007F
:10E2D000212C23000040EB00804878000000EB0078
:10E2E000209689000000EB00309689000080FA003B
:10E2F000000006000800FA00204798003147980007
:10E3000022079800BE4090002E40900018010700A0
:10E31000030037001E4078008040EB001B0307001D
:10E320002E009000104F78001E4078006047980043
:10E330006E4090000004E0000200320010C0B30004
:10E34000604798006E409000AE0090008100E800A9
:10E35000210798000004E000EEFF3A000080FA0078
:10E36000000006000E00FA00204F9800314F980080
:10E37000620798006400470021092C00040009008E
:10E38000315878005000B100E50040000040EB003B
:10E390008048780030002000100798006E00900040
:10E3A0001000BE001009020000000000000F7800FD
:10E3B000170037009E0190001E007800A200200088
:10E3C000110009000200D8008000FD0002C3B30064
:10E3D000824040006400470000804100014878000E
:10E3E0001E0090000000E900100798001E00780051
:10E3F000A2002000110009000200D800000F7800E0
:10E4000064014700BE4890002E489000B9FF070005
:10E410001E00E000E7FF3C000080FA00000006005C
:10E420000400FA0040C0B3002BFF0700508020001A
:10E4300010407800704060000004E00001003200ED
:10E44000200407000000EB00000F78001E003700DA
:10E450001E007800644040008040EB00C4000700CC
:10E460000000EB0010079800130037002196810090
:10E470001E009000008140001E0078007400B9006A
:10E4800000004100C2032000110009000200D80072
:10E490008000FD008000780060282300008040009C
:10E4A000104078008040EB00B80207001E0090008A
:10E4B0000000E800100798001E009000F30F5000C5
:10E4C000EAFF34001E0FE800200020009E0F10001D
:10E4D000DFFF34008040EB0070C0B300A4000700F1
:10E4E000D00307000080FA00000006000200FA00D6
:10E4F000004F78001E80FB00F10720000100600043
:10E50000E80F500029003A0030968100F40F4000D7
:10E5100026003400209681000000E9002096890042
:10E520008040EB0000C2B3009802070030968100E3
:10E530000000E90030968900309681000000E0007C
:10E540000E003D00309681006600B9008047B000A3
:10E550008040780060C0B30085000700B103070069
:10E56000309681006600B9008047B0008040780096
:10E5700060C0B3007E0007003B003700309681008A
:10E580006600B9008040780070C0B30078000700D2
:10E59000A4030700309681006600B900804078002F
:10E5A00070C0B300720007002F0037001E80FB0010
:10E5B000F107200001006000E80F50002A0032003F
:10E5C0008040EB001E40780070020700309681000A
:10E5D000E10F400001003200920307002096810005
:10E5E0000000E0000400350020968100612823002F
:10E5F000010040001E487800209681000000E800DD
:10E600002096890020968100C20320001100090095
:10E610000200D8008000FD0020968900309681001D
:10E620000000E80030968900309681000000E0008C
:10E6300007003A008040EB0070C0B3004C000700B8
:10E64000780307008040EB0070C0B300480007006B
:10E6500030968100F40F500003003A000000EB00F8
:10E66000309689006EFF0700D01982000000E0009C
:10E6700003003200D0198200E20F50000A003A0075
:10E680005080200010407800704060000004E000DE
:10E69000050032001E4078000074A10011C0B300D4
:10E6A000567C0200000000000080FA000000060016
:10E6B0000200FA00004F7800E0C3B3001E40700073
:10E6C0008040780020C0B300700007000080FA008E
:10E6D000000006000200FA00004F780030C0B300CE
:10E6E0009E4F100002003600102522001E487800C0
:10E6F00080CBB3009E40700020C0B30063000700D1
:10E700000080FA00000006000200FA00004F7800C6
:10E71000F0C3B3009E4F1000090036001E40780081
:10E72000F2C3B3008240600000C4B30000C07000B8
:10E730008040780010C0B300540007000800370084
:10E740001E407800F2C3B3008240600000C4B300F2
:10E7500000C07000804078000040EB004B000700D4
:10E76000002522001E4878000080FA000000060004
:10E770000200FA00004F7800114798001E40780010
:10E78000D4FF07001E409000DFFF07000080FA0062
:10E79000000006000200FA00004F780011479800C0
:10E7A000002522009040780000C4B30080CF5000C4
:10E7B00005003A000025220010407800D2FF070033
:10E7C000D642A800D662A900002522009040780019
:10E7D00000C8B30080CF500008003A000125220095
:10E7E0000040EB00804878000025220010407800AF
:10E7F000C5FF0700D642A900D662A800D6A2A9008C
:10E80000D682A800EBFD0700D6C2A80004FE0700D0
:10E81000D01680004700DE00610060000004E000C8
:10E82000FBFF3A00F9FD0700D6C2A900FCFD070076
:10E83000D682A900D6A2A800F4FD0700D6C2A8007F
:10E840001E4090000004E000040032001E80FB0027
:10E850000080EA00E0168800020037001E80FB00FE
:10E86000E0168800DEFD0700EDFD0700D6C2A90016
:10E8700000252200104078008040E800002522009A
:10E88000014878000080FA00000006000800FA0045
:10E89000004F780011479800D6A2A900D682A800A0
:10E8A000C4FD07000040EB00704798001E04E00024
:10E8B00002003A0011C0B300714798000041EB001C
:10E8C0006247980020C0B3009E4F100002003A003B
:10E8D00011C0B300614798007E419000EE40900067
:10E8E000014071000004E0000D003200D642A90092
:10E8F000D662A800C5FD0700D6C2A800C8FD070063
:10E90000D01680004700DE00610060000004E000D7
:10E91000FBFF3A00BDFD0700D6C2A900C0FD0700FD
:10E920000041EB005247980010C0B3009E4F10000A
:10E9300002003A0011C0B300514798000041EB00BB
:10E940004247980020C0B3009E4F100002003A00DA
:10E9500011C0B300414798005E419000CE40900046
:10E96000014071000004E0000D003200D642A80012
:10E97000D662A900A5FD0700D6C2A800A8FD070021
:10E98000D01680004700DE00610060000004E00057
:10E99000FBFF3A009DFD0700D6C2A900A0FD0700BD
:10E9A0001E81FB00120798001E009000E10F50002E
:10E9B0000A0032009E009000E28F50000A003200F0
:10E9C0001E0190000200E000010032000800370044
:10E9D000D642A900D662A80005003700D642A8009A
:10E9E000D662A90002003700D642A900D662A9006B
:10E9F000D682A90085FD0700D6C2A8001E4090005F
:10EA00000080FB00E016880075FD070084FD07000C
:10EA1000D6C2A9000080FA00000006000A00FA0031
:10EA20003007980000252200904078002025220021
:10EA30000148780030C0B30026FF0700E0198200CB
:10EA4000E70F500073003A000000EB002007980029
:10EA5000080037002E0090002BFF07008040EB00DD
:10EA600010C0B3004BFF07002E0090000000E8002C
:10EA700020079800AE009000F0072000808F500023
:10EA8000F4FF3400309281008000400040232300D6
:10EA90000080400010007800CF80DE00BA0802003D
:10EAA0000000000002002000A317240096070200C7
:10EAB000000000000001BE0000080200000000008D
:10EAC0000001BE0000002000A15F24001207020028
:10EAD000000000001009020000000000000F780094
:10EAE0001E00EA0020079800BE0090002E00900053
:10EAF00000804000100798003E0037001E00900084
:10EB00000000E000350035001E009000FEFE07000A
:10EB10009E00EA002E009000808F5000030032001B
:10EB20002E0090009E0F500004003A008040EB0041
:10EB3000F0C0B30017FF0700280037002E00900038
:10EB4000400798004E0090000000E0001B003200DB
:10EB50004E0090000000E00007003C004E009000D6
:10EB6000E20F40000B0032004E009000E10F400029
:10EB70000D003200160037004E009000E10F5000EB
:10EB8000090032004E009000E20F500001003200F8
:10EB90000F003700300B2B00104078008040EB0056
:10EBA000FCFE07000D003700400B2B0010407800E2
:10EBB0008040EB00F7FE070008003700500B2B00E9
:10EBC000104078008040EB00F2FE070003003700A1
:10EBD0008040EB0090C0B300EEFE07001E009000E6
:10EBE0000000E800100798002E0090000000E800E8
:10EBF000200798002E0090009E0F500021003C003E
:10EC00009E009000F0072000808F5000BBFF340072
:10EC10001C0037000000EB002007980016003700AA
:10EC2000BE0090002E009000008040000080E900AF
:10EC3000100798001E0090000000E0000B00350057
:10EC40009E009000F0072000808F500007003C00DD
:10EC50001E009000ACFE0700AE009000300B2B00B1
:10EC6000614078008040EB00CAFE07002E00900053
:10EC70000000E800200798002E009000E40F5000EC
:10EC8000E7FF340020252200904078001025220064
:10EC900010407800B6FE07000080FA000000060071
:10ECA0000400FA0020978100CF80DE00BA0802003D
:10ECB00000000000B2472100E30A2400FE07020022
:10ECC000000000000200200003F023000008020002
:10ECD000000000001009020000000000100798006A
:10ECE00020978100CF80DE00BA08020000000000FB
:10ECF000B2472100E30A24000008020000000000DF
:10ED00000200200003F023000008020000000000C1
:10ED10001009020000000000000F78001E009000A3
:10ED20003EFF07001E0078003CFF07000080FA004D
:10ED3000000006000200FA00002522009040780042
:10ED400020252200014878008040EB0030C0B3004D
:10ED500087FE07000000EB00000F7800040037007A
:10ED60008040EB0010C0B3008AFE07001E0FE800D1
:10ED7000F00720009E0F1000F9FF3400202522002C
:10ED800090407800102522001040780078FE07009F
:10ED90000080FA00000006000600FA0000252200AC
:10EDA0009040780020252200014878000000EB0008
:10EDB000200798006B0037002E00900080407800FC
:10EDC00020C0B3000140500042FE07000040EB00AD
:10EDD0004DFE07000000EB001007980027003700E9
:10EDE0001E0090008000400060462200008040002D
:10EDF000900078002E0090004300DD00008050005D
:10EE0000000F78001E00E00002003D000000EB0053
:10EE1000000F7800800020009E0F100002003400D8
:10EE200080002000000F78001E0078008080FB002A
:10EE3000A00A2B00614078000080FB00000F7800E2
:10EE40002E009000620010009E0090004700DD0040
:10EE500081004000E09B2100614078000000FB0041
:10EE60001E0F68001E0078008040EB0049FE07007E
:10EE70001E0090000000E800100798009E0090001F
:10EE8000F0032000808F5000D5FF340000C4B30091
:10EE90001DFE07000000EB00100798002A00370055
:10EEA0001E0090000004B000800040006046220078
:10EEB00000804000900078002E0090004300DD00AC
:10EEC00000805000000F78001E00E00002003D00AE
:10EED0000000EB00000F7800800020009E0F100063
:10EEE0000200340080002000000F78001E0078002F
:10EEF0008080FB00A00A2B00614078000080FB00AE
:10EF0000000F78002E009000620110001E0090009B
:10EF100001042000808040004710DD008100400097
:10EF2000E09B2100614078000000FB001E0F68009C
:10EF30001E0078008040EB0016FE07001E009000C7
:10EF40000000E800100798009E009000F0032000E9
:10EF5000808F5000D2FF34002E0090000000E800A7
:10EF6000200798002E009000E20F500092FF34001E
:10EF700020252200904078001025220010407800C3
:10EF8000FBFD07000080FA00000006000600FA0002
:10EF900040479800514798004E4090000074A100EF
:10EFA00010479800CE4090000040EB00004F7800E2
:10EFB0000104E00002003D0010C0B300004F7800E3
:10EFC0001E409000ED4F500002003A0070C1B300A7
:10EFD000104798000000EB00100798000D00370064
:10EFE0001E4090000080FB001E0190006500B900EB
:10EFF0008200400020E12B00614078001E4070003C
:10F00000DE409000E3FD07001E0090000000E800D5
:10F01000100798001E009000E40F5000F0FF34002D
:10F02000DE4090001E407800DAFD07000080FA0004
:10F0300000000600DC00FA006500470081092C0092
:10F0400015000900315878006001B1007B004700CD
:10F05000E20A2C0015000900325878006001B10066
:10F06000100320000E004000410C2C001500090088
:10F07000315878006001B100700420000E0040009B
:10F08000A20D2C0015000900325878006001B10073
:10F09000D00520000E004000010F2C0015000900D3
:10F0A000315878006001B100300720000E004000A8
:10F0B00062102C0015000900325878006001B10080
:10F0C000900820000E004000C1112C00150009001E
:10F0D000315878006001B100F00920000E004000B6
:10F0E00022132C0015000900325878006001B1008D
:10F0F000500B20000E00400081142C00100009006D
:10F10000315878001001B100600C20000E00400062
:10F1100092152C0010000900325878001001B1003F
:10F12000D0052000000F4700002522009040780005
:10F1300041479800F20920000E0141008040EB0099
:10F1400010C0B3006BFC0700009120001040780055
:10F150000000FB0050AF98005EA99000E20F510044
:10F16000150032005EA89000E20F500007003C003E
:10F17000DEA890000100E0000B0032005EA99000C4
:10F18000E10F51000A003200720037005EA89000C3
:10F19000E60F50000B003200DEA89000E78F500011
:10F1A0000B0032006B003700650F47006900370025
:10F1B0007B0F47006700370012032000020F470053
:10F1C0006400370070042000000F47006100370022
:10F1D000902D2300104078000004E000030032006E
:10F1E00031072000010F470009003700A02D230040
:10F1F000104078000004E000030032009208200074
:10F20000020F470002003700D0052000000F470022
:10F2100060CD80000000E00006003A00620C200093
:10F220000E014100E1C1B30020C0B30031FC070072
:10F2300048003700009B2100104078000001FB00CF
:10F2400000FA2000110009000200D8001007980001
:10F250001E009000703EB00080007800E07C20002E
:10F26000808F5000080036001E009000823E200073
:10F27000110009000200D80001C3B3008140400022
:10F2800001DF99000200370002C2B30002DF9900DB
:10F29000500B20000E0040008ED8910001489800CD
:10F2A0001E009000823E2000110009000200D800DC
:10F2B0008000FD00100798001E009000420620000C
:10F2C000110009000200D80002C3B30082404000D0
:10F2D000500B20000E004000114898001E009000C6
:10F2E00042062000110009000200D8008000FD0045
:10F2F000100798001E009000A200200011000900D5
:10F300000200D80002C3B30082404000500B20002E
:10F310000E004000214898001E009000A20020002E
:10F32000110009000200D8008000FD0002C3B300F4
:10F3300082404000500B20000E00400031489800F1
:10F34000520B20000E014100E1C1B30020C0B30008
:10F35000E8FB070040A081000000E00004003A0044
:10F360000091200010407800E74F500020003A0044
:10F370001E007800EB00400000C2B3008048780017
:10F380001E017800F1004100A09A21001040780091
:10F390000000FB00A2002000811F7800110009007E
:10F3A0000200D80001017800CF0078000043B000CF
:10F3B000804878001E007800F2004000A09A2100EA
:10F3C000104078000000FB00A2002000811F7800A0
:10F3D000110009000200D800000178000100780047
:10F3E000CF0078000043B000804878000400370068
:10F3F0001E017800EB0041000040EB0080487800DF
:10F400001E0178008040EB0010C0B300B9FB07007C
:10F4100000252200CE409000014878000080FA00CC
:10F42000000006000200FA000000EB00000F780068
:10F43000040037008040EB0000C8B300D5FC070093
:10F440001E0FE800500020009E0F1000F9FF34004E
:10F45000002522001040780066405000804078006F
:10F460000025220001487800002522001040780085
:10F47000A5FC07000080FA00000006000000FA006A
:10F4800051C0B30010C0B300B9FC07008040EB00CE
:10F4900040C5B300BDFE07008040EB0050C5B3007F
:10F4A000BAFE07008040EB00E0C4B300B7FE0700DF
:10F4B0008040EB0050C4B300B4FE07000080FA00A7
:10F4C000000006000000FA0091C7B30040C0B3007E
:10F4D000A7FC070011C0B3000040EB00ADFC070023
:10F4E00011C0B30020C5B300A8FE070091C7B30048
:10F4F00050C0B3009EFC070011C0B3000040EB00F9
:10F50000A4FC070011C0B30050C4B3009FFE070065
:10F5100091C7B30060C0B30095FC070011C0B300F1
:10F520000040EB009BFC070011C0B30030C4B300E7
:10F5300096FE070091C7B30070C0B3008CFC0700B3
:10F5400011C0B3000040EB0092FC070011C0B300F3
:10F5500000C2B3008DFE0700309681006600B9003E
:10F560008040780070C0B30081FC07000080FA0082
:10F57000000006000000FA0091C7B30040C0B300CD
:10F580007BFC070011C0B3000040EB0081FC0700CA
:10F5900011C0B30020C4B3007CFE070091C7B300C4
:10F5A00050C0B30072FC070011C0B3000040EB0074
:10F5B00078FC070011C0B30030C4B30073FE07002D
:10F5C00091C7B30060C0B30069FC070011C0B3006D
:10F5D0000040EB006FFC070011C0B300E0C4B300B3
:10F5E0006AFE070091C7B30070C0B30060FC07005B
:10F5F00011C0B3000040EB0066FC070011C0B3006F
:10F6000000C2B30061FE0700309681006600B900B9
:10F610008040780070C0B30055FC07000080FA00FD
:10F62000000006001400FA0050EA8000801F7800F5
:10F63000A0162C00801F78000E00780038180200F9
:10F6400000000000E48757000E0178008040EB00C6
:10F650000040EB0027FB07008040EB0070C0B300C8
:10F6600043FC07000080FA00000006000200FA00D8
:10F670000000EB00000F78000B0037001E00780040
:10F680006440400091C7B30039FC07008040EB00A4
:10F690000040EB003FFC07008040EB0000C2B300DD
:10F6A0003AFE07001E0FE800300020009E0F1000F9
:10F6B000F2FF3400309681006600B9008040780087
:10F6C00070C0B3002AFC07000080FA0000000600AA
:10F6D0000000FA0031C7B30010C0B30024FC0700DB
:10F6E00030408000640060000000E0000400320050
:10F6F0008040EB0060C4B30024FE07000300370025
:10F700008040EB00C0C4B30020FE070091C7B300E7
:10F7100010C0B30016FC0700304080006800600095
:10F720000000E000040032008040EB0020C5B30080
:10F7300016FE0700030037008040EB00E0C4B30072
:10F7400012FE07002025220090407800102522009C
:10F750001040780006FC07000080FA000000060058
:10F760000200FA00000F7800100020009E0F100029
:10F7700003003A0040012000C01188000200370059
:10F7800030102000C011880000002800801188007F
:10F7900000402000901188000080FA000000060060
:10F7A0000400FA00000F78000000EB0010CD880084
:10F7B0000000370011CD800000E22400808F50004F
:10F7C00006003400000000000000EB0010CD8800AF
:10F7D00030002000100798001900370032C2BF0027
:10F7E000644060000004E0000300320020002000BC
:10F7F000100798001200370032C2BF00624060005C
:10F800000004E000020032003222A900E9FF3700C4
:10F8100032C2BF00614060000004E000E5FF32003A
:10F82000B0118000804078001E0078000148780008
:10F830000000EB0010CD88000000EB0010079800DE
:10F840001E0090000080FA00000006000600FA008A
:10F85000100798004147980003003700CE40900001
:10F860001E407800110007001E009000104F780025
:10F870001E407800504798005E4090000004E00071
:10F880000200320010C0B300504798005E40900064
:10F890009E0090008100E800110798000004E0003D
:10F8A000EEFF3A000080FA00000006000400FA00B3
:10F8B000204798003147980033C2BF006140600084
:10F8C0000004E000FCFF3200D5C2BF0064406000CD
:10F8D0000004E000FCFF3A002E4090000000FB0016
:10F8E000A01188003E4090000004E0000E003200AD
:10F8F00000CD80000000E80000CD880000CD800031
:10F90000F40F500008003A000000EB0000CD880022
:10F91000510020000000EB00060007008040EB00D3
:10F92000007A2C00C9FF07000000EB000080FA00FD
:10F93000000006000C00FA0020079800310798002C
:10F940000000EB00000F78000040EB00204798001B
:10F9500090A08100E20F500003003C003E009000A8
:10F960000000E0004E003A002E0090000000E00091
:10F9700002003A000000EB0080A189003222A900B9
:10F980003D0037000E80E80085FF0700000F78007B
:10F990001E007800500798005E009000E10F5000B4
:10F9A0001E0032005E009000E10F500004003C0099
:10F9B0005E0090000000E0000800320029003700DF
:10F9C0005E009000E20F50001A0032005E009000CE
:10F9D000E30F50001D0032002200370082A1810099
:10F9E000AE409000003D2300017178000200E80065
:10F9F00080A1890080A18100400798004E009000FE
:10FA0000F80F5000020034008001200040079800E9
:10FA10004E00900080A1890017003700827A2C00E8
:10FA20008040EB0030C0B3007A710200000000009B
:10FA300011003700E27B2C008040EB0030C0B300A7
:10FA40007A710200000000000B003700427D2C009C
:10FA50008040EB0030C0B3007A710200000000006B
:10FA600005003700A27E2C008040EB0030C0B300C0
:10FA70007A710200000000001E00E00003003A005E
:10FA80002E409000ED4F5000BEFF3A001E00E000F7
:10FA90000600320070B202000000000003003700D0
:10FAA0003E00900050700200000000001E00780030
:10FAB0000080FA00000006000800FA001007980015
:10FAC000210798008040EB00D0C0B30077FF07000B
:10FAD000AE0090001E00900096FF0700000F780017
:10FAE0001E00E000030032001E007800300798007E
:10FAF0001B003700003D23009040780040C4B30055
:10FB000080CF500005003A00103D2300904078005F
:10FB1000A0C3B30080CF50000F00320080A181004D
:10FB20000001E900013D23000040EB0000F17800F6
:10FB3000023D23008040EB0020C0B3007A71020038
:10FB40000000000070B20200000000000080EB0026
:10FB500030079800020037000000EB0030079800E3
:10FB60003E0090000080FA0000000600020404003D
:10FB700000000000000006000200FA000030230030
:10FB8000104078000080FB00000F78004030230018
:10FB9000104078008040E8004030230001487800A1
:10FBA0004030230090407800B0C3B30080CF5000B5
:10FBB00062003600413023000040EB0080487800AE
:10FBC00030302300104078008040E80030302300BF
:10FBD000014878003030230090407800B0C3B30073
:10FBE00080CF500055003600313023000040EB003C
:10FBF0008048780020302300104078008040E800E2
:10FC00002030230001487800203023001040780085
:10FC1000F74F500049003600213023000040EB0030
:10FC200080487800200020009E0F100012003A004B
:10FC3000F02F2300104078000080FB00630060007C
:10FC40000000E0000C003A00F02F23001040780084
:10FC50000004E00006003A00E02F23001040780086
:10FC60000080FB00630060000000E00002003A003A
:10FC70000000EB00000F78001030230010407800E7
:10FC80008040E80010302300014878001030230045
:10FC9000104078000081FB001E00780080004000CA
:10FCA000E0472C000080400010007800800F5100D9
:10FCB000220035001130230010C0B30080487800C6
:10FCC00000302300104078008040E800003023001E
:10FCD000014878000030230010407800EC4F5000BD
:10FCE000160036000130230010C0B30080487800B1
:10FCF000F02F2300104078008040E800F02F230010
:10FD000001487800F02F23009040780030C6B300FF
:10FD100080CF500009003600F12F23000040EB0097
:10FD200080487800E02F2300104078000040E80071
:10FD300080407800E02F2300014878000080FA001E
:10FD4000000006000400FA00100798001E00900052
:10FD5000E700400050C5B300804878000000EB0089
:10FD6000000F78000D0037001E0090006701400072
:10FD70001E00900067004000904178001E0078004F
:10FD8000800078001E009000008040001040780045
:10FD900000C04100004978001E0FE800600020000C
:10FDA0009E0F1000F0FF34001E009000E70040009E
:10FDB0001E009000670040001040780000C0EA007C
:10FDC000804878000080FA00000006000400FA0075
:10FDD000000F7800900020009E0F100005003C00EE
:10FDE0001E0078000043B0000080FB001007980060
:10FDF000040037001E007800B043B0000080FB0014
:10FE0000100798001E0090000080FA000000060015
:10FE10000400FA00881F7800004F7800110798004E
:10FE20001E80FB00A2002000110009000280D80003
:10FE30000080FB00E5FF0700804078001E00900076
:10FE4000014878001E0090000004E8001E80FB00BE
:10FE5000A2002000110009000280D8008000FD00EF
:10FE60000080FB00D9FF0700004C78004F047800A9
:10FE70000080FA00000006001A00FA00400798000F
:10FE8000510798006207980073079800045798007C
:10FE90000000EB00300798006E00900010079800FB
:10FEA0004E009000104F7800D10037000000EB00AA
:10FEB00020079800CB0037001E00FB006101B9004D
:10FEC00000FE2F00F1FF2F00020140008381480057
:10FED000220F9800330F98008005200001002000B9
:10FEE0002E099000BE099000800F5100818F5900AB
:10FEF0009B003E002E089000BE08900000600100AC
:10FF000094003700930037009500370094003700C5
:10FF100093003700920037009100370090003700BF
:10FF20008F0037008E0037008D0037008C003700BF
:10FF30008B0037004B003700590037004E00370068
:10FF400087003700860037008500370084003700BF
:10FF500083003700820037008100370080003700BF
:10FF60007F0037007E003700480037007C003700F4
:10FF70007B0037007A0037007900370078003700BF
:10FF8000770037004B003700750037004E00370010
:10FF900073003700720037005000370070003700E0
:10FFA0006F0037006E0037006D0037006C003700BF
:10FFB0006B0037004E0037006900370068003700DB
:10FFC00050003700660037006500370064003700D6
:10FFD00063003700620037004F00370053003700DE
:10FFE000570037005E0037005D0037005C003700C7
:10FFF0005B0037005A0037005900370058003700BF
:020000040001F9
:10000000570037002B003700550037002E0037000F
:1000100053003700520037003000370050003700DF
:100020004F0037004E0037004D0037004C003700BE
:100030004B0037002E0037004900370048003700DA
:1000400030003700460037004500370044003700D5
:1000500043003700420037002F00370033003700DD
:10006000370037002E009000614B2C0060C07800F4
:1000700010479800430037002E009000914B2C0051
:1000800060C07800104798003E0037002E009000B6
:10009000C14B2C0060C07800104798003900370031
:1000A0002E009000F14B2C0060C0780010479800A3
:1000B000340037002E009000214C2C0060C07800E6
:1000C000104798002F0037002E009000514C2C0054
:1000D00060C07800104798002A0037002E0090007A
:1000E000814C2C0060C07800104798002500370034
:1000F0002E009000B14C2C0060C078001047980092
:10010000200037002E009000E14C2C0060C07800E9
:10011000104798001B0037002E009000114D2C0056
:1001200060C0780010479800160037002E0090003D
:10013000414D2C0060C07800104798001100370036
:100140002E009000714D2C0060C078001047980080
:100150000C0037000040EB00104798000900370002
:100160009E00FB0000FD2F00008040002E0190004B
:100170006300B9008200400080492C006140780093
:10018000104798001E009000800078005E009000EC
:1001900080804000110F98007E0090000000E00079
:1001A000050032009E4090000E50900080C0680014
:1001B00011579800020037008040EB00115798005B
:1001C0009E5190001E099000034978001E00900087
:1001D0000000E800100798002E0090000000E800E2
:1001E000200798002E009000E20F500032FF3400EC
:1001F0003E009000800078004E009000008040009B
:10020000104F78001E407800005F98008E589000D4
:100210000104E0000200320012C0B300025F980047
:100220000E589000BE0090008100E8003107980051
:100230000004E0001DFF3A000080FA000000060004
:100240001600FA0066004700A14D2C0006000900C8
:10025000315878007000B1000000EB0020079800D2
:100260000000EB001007980010002000000F78003D
:100270000000EB00200798006000370030988100F4
:10028000AE0090004300DD0081004000E0432C0000
:10029000614078000000FB00000F78001E00E000C5
:1002A000530032001E007800200F98004006200006
:1002B000AE089000808F50003900320040062000C8
:1002C000AE089000808F500008003C002E0890007F
:1002D0000000E0004300320030062000AE0890002D
:1002E000808F50000A00320039003700D00620000D
:1002F000AE089000808F50001D0032009007200053
:10030000AE089000808F50000D00320030003700A2
:100310001E00900080007800803023008080400024
:100320001E0090000000E80010079800E02F230056
:10033000104078000074A100B5FE070029003700C6
:100340001E009000800078008030230080804000F4
:100350001E0090000000E80010079800F02F230016
:10036000104078000074A100A9FE07001D003700AE
:100370001E009000800078008030230080804000C4
:100380001E0090000000E8001007980000302300D5
:10039000104078006F4060009DFE0700110037009C
:1003A0001E00900080007800803023008080400094
:1003B0001E0090000000E800100798001030230095
:1003C000104078007F40600091FE07000500370074
:1003D0001E0190001E0078008040780080302300CD
:1003E000017178001E0090000000E80010079800DE
:1003F0002E0090000000E800200798002E009000DA
:10040000E50F50000D003C001E009000EA0F500068
:100410000A003C001E00E00098FF3A000700370089
:100420001E019000813023000040EB0000F17800B5
:100430001E0090000000E800100798001E009000C9
:10044000EA0F5000F6FF34002030230010407800FF
:100450007F406000313123006DFE070061312300D1
:100460003030230010407800F043B20068FE0700EF
:10047000913123004030230010407800F043B20057
:1004800063FE0700303382000074A100E6004700DD
:100490005FFE0700A09B8100620060000000E0009A
:1004A00007003200A09B8100610060000000E000B6
:1004B0000300320010002000100F980002003700E7
:1004C0008000EB00110F9800E19B21000042EB003F
:1004D0009E0990000001EB008030230066FE0700BB
:1004E000103F23009040780030C3B30080CF50000D
:1004F00008003400103F23009040780080C3B30010
:1005000080CF500003003C00F0C3B30000579800B8
:10051000020037008040EB0001579800E19B21006A
:10052000103F23000E52900013002000A202200072
:1005300051FE0700303382000000E0000600320068
:10054000E0198200E70F500003003A00100020007D
:1005500070079800020037008000EB0071079800D8
:10056000E19B2100660047000042EB00FE01900085
:10057000C203200040FE0700B0808100E10F500060
:1005800007003A00E19B21000042EB00130020002D
:1005900012052000104E2C0037FE07000600370021
:1005A000E19B21000042EB00130020001205200017
:1005B000504E2C0030FE0700E19B21000042EB0072
:1005C00013002000D2052000C03123002AFE0700BE
:1005D000A09B8100614060000080FB00E19B210046
:1005E0000042EB00800178008206200030312300B9
:1005F00021FE07000080FA00000006000200FA0059
:100600000025220090407800202522000148780033
:100610000BFF07000040EB006A73020000000000BF
:100620000040EB0084730200000000000000EB00BB
:10063000000F7800070037009E007800E09B210043
:10064000614078008040EB00CA73020000000000A7
:100650001E0FE800F00320009E0F1000F6FF34008C
:1006600000C4B30084730200000000000000EB002F
:10067000000F780008003700000420009E004000B2
:10068000E09B2100614078008040EB00CA730200CB
:10069000000000001E0FE800F00320009E0F100075
:1006A000F5FF34002025220090407800102522001C
:1006B00010407800B8730200000000000080FA00CB
:1006C000000006000A00FA001007980021079800B1
:1006D000320798001E0090008000E80000D521003D
:1006E000614078008000FB0000FD2F00008F40007B
:1006F0001E00E00003003500900020009E0F100057
:100700000300340010002000400798001700370055
:100710009E00900000D52100614078000000FB00A1
:100720006A00B9009E00400000E22F00008F4000E8
:100730001E00E000030035003E0090009E0F1000F8
:100740000300340010002000400798000700370025
:100750002E0190001E00780080407800602F23005A
:10076000017178000000EB00400798004E009000F7
:100770000080FA00000006001000FA000000EB0004
:10078000200798000000EB00100798000000EB0025
:10079000000F78000000EB00100798004B003700B6
:1007A000309881009E0090004300DD0081004000F1
:1007B000E0432C0061417800024F98000E48900001
:1007C0000000FB007007980040062000FE0090002B
:1007D000808F500030003200400620007E019000E3
:1007E000800F510005003C0030062000FE00900004
:1007F000808F50000A00320030003700D006200001
:100800007E019000800F51001900320090072000F7
:10081000FE009000808F50000B0032002700370050
:100820001E0078001E0FE800E20120008000EB00AF
:10083000A4FF0700800078002E00900001007000E7
:10084000200798001D0037001E0078001E0FE800EA
:1008500032062000110020009AFF07008000780077
:100860002E00900001007000200798001300370050
:100870001E0078001E0FE800C200200021002000AA
:1008800090FF0700800078002E00900001007000AB
:1008900020079800090037001E0078001E0FE800AE
:1008A000F20120003100200086FF07008000780060
:1008B0002E00900001007000200798001E0090009C
:1008C0000000E800100798001E0FE8001E009000CE
:1008D000E70F5000B2FF3400802F23001040780053
:1008E000E24F500010003A00702F230010407800B3
:1008F0000080FB00630060000000E0000A003A0096
:10090000702F2300104078000004E0000B003A0034
:10091000602F2300104078000080FB00630060001F
:100920000000E00005003200802F23001040780016
:100930000080FB0060079800020037000001EB0018
:10094000620798006E00900030079800902F2300F7
:10095000104078000081FB003E00900080004000C5
:10096000E0472C0000804000100078000000E90003
:100970008000EB0051079800800F51000200340006
:1009800012002000520798002E009000DE00900018
:1009900001007000200798002E0090000000E00089
:1009A00014003A002030230010407800FF4060001F
:1009B000A02F230001487800303023001040780039
:1009C000F2C3B30082406000B02F230001487800DA
:1009D0004030230090407800C02F23000148780069
:1009E00010002000A0978900A09B81000010A000AB
:1009F000A09B89002E0090000080FA0000000600F5
:100A00000200FA000000EB00000F780072012000E5
:100A1000410020000000EB002AFF07001E0F7000BD
:100A2000B2032000510020003000200025FF070005
:100A30001E0F7000B2032000610020006000200043
:100A400020FF07001E0F70001E00E00014003A0097
:100A5000E02F230090407800602F230001487800A9
:100A6000F02F230090407800702F23000148780079
:100A70000030230010407800EF406000802F2300FA
:100A8000014878001030230010407800FF406000DB
:100A9000902F23000148780010002000A0978900C3
:100AA0001E0078000080FA00000006000200FA0034
:100AB000D01982000000E00014003A000000EB00B2
:100AC000000F7800070037001E0178009E007800B4
:100AD00080302300E140780000D5210001717800CA
:100AE0001E0FE800900020009E0F1000F6FF34005B
:100AF000A1D521000040EB00804878005000200084
:100B000060338A001000200080A089000080FA0075
:100B1000000006000200FA00D01982000000E00088
:100B200014003A000000EB00000F780007003700C7
:100B30001E0178009E00780030312300E1407800EB
:100B400000D52100017178001E0FE8007000200020
:100B50009E0F1000F6FF340081D521000040EB000D
:100B6000804878006000200060338A001000200078
:100B700080A089000080FA00000006001200FA0040
:100B8000E6004700A0CAB30080487800E6004700AE
:100B9000D0C0B3009040980068004700914E2C00F0
:100BA0000900090031587800A000B1000080EB0076
:100BB000000F7800803E2000B09B89000000EB0011
:100BC000809B89000000EB00909B8900A09B810026
:100BD0000010A100A09B89000000EB00A0978900F5
:100BE000E0C2BF00704060000004E000420032003C
:100BF0000000EB00200798003500370050C5B30017
:100C0000C00007006600470021002000CB0007005D
:100C10003222A9006800470022032000A100200022
:100C2000DA000700100798001E009000EA0F50003D
:100C300024003A006800470090407800A0CAB30042
:100C400080CF50001F003A0010002000909B8900C8
:100C5000A09B81000010A000A09B890068004700B5
:100C6000304090008080FB00000F2000008060007A
:100C70004401DD0068004700404090008080FB0098
:100C8000000E200000806000000141006800470065
:100C9000504090008080FB00000E2000008060002B
:100CA0004380DE0080004100680047006040900003
:100CB0000080FB004600DE000080FB00008F40004B
:100CC000060037002E0090000000E8002007980082
:100CD0002E009000E10F5000C8FF3400A200200059
:100CE0008000EB00304F2C002A0107002003200079
:100CF00050700200000000001E0078000080FA0022
:100D0000000006001200FA00E5004700A0CAB30088
:100D100080487800E5004700D0C0B30090409800BC
:100D200067004700514F2C00090009003158780036
:100D3000A000B100909B81000000E0005100320053
:100D40005080200010407800704060000004E000F7
:100D50004C003A000000EB00809B890050C5B300B6
:100D600068000700A09781000000E0000A00320040
:100D7000602F2300F3FB070081002000602F230079
:100D80006E0007008040EB00D0C0B300567C02002C
:100D9000000000000300370065004700210020002C
:100DA000660007006700470052002000A1002000F5
:100DB00076000700000F7800A00020009E0F1000B2
:100DC0002B003A006700470090407800A0CAB300AB
:100DD00080CF500026003A00A0CAB30040479800D8
:100DE0001000200010079800090037009E009000B6
:100DF00067004700E14078004E409000014040000D
:100E0000404798001E0090000000E800100798007E
:100E10001E009000E80F5000F4FF34004E40900098
:100E2000E14F400012003A000000EB00A09789005B
:100E300010002000100798000A0037001E009000E4
:100E40000001E9009E00900067004700E140780043
:100E5000E02F2300017178001E0090000000E800E0
:100E6000100798001E009000E80F5000F3FF3400B8
:100E7000820C20008000EB00304F2C00C5000700E2
:100E80001D003700A09781000000E0001400320030
:100E90000000EB00809B89000000EB00A097890018
:100EA0000000EB0010079800090037001E019000B9
:100EB0009E009000602F2300E1407800E02F230087
:100EC000017178001E0090000000E80010079800F3
:100ED0001E009000E70F5000F4FF340006003700BA
:100EE0009760A900809B81000000E900809B890039
:100EF0009760A80020FB0700C0FD07000080FA00F3
:100F0000000006000400FA002047980033C2BF002A
:100F1000614060000004E000FCFF32003362A80082
:100F2000F00F2000A01188002E4090000000FB0070
:100F3000A01188000080FA00000006000600FA00F8
:100F400010079800210798000000EB00000F7800C0
:100F5000090037001E007800800078001E00900015
:100F600000804000104078008040EB00567C02007A
:100F7000000000001E0FE8002E0090009E0F1000E1
:100F8000F4FF35000080FA00000006000A00FA00B5
:100F90001007980021079800320798000000EB0026
:100FA000000F78000000EB0010CD88003222A9006D
:100FB0002800370032C2BF00644060000004E00037
:100FC000090032001E007800800078001E009000AA
:100FD00080804000B011800080487800F0F72F003A
:100FE000400798002000370032C2BF006240600016
:100FF0000004E000040032003222A90000F82F00B3
:10100000400798001800370010CD8000800078005D
:101010003E009000808F5000030036001E00EA0062
:10102000400798001000370032C2BF0061406000E6
:101030000004E000070032001E0078008000780005
:101040001E00900080804000B01180008048780031
:101050001E0FE8002E0090009E0F1000D5FF3500F7
:101060001E007800400798004E0090000080FA00B3
:10107000000006000E00FA002007980031079800D3
:10108000024F9800530798000040EB00204798005B
:101090000000EB00000F78000000EB0010CD88008E
:1010A0003222A9002900370011CD80005E00900097
:1010B000808F5000030034001E00EA006007980093
:1010C0003100370032C2BF00644060000004E0001D
:1010D00005003200B011800020479800F1F72F0082
:1010E000610798002800370032C2BF0062406000EC
:1010F0000004E000020032003222A900EAFF3700BB
:1011000032C2BF00614060000004E000E6FF320030
:10111000B0118000204798000000EB0010CD88003F
:101120003E0090009E0F10000100350007003700C0
:101130001E007800800078002E00900000804000A3
:10114000AE409000014878001E0FE8000E48900065
:101150000004E00004003200AE4090000E48900011
:1011600080CF5000D0FF3A000E4890000004E0000D
:1011700003003A003E0090009E0F1000CAFF3500A9
:101180001E007800600798006E0090000080FA0052
:10119000000006001000FA00400798005107980070
:1011A0006207980010002000300798000000EB0054
:1011B00020079800070037002E0190008137230098
:1011C0000040EB0000F178002E0090000000E800E5
:1011D000200798002E009000F80F5000F6FF340012
:1011E0008000EB004E009000267C02000000000012
:1011F000EE019000D2C0B30091012000803723009F
:101200009CFF0700100798001E009000E10F50009F
:10121000070034001E0090008080E9008037230022
:10122000E1407800E0C3B30080CF500003003200FB
:101230005E0090000000E00003003A000000EB00B8
:10124000700798003B0037003E0090000000E90066
:10125000300798003E0090000000E00032003D00A2
:101260009E00900000F82F00808F500006003A008A
:10127000F24F2C008040EB0050C0B3007A710200A6
:1012800000000000230037009E009000F0F72F00C0
:10129000808F500006003A00D2502C008040EB00B6
:1012A00050C0B3007A71020000000000190037003E
:1012B0004E0190008040EB0040C0B3007A71020004
:1012C00000000000B2512C008040EB0050C0B30081
:1012D0007A7102000000000080372300104078007F
:1012E0000004E00006003200823723008040EB005B
:1012F00060C0B3007A7102000000000005003700F2
:1013000092522C008040EB0060C0B3007A71020062
:101310000000000070B20200000000001E009000FB
:1013200070079800030037003A70020000000000C8
:101330009EFF37007E0090000080FA00000006004B
:101340000400FA00000F78001107980011C0B300E4
:10135000A0C0B300567C0200000000001100200075
:101360001E007800267C02000000000011C0B300BF
:10137000C0C3B300567C0200000000001E009000B5
:101380000000E00015003200A09B810062006000B8
:101390000000E00005003200110020008030230032
:1013A000267C020000000000080037003098810011
:1013B0006D00B9008000780060452C00008040007E
:1013C00011002000267C02000000000011C0B300C4
:1013D00000C2B300567C0200000000001100200093
:1013E00030312300267C02000000000011002000A4
:1013F00050532C00267C0200000000000080FA0000
:10140000000006000000FA000080FA00000006005C
:101410000000FA00C0C72800B03A8A00A05828008F
:10142000C03A8A00C0C62800103B8A00E03D29006F
:10143000203B8A00A0392B00303B8A0060552800F1
:10144000403B8A00C0592900503B8A00C0F928005F
:10145000603B8A0000BB2800703B8A00A012270076
:10146000803B8A0040522900903B8A00404E290070
:10147000A03B8A0060882900B03B8A0000612900F7
:10148000C03B8A00A03B2B00D03B8A00604D290066
:10149000E03B8A00E0C12A00F03B8A0080C12800BE
:1014A000003C8A00E0FF2800103C8A00E0FF280092
:1014B000203C8A00E0FF2800303C8A00E0FF280042
:1014C000403C8A00E0FF2800503C8A00E0FF2800F2
:1014D000603C8A00E0FF2800703C8A0020762900EA
:1014E000803C8A00A0FD2800903D8A0060382B00D7
:1014F000B03D8A0000372B00A03D8A0060752900AE
:10150000C03D8A00803E2900D03D8A0020AE2A00DE
:10151000E03D8A0000CA2800F03D8A0080CC280007
:10152000003E8A00C0C82800103E8A0040CB280038
:10153000203E8A00A0CA2800303E8A0020CD280024
:10154000403E8A0060C92800503E8A00E0CB280057
:10155000603E8A0040302900703E8A00A032290097
:10156000803E8A00C0972600903E8A00C0D42800A2
:10157000A03E8A00C0972600B03E8A00C097260091
:10158000C03E8A00C0972600D03E8A00C097260041
:10159000E03E8A00C0972600F03E8A00C0972600F1
:1015A000003F8A00C0972600103F8A00C09726009F
:1015B000203F8A00C0972600303F8A00C09726004F
:1015C000403F8A00C0972600503F8A00C0972600FF
:1015D000603F8A00C0972600703F8A00C0972600AF
:1015E000803F8A00C0972600903F8A00C09726005F
:1015F000A03F8A00C0972600B03F8A00C09726000F
:10160000C03F8A000080FA00000006000200FA00D5
:10161000000F7800619781000181400080802000E8
:10162000000041001E0878000100E8006097890072
:1016300061978100F00320000080600060978900BE
:101640000080FA00000006000400FA0061978100A3
:1016500070978100808F500003003A000000EB007B
:10166000100798000D00370071978100018140003C
:101670008080200000004100100F78000100E80089
:101680007097890071978100F0032000008060004E
:10169000709789001E007800100798001E009000C7
:1016A0000080FA00000006000000FA000000EB00D5
:1016B0007097890070978100609789000080FA0018
:1016C000000006000200FA00000F780081978100F8
:1016D0000181400080882000000041001E08780041
:1016E0000100E8008097890081978100F0032000C5
:1016F00000806000809789000080FA0000000600EA
:101700000400FA008197810090978100808F50003B
:1017100003003A000000EB00100798000D003700AE
:1017200091978100018140008088200000004100E5
:10173000100F78000100E8009097890091978100D0
:10174000F003200000806000909789001E00780060
:10175000100798001E0090000080FA0000000600AC
:101760000000FA000000EB0090978900909781003C
:10177000809789000080FA00000006000400FA004B
:1017800010079800D762A9009E009000F0FF20008B
:1017900080806000000023000080700040128800FC
:1017A00040C2BF00614060000004E000FCFF320066
:1017B00040128000000F7800D762A8000080FA0075
:1017C000000006000400FA0010079800D762A90084
:1017D0009E009000F0FF20008080600000002B0041
:1017E000008070004012880040C2BF00614060006D
:1017F0000004E000FCFF320040128000000F78007F
:10180000D762A8000080FA00000006000000FA007D
:1018100020C3BF00614060000004E000FCFF320014
:101820002003A900001880000080FA0000000600D4
:101830001000FA00E0968100F1968100809FBE00C2
:10184000A08E2900801F78000E0078003818020052
:1018500000000000E68757000E0178008040EB0092
:1018600040C0B3007A710200000000008040EB002D
:1018700070C0B300B8730200000000000080FA00DE
:10188000000006001200FA00000F98000E089000F9
:10189000801F7800708F2900801F78000E0078006C
:1018A0003818020000000000E48757000E0178009D
:1018B0008040EB0040C0B3007A71020000000000DD
:1018C0008040EB0070C0B300B8730200000000005D
:1018D0000080FA00000006000000FA00100020005E
:1018E000B08089003191200010C0B300804878009A
:1018F0000080FA00000006000000FA000000EB0083
:10190000B0808900319120000040EB0080487800D1
:101910000080FA00000006000000FA00100020001D
:10192000250007000080FA00000006000000FA0011
:1019300050002000200007000080FA000000060090
:101940000000FA00200020001B0007000080FA00C1
:10195000000006000000FA00A000200016000700AA
:101960000080FA00000006000000FA000080EB0092
:10197000110007000080FA00000006000000FA00D5
:10198000B0FF2F000C0007000080FA0000000600E6
:101990000000FA00E0FF2F00070007000080FA00B7
:1019A000000006000000FA0060FF2F0002000700A0
:1019B0000080FA00000006000600FA0010079800F8
:1019C000D01982000000E00031003A00E0198200E6
:1019D000E70F500003003A000004200020079800A1
:1019E00002003700F0072000200798002E0090002A
:1019F000000F7800219781001E00900000804000B9
:101A000020978900209781000000E00002003D003F
:101A10000000EB0020978900209781009E0F500066
:101A2000020034001E00780020978900C04C80001E
:101A30000060A000C04C88000000EB00304C880023
:101A400020978100CF80DE00BA080200000000006D
:101A500002002000A31724009607020000000000E7
:101A600002002000A33F2400000802000000000044
:101A7000E0968900F19689006DFF0700E019820069
:101A8000E70F500002003A0076C20200000000009A
:101A90000080FA00000006001400FA00889FBE00D3
:101AA000D01982000000E0006C003A006000B8002D
:101AB00060079800710798006000B8004007980020
:101AC000510798006000B800008FBE00E0FF2F00B3
:101AD000F1FF2F00000F9800110F98002F00370022
:101AE000209781000002B0006101B9000E0890004B
:101AF0009E08900002004000838048008000400063
:101B000060262200008040001000780001002000C4
:101B10002007980031079800AE0090000E08900052
:101B2000000AB800AE0090001E0890000088B900BE
:101B300005017800000141008E0890003E009000F1
:101B40000088B90000014100820278006E00900018
:101B5000FE0090000000420081804A00600798006B
:101B6000710798004E019000DE0190002E00900059
:101B7000BE009000020040008380480040079800AB
:101B8000510798000E0890009E08900061004000E8
:101B9000E0804800000F9800110F98000E09900097
:101BA0009E0990002000200001002000800F5100BD
:101BB000818F5900CAFF34004E009000DE00900073
:101BC000E00F5000E08F58000E0032006E009000D1
:101BD000FE009000BA080200000000000004BE00F1
:101BE0004E009000DE009000BA08020000000000E5
:101BF0000001BE000800BE00120702000000000045
:101C0000008FBE00E0198200E60F50000B0032008A
:101C100002002000A31724001E00BE009607020049
:101C200000000000E2968100F396810000080200A7
:101C300000000000E0968900F1968900E09681009E
:101C4000F19681004C3C0200000000000000EB0017
:101C5000209689000000EB00309689004F04BE00FA
:101C60000080FA00000006000600FA009460A90057
:101C7000D0198200200798002E009000E10F50003C
:101C8000730032002E009000E30F5000700032000D
:101C90002E0090000000E00001003200A10037009B
:101CA00020268200E10F500002003A0010002000C0
:101CB00060198A00219681003096810000805000D2
:101CC000730040002096890020968100C203200006
:101CD000110009000200D8008000FD002096890054
:101CE0000000EB003096890000C1B300767202005C
:101CF000000000001072020000000000C28F2900E6
:101D00008040EB0020C0B3007A71020000000000A8
:101D10001A780200000000008040EB0070C0B300A1
:101D2000B873020000000000127A020000000000F8
:101D3000C0858100D185810070278A0081278A00B3
:101D4000C0858100D1858100604C8800714C88007D
:101D50000091200010407800E74F500003003A0047
:101D6000100020001007980002003700300020000B
:101D7000100798001E009000D0198A00902D2300B3
:101D8000104078000004E00005003A00A02D230078
:101D9000104078000004E00001003A00E222A800B0
:101DA0000000EB0030268A000000EB0040268A008D
:101DB0000000EB0030228A00519120000040EB002F
:101DC0008048780038FE070065FE0700F4680200CE
:101DD000000000000000EB003096890050802000D9
:101DE00010407800704060000004E0000C003200F9
:101DF00011C0B300D0C0B300567C02000000000048
:101E000011C0B300A0C0B300567C02000000000067
:101E10008000EB0010912900A08902000000000062
:101E20000091200010407800E74F500003003A0076
:101E300010002000000F7800020037003000200062
:101E4000000F78001E007800D0198A003500370096
:101E50000091200010407800E74F500002003A0047
:101E6000CC0207000200370040002000D0198A0091
:101E7000683D020000000000604C8000714C800052
:101E8000C0858900D1858900729229008040EB00CD
:101E900010C0B3007A7102000000000072922900A5
:101EA0008040EB0020C0B3007A7102000000000007
:101EB0002A710200000000004E71020000000000C4
:101EC0000000EB00309689008040EB0070C0B3004A
:101ED000B8730200000000000080200027FE070009
:101EE0005080200010407800704060000004E00046
:101EF0000C00320011C0B300D0C0B300567C020009
:101F00000000000011C0B300A0C0B300567C020066
:101F1000000000008000EB00D0932900A08902009F
:101F2000000000000CDE0200000000009460A80029
:101F30000080FA00000006000000FA005080200037
:101F400010407800704060000004E000170032008C
:101F5000D01982000000E00014003A0020002000A8
:101F6000D0198A008000EB0030952900A08902007A
:101F70000000000030C0B3003C0F0700D019820001
:101F80000000E00005003A008000EB00A096290068
:101F9000A089020000000000040037008000EB0070
:101FA00010982900A0890200000000000080FA00BB
:101FB000000006000000FA000080FA0000000600A1
:101FC0000000FA0080002000D0198A00C04C800078
:101FD00000F0A000C04C8800E0CC80004701070062
:101FE00040488800404880005048880040C0B30006
:101FF0001E0F07000080FA00000006000E00FA0025
:10200000E0CC80003D0107001007980000912000FF
:1020100010407800E74F500003003A000004200011
:1020200060079800020037008000EB00610798000D
:10203000EE0090001E009000E42502000000000069
:10204000104798001E409000E14F40006F003200A2
:10205000D01982000000E00007003A001E40900006
:10206000E34F500069003A00FFFE07001E00900099
:102070000000E800100798001000200020CD880024
:10208000D01982000041EB00324F9800E10F500060
:1020900002003A0010C0B300304F9800D0198200FF
:1020A0008040EB00214F9800E30F500002003A00FF
:1020B00012C0B300224F9800BE4890002E499000F5
:1020C00002C070000004E0004E0032000000EB008F
